:020000040800F2
:10000000F0C90220D1010008B57B0008573D000867
:10001000B7710008310E0008E98E000800000000EA
:100020000000000000000000000000000B89000834
:100030008D0F000800000000D77B000891890008A0
:10004000EB010008EB010008EB010008EB010008E0
:10005000EB010008EB010008EB010008EB010008D0
:10006000EB010008EB010008EB010008EB010008C0
:10007000EB010008EB010008EB010008EB010008B0
:10008000EB010008EB010008EB010008EB010008A0
:10009000EB010008EB010008EB010008EB01000890
:1000A000EB010008EB010008EB010008EB01000880
:1000B000EB010008E9890008218A0008EB0100082B
:1000C000EB010008EB010008EB010008EB01000860
:1000D000EB0100087D8E0008EB010008EB01000831
:1000E000EB010008EB010008EB010008EB01000840
:1000F000EB010008EB010008EB010008EB01000830
:10010000EB010008EB010008EB010008EB0100081F
:10011000EB010008EB010008EB010008EB0100080F
:10012000EB010008EB010008EB010008EB010008FF
:10013000EB010008EB010008EB010008EB010008EF
:10014000EB010008EB010008EB010008EB010008DF
:10015000EB010008EB010008EB010008EB010008CF
:10016000EB010008EB010008EB010008EB010008BF
:10017000EB010008EB010008EB01000800000000A3
:10018000EB010008EB010008EB010008EB0100089F
:10019000EB010008EB010008EB010008EB0100088F
:1001A000EB010008EB010008EB010008DFF80CD0C0
:1001B00000F0FCFB004800472DDC0008F0C90220DD
:1001C00030BF72B6704762B6704780F308887047D8
:1001D0000648804706480047FEE7FEE7FEE7FEE7E1
:1001E000FEE7FEE7FEE7FEE7FEE7FEE7958900088B
:1001F000AD0100082DE9F05F0546002092469B46C0
:1002000088460646814640241BE02846414647462C
:10021000224600F04AF953465A46C01A914110D37B
:1002200011461846224600F031F92D1A67EB0108F5
:100230004F4622460120002100F028F917EB000963
:100240004E41201EA4F10104DFDC484631462A4617
:100250004346BDE8F09F40EA01039B0703D009E055
:1002600008C9121F08C0042AFAD203E011F8013BA2
:1002700000F8013B521EF9D27047D2B201E000F8FB
:10028000012B491EFBD270470022F6E710B513463A
:100290000A4604461946FFF7F0FF204610BD421EED
:1002A00012F8013F002BFBD111F8013B02F8013B92
:1002B000002BF9D1704710B5002200E0521C835C7E
:1002C0008C5CA34201D1002BF8D1D8B2E1B2401A24
:1002D00010BD2DE9FE4F81EA030404F0004421F033
:1002E000004100944FF0000B23F0004350EA01045A
:1002F0005ED052EA03045BD0C3F30A54C1F30A553B
:100300002C44A4F2F3340194A0FB0254C1F3130172
:1003100041F48011C3F3130343F4801301FB02443F
:1003200000FB034E840A970A44EA815447EA835744
:10033000A4FB076802958D0A05FB07854FEA932CFD
:1003400004FB0C542705029D4FEA065847EA16376E
:10035000B5EB08056EEB070C870E920E47EA811786
:1003600042EA8312A7FB0201B6EB0B0164EB000427
:100370002B0D43EA0C335E1844EB1C50DA46514611
:10038000E7FB0201C5F313044FEA0B3343EA1453AE
:100390004FEA0432019C43EA0603A4F10C040294E0
:1003A000009CCDE900B400F025F903B0BDE8F08F62
:1003B00000200146F9E70EB540F2334102910021D9
:1003C000CDE900110A460B4600F014F903B000BD58
:1003D000C1F30A5210B5C1F3130140F2FF3341F4E7
:1003E00080119A4201DA002010BD40F233439A4254
:1003F000A2F2334203DC524200F057F810BD9040A5
:1004000010BD00F0004230F000400AD0C10D01F5EF
:100410006071C0F3160042EA0151C208400711435F
:10042000704700200146704701F0004330B421F0CE
:10043000004150EA010206D00A0DA2F56072C1F334
:100440001301002A02DC30BC00207047440F44EA4C
:10045000C104C100E01830BC00EBC25000F084B809
:1004600030B50B46014600202022012409E021FA84
:1004700002F59D4205D303FA02F5491B04FA02F581
:100480002844151EA2F10102F1DC30BD202A04DB54
:10049000203A00FA02F1002070479140C2F1200397
:1004A00020FA03F3194390407047202A04DB203AD6
:1004B00021FA02F00021704721FA02F3D040C2F184
:1004C0002002914008431946704700000FB40023F2
:1004D00000B589B00CA900910B996FF00042CB6078
:1004E0001E4B06931E4B07930423CDE901321D4A90
:1004F000089202466B46002000F002FB09B05DF84E
:1005000014FB70B586B006464FF0FF300091CDE980
:100510000101002015460C4604903246694604A8A5
:10052000FFF7D4FF02460498211825B108B1084608
:1005300000E020462860049800280DD0002A02DD43
:100540000098884208D0081B0094CDE90104324687
:10055000694604A8FFF7BAFF06B070BD390D000860
:10056000570D0008F50900080029A8BF7047401C76
:10057000490008BF20F00100704710B4B0FA80FCB9
:1005800000FA0CF050EA010404BF10BC704749B1F6
:10059000CCF1200421FA04F411FA0CF118BF012166
:1005A00021430843A3EB0C01CB1D4FEA00614FEA46
:1005B000102042BF002010BC704700EBC350104415
:1005C0000029A4BF10BC7047401C490008BF20F0A0
:1005D000010010BC704710B5141E73F1000408DA56
:1005E000401C41F1000192185B411A4301D120F0F7
:1005F000010010BD2DE9F04D92469B4611B1B1FAB4
:1006000081F202E0B0FA80F220329046FFF73EFF1E
:1006100004460F4640EA0A0041EA0B0153465A4697
:10062000084313D0114653EA010019D0C8F1400223
:100630005046FFF73AFF05460E4650465946424699
:10064000FFF724FF084305D0012004E02046394687
:10065000BDE8F08D0020054346EAE0762C433743A1
:100660000A986305E40AA0EB08000022FD0A44EAA8
:1006700047540A3002D500200146E9E70105101968
:100680006941DDE9084500196941BDE8F04DA2E77F
:100690002DE9FE4F804681EA0300C00F0C46009012
:1006A00021F0004123F00045B8EB0200A94105D23A
:1006B0004046214690461C460B46024623F0004029
:1006C000104347D0270DC7F30A00C3F30A51029025
:1006D000401A019040286BDAC3F3130040F4801BEA
:1006E0000098924620B10023D2EB030A63EB0B0B78
:1006F00001985946C0F140025046FFF7C7FE064632
:100700000D4650465946019A00F062F910EB080078
:100710006141002487EA115284EAE7731A4340D00A
:10072000009A62B3019A012A4FEA075215DC001BB6
:1007300061EB02014FF0004202EA0752CDE90042AC
:10074000001C41F5801132462B46FFF753FF03B0E2
:10075000BDE8F08F40462146F9E7001B61EB02013E
:10076000001C41F5801300185B412018A2F500170A
:1007700047EB030140EAD570B6196D4111E06D08F1
:100780004FEA360645EAC0754FEA0752001B61EB97
:100790000201001C41F5801149084FEA30000019A0
:1007A000514132462B4603B0BDE8F04FFFF713BF6F
:1007B0000098012240000023D0EB020263EBE073BB
:1007C000009821464FEAE074B8EB000061EB0401A9
:1007D000E9E783F000435BE781F0004158E72DE94A
:1007E000F04D81EA030404F0004B21F0004514466B
:1007F0004FF0000A23F0004150EA050220D054EAED
:1008000001021DD0C5F30A570246C5F31303C1F315
:100810001300C1F30A5640F4801543F48013A7EB8C
:100820000608101BD64608F2FD3873EB050002D30C
:1008300008F1010801E092185B41B8F1000F03DAFA
:1008400000200146BDE8F08D00204FF480110646DF
:1008500084460EE0171B73EB050705D3121B63EBF1
:10086000050306434CEA010C49084FEA3000921890
:100870005B4150EA0107EDD152EA030012D082EA4F
:10088000040083EA0501084305D0101BAB4106D2E2
:100890000122002306E000224FF0004302E06FF047
:1008A000010253101AEB06004CEB085110EB0A0042
:1008B00041EB0B01BDE8F04DFFF78DBE0EB5C10F4A
:1008C00080EAE0700844CA07002140F233438DE813
:1008D0000E000A460B46FFF78DFE03B000BD70B553
:1008E000C1F30A5201F000450024C1F3130140F2A4
:1008F000FF3341F480119A4201DA002070BD40F2CA
:1009000033439A42A2F2334203DC5242FFF7CDFD59
:1009100000E090402C43F1D0404270BDC1F30A5238
:10092000C1F3130140F2FF3341F480119A4202DA1D
:1009300000200146704740F233439A42A2F233420C
:1009400002DC5242FFF7B1BDFFF7A0BD30B5041E77
:1009500071F1000404DB4FF00044404264EB0101FC
:10096000141E73F1000405DB1C464FF00043524295
:1009700063EB04038B4208BF824230BD30B5041ED6
:1009800071F1000404DB4FF00044404264EB0101CC
:10099000141E73F1000405DB1C464FF00043524265
:1009A00063EB0403994208BF904230BD064C074DEB
:1009B00006E0E06840F0010394E80700984710342F
:1009C000AC42F6D3FFF7F6FB5C0604087C0604088D
:1009D000202A06DBCB17203A41FA02F043EAE07303
:1009E00006E041FA02F3D040C2F1200291400843F0
:1009F00019467047C0B24FF4F05100F0BDB9000085
:100A00002DE9FF4F087881B09946FF2805D0491C91
:100A10002D2804D00024002308E000230BE001244B
:100A2000F9E703EB830300EB4303491C0878FF2835
:100A3000F7D104B15B4200200090147801462D2CC0
:100A400001D02B2C04D1521C2D2C12D00024009448
:100A500000251678FF2E0ED00A24A0FB04C801FB47
:100A60000481002700FB0711521C16EB0C006941A2
:100A7000EFE70124EBE7994450EA01020ED000248D
:100A8000AA4D2646DFF8A88200F08AF982468B46F6
:100A9000B9F1000009DAC9F100071BE00198002153
:100AA000C0E9001105B0BDE8F08F074612E0F80775
:100AB00007D022462B4630464146FFF70AFC064641
:100AC000884622462B4610461946FFF702FC04468C
:100AD0000D467F10002FEAD1B9F1000F3246434690
:100AE0005046594602DAFFF77AFE01E0FFF7F1FBC4
:100AF000009A0AB181F00041019AC2E90001D1E7F0
:100B00002DE9FF4F1F468DB0D7E901464FF0FF3862
:100B10002E2045464FF000090B90B9696D1C0E98C8
:100B20008847396A824688470028F6D1BAF1FF3FE4
:100B30000AD024F4D064002E11DDBAF12B0F08D0B6
:100B4000BAF12D0F0BD102E0404611B0ABE744F4EF
:100B50008064B9696D1C0E9888478246761E694686
:100B6000600501D52D2000E02B208DF8000001F15B
:100B7000010B0DF1200809E0B9696D1C0E9888473A
:100B800082460F9844F40074761E0560002E02DD44
:100B9000BAF1300FF0D00B998A453ED144F0800471
:100BA00006E00F99681CA9F1010944F4007408607B
:100BB000B9696D1C761E0E98884782463028F0D0A1
:100BC0002BE00B998A4505D1200603D444F080041C
:100BD000761E18E0504608F0C9FE08B30DF1130167
:100BE000761E44F400748B4508D2AAF130000BF84D
:100BF000010B200607D5A9F1010003E0200602D46D
:100C000009F101008146A00502D50F99681C086012
:100C1000B9696D1C0E9888478246002ED1DC53E0DE
:100C2000002E51DDBAF1650F02D0BAF1450F4BD15C
:100C3000A00549D5B9696D1C24F44074761E0E9840
:100C400088478246002E0CDD2B2804D0BAF12D0FE8
:100C500007D144F48074B9696D1C0E9888478246A8
:100C6000761EE00501D52D2100E02B2108F8011B9F
:100C7000CDF82C8021E00DF12901761E44F400749A
:100C800088450CD2AAF1300010F0FF0088F800006F
:100C900002D10B99884509D908F1010806E0E00561
:100CA00001D5244801E042F20F708146B9696D1CFC
:100CB0000E98884782460F980560002E04DD504646
:100CC00008F054FE0028D6D1F9690E988847FF2015
:100CD0008BF8000088F800000020069007904B4633
:100CE0006A4608A906A8FFF78BFEA00502D46FF09C
:100CF00001002AE714F0240F0AD0E00714D1DDE93F
:100D000006123868031D3B600068C0E900120BE062
:100D1000DDE90601FFF788FB0146E00704D13868EA
:100D2000021D3A600068016028460EE7000024407A
:100D30000000F03FF1D8FFFF426842B1016811F8AE
:100D4000013B23B1521EC0E9001218467047012131
:100D5000C160881E704742685AB1C368016843B9D0
:100D600083688B4205D0491E521CC0E90012002046
:100D700070474FF0FF3070477F2801D9002208E00C
:100D8000064A02EB5002C007127800D1120902F0A5
:100D90000F02012090400840704700000000040846
:100DA0000EB540F2334202920022CDE900221346F2
:100DB000FFF720FC03B000BD70B58C1810F8015B84
:100DC00015F0070301D110F8013B2A1106D110F8E4
:100DD000012B03E010F8016B01F8016B5B1EF9D1E8
:100DE0002B0705D40023521E0DD401F8013BFAE76E
:100DF00010F8013BCB1A921C03E013F8015B01F8D9
:100E0000015B521EF9D5A142D8D3002070BD10B5A8
:100E100000230AE000EB8304D4ED000A02EB830414
:100E20005B1C70EE800AC4ED000A8B42F2DB10BD41
:100E3000FEE70000F0B500269FED101A1AE000252D
:100E400015E006FB0257B0EE410A002408E050F816
:100E500024C0641C0CEB870CDCED000A30EE800A29
:100E60008C42F4DB03EB87046D1C84ED000A954291
:100E7000E7DB761C9642E2DBF0BD000000000000DC
:100E800010B5DFED0A0A00230AE000EB830494EDBD
:100E9000001A02EB83045B1CD4ED001A41EE210A18
:100EA0008B42F2DB30EE800A10BD00000000000033
:100EB0002DE9F04F8046934603EBD37042108946EC
:100EC000514209EB410E1546A9EB020A2CE01446EB
:100ED00027E09FED170A002117E000206E18B61AD0
:100EE00010E02718BF1A06FB097C01FB030708EB7B
:100EF0008C0C0BEB8707DCED000A97ED001A401C09
:100F000000EE810A9842ECDB491C9942E5DBA11A0C
:100F1000AE1A06FB0E100999641C01EB800080EDEF
:100F2000000AA245D5DC6D1CAA45D0DCBDE8F08FD7
:100F3000000000000649087820B10020087018B1B0
:100F400004A102E00120F9E703A104A008F07CB9A4
:100F5000180300204F4E00004F46460044454255BE
:100F6000472049533A202573000000000FB406487B
:100F700010B50078002803D003A9029808F088F97A
:100F800010BC5DF814FB0000180300207047102A05
:100F90000FD0C26AD1E9002342EA03220B89097B00
:100FA0004FEA034343EA016142EA010203D1C2600E
:100FB00002E0C268EEE7C2624FF000007047102AFC
:100FC0000FD0826AD1E9002342EA03220B89097B10
:100FD0004FEA034343EA016142EA010203D182601E
:100FE00002E08268EEE782624FF000007047000086
:100FF00030B50A68102A1AD0026A104B02EA0302BE
:10100000D1E9013443EA0403D1E9034544EA050484
:1010100043EA04034C69896943EA442343EA4131C2
:1010200041EA020141F0080103D1016002E00268D7
:10103000E3E701624FF0000030BD00008101F0FFE6
:1010400070B5B3F5804F05D06FF0704140F82210B5
:10105000002070BD50F82230084C2340D1E90045F3
:1010600044EA05148D688E892D0245EA0645896992
:101070002C430C431C4340F82240E9E70000F0CF2A
:10108000F0B50C6850F82450194A1540D1E90123F5
:10109000D1E903671A433E4332434E6932438E69B6
:1010A0003243CE6932430E6A32434E6A32438E6A0D
:1010B0003243CE6A3243CE6B32430E6B32434E6BB9
:1010C00032432A43082B01D142F0400240F8242049
:1010D0004A6BB2F5801F08D10A6832B14FF48072B2
:1010E0000A6104490268114301600020F0BD00005C
:1010F0008000E0FF00011000F0B500EB82025368B1
:101100008E8903F04044D1E9003543EA05138D6828
:101110002D0245EA06452B430E8A0D4D05EB06567A
:1011200033430E7D6F0107EB066633438E6933430D
:10113000234353600268D20207D54268098A22F429
:10114000700205EB0151114341600020F0BD000029
:101150000000F0FF30B5D1E901231A43D1E903348F
:1011600023431A434B690D681A438B691A43D1E92B
:101170000734012D496A05686FF30E0505D01A433F
:1011800022430A432A43026008E0234329430B43D6
:10119000416803606FF30E010A434260002030BDD6
:1011A000426942EA4101416100207047F8B51446A6
:1011B0000546D1E9000210438A686FF01F03C96831
:1011C00003EB421242EA412108430090286100F0FB
:1011D00057FD064609E0601C07D024B100F050FD21
:1011E000801BA04201D90320F8BDA8698006F2D473
:1011F0000020F8BDF0B56FF00F05D1E9003405EB24
:1012000004145B1E2E0123438C682F0306EB042479
:101210004FEA054C23430D8A8E8ACC68097E4FF035
:101220007F4E07EB05450CEB06560EEB0161012ADC
:101230000CD082683F1107EB043423432B43334324
:1012400002F070420B43134383600FE0C2682B43EC
:101250000B4302F070428168134301F07042210396
:10126000A1F5805131431143C36081600020F0BD7E
:1012700038B50446094D4FF0AA300090A8790423F0
:1012800060436A46002106F085FCA8790423604388
:101290006A460021401C06F07DFC38BDD8180020AD
:1012A0002DE9FC47254F89460646002500240DF10F
:1012B000040810E0CDF80080798870438B084A4616
:1012C000002106F0FFFA7888BDF80410B1EB900F0A
:1012D00004D1641CA4B2B879A042EBD8B879A0427A
:1012E00002D10020BDE8FC87304606F0E5F820B1C9
:1012F000294613A007F0A8FF16E0B9F1FF3F13D06D
:1013000000200AE07A8806FB0010930800221146AC
:1013100006F016FCBDF80400401CADF80400B879D6
:10132000BDF804108842EDD86D1CADB2032DBDD3BD
:10133000314609A007F088FF0120D3E7D818002024
:101340006572726F7220657261736520626C6F6383
:101350006B3A25640D0A000062616420626C6F6361
:101360006B20636865636B65643A25640D0A000051
:1013700038B50446104D00208DF80000A8790123EF
:1013800060436A46002106F0D1FA9DF80000FF286C
:1013900001D0022038BDA879012360436A460021AC
:1013A000401C06F0C3FA9DF80000FF2801D0012080
:1013B00038BD002038BD0000D81800202DE9F84FB6
:1013C00091462F4A8A461D469179B0FBF1F3B0FB56
:1013D000F1F801FB130B404600F0B8F82849074626
:1013E0004889B84202D20120BDE8F88F002428E0E5
:1013F0005C4516D3ADB14A88A2EB0A01A94201D2DD
:101400008EB200E0AEB207FB004108FB00404B4645
:101410005246009605F0D0FE4FF0000AB144AD1BD5
:1014200005E007FB004108FB004005F099FF30B1E3
:101430003846FFF71DFF012000F024F8CBE7641CBD
:10144000A4B20F498879A042D2D80D46A879A0420B
:1014500014D1384600F028FA404606F02DF8002056
:101460006A89696908E031F81040444502D121F8E1
:10147000107003E0401C80B28242F4D80020B3E731
:10148000D8180020F8B506460021294D4FF6FF7008
:1014900003E06A6922F81100491C6A898A42F8D877
:1014A0000020A88104461CE0A879042360436A4612
:1014B000002106F03BFA9DF80000FF280CD1B6B1E0
:1014C000A879012360436A460021401C06F02EFAE9
:1014D0009DF80000FF280AD0214616A007F0B4FEB0
:1014E000641C6989A142DFD800206A6916E09DF872
:1014F00002009DF8031000EB01206989814202D9A6
:10150000696921F81040A889401CA881E8E732F8F1
:1015100010308B4201D3E88102E0401C8142F6D8B2
:10152000E889642801D20220F8BD0020F8BD00003F
:10153000D818002062616420626C6F636B20696E52
:101540006465783A25640D0A0000000070B5104EFD
:10155000104C71892268491E914200D2216000F02E
:1015600001052946206800F017F8411C0AD170894E
:101570002168401E884207D92946206000F00CF8F7
:10158000411C01D0206070BD4FF0FF3070BD0000E5
:10159000D818002038000020F8B50D460021401C66
:1015A0000091040012D00C4F012626EA0400A84244
:1015B0000AD1B879611E484304236A46002106F027
:1015C000B5F90098401C04D0641EEED14FF0FF30F6
:1015D000F8BD601EF8BD0000D8180020F8B5254EF3
:1015E00000273C46B78113E02046FFF7C1FE70B9E3
:1015F000204605F061FF38B121461FA007F024FE08
:101600002046FFF735FE02E0B089401CB081641C23
:101610007089A042E8D8B1891BA007F015FEB089F7
:10162000642801D20120F8BDC0EB4010642100EB1A
:101630004000B0FBF1F50024009710E02046FFF7D2
:1016400097FE58B9B079022360436A46194606F0FE
:10165000A1FA0098401C0090A84203D0641C708935
:10166000A042EBD80120FFF70DFF0028DBD00220BD
:10167000F8BD0000D818002042616420626C6F63DE
:101680006B3A25640D0A0000676F6F645F626C6FD0
:10169000636B6E756D3A25640D0A000010B505F098
:1016A0005FFF00BB184C616911B100200DF04AFFCB
:1016B0006089410000200DF051FF6061618949009F
:1016C000FEF7E2FD606970B10120FFF7DBFE60B15B
:1016D0000EA007F0B9FDFFF781FF90B111A007F050
:1016E000B3FD022010BD012010BD618912A007F0DA
:1016F000ABFDA18916A007F0A7FDE18919A007F0AD
:10170000A3FD002010BD0000D8180020666F726D88
:101710006174206E616E6420666C6173682E2E2E7B
:101720000D0A0000666F726D6174206661696C65F8
:1017300064210D0A00000000746F74616C20626CFB
:101740006F636B206E756D3A25640D0A0000000012
:10175000676F6F6420626C6F636B206E756D3A25E6
:10176000640D0A0076616C696420626C6F636B20A3
:101770006E756D3A25640D0A000000000549CA899E
:10178000824202D24FF6FF707047496931F810006B
:1017900070470000D81800202DE9FF5F9B461546D2
:1017A0008246002679E03F4C6088B0FBF5F1A079D5
:1017B000414301988319B3FBF1F0FFF7DFFF618923
:1017C000814203D8012004B0BDE8F09F354C618808
:1017D000A479B1FBF5F26243B3FBF2F702FB1732D7
:1017E0006A43B2FBF1F300FB0437B2FBF1F001FBFB
:1017F0001028A1EB0800B0FBF5F084B2ABEB0600BB
:10180000A04200D284B204FB05F91FFA89F31FFA43
:1018100088F15246384605F037FF032809D11FFAF0
:1018200089F31FFA88F15246384605F02DFF032848
:1018300004D004282ED068B30220C4E74B461FFA18
:1018400088F152463846FFF7B9FDDFF858804FF06F
:10185000FF3198F80600B7FBF0F0FFF721FD80B9E3
:1018600098F806000021B7FBF0F0FFF719FD81465C
:1018700098F80600B7FBF0F005F01EFEB9F1000F76
:1018800008D098F80600B7FBF0F0FFF7F1FC012054
:10189000FFF7F8FD05FB04AA26445E4583D300202C
:1018A00091E70000D818002008B5CC218DF8001071
:1018B000044901236A4689794843194606F06AF9C2
:1018C00008BD0000D81800202DE9FF4F85B015464F
:1018D00000274FF0FF3B7BE0404C6088A179B0FBD4
:1018E000F5F048430699CB19B3FBF0F0FFF746FF3C
:1018F00061898046414503D8012009B0BDE8F08FD9
:10190000364A50889279B0FBF5F15143B3FBF1F4BC
:1019100001FB143101FB05FABAFBF0F308FB0231BD
:10192000BAFBF0F200FB12A9A0EB090080B2B0FBF9
:10193000F5F002910899ADF80400C91B8CB203912F
:10194000844200D3044601A804FB05F600901FFA68
:1019500089F1C6F38F034FF0FF32029805F0B2FF12
:1019600008B10220C9E7BDF80400B0EB960F0FD113
:10197000B3B21FFA89F1059A029806F035F838B922
:101980004146C34520D00846FFF78EFFC346D8B175
:101990001248817940884143A1EB0A00B0FBF5F081
:1019A000039980B28CB2ADF80400844200D304469F
:1019B00004FB05F61FFA89F13346059A0298FFF7F2
:1019C000FDFC08B1032098E70598274430440590B2
:1019D0000898874280D300208FE70000D8180020A5
:1019E000F0B500261AE0002506FB02FC13E00024F7
:1019F0000EE005FB024750F826E0641C0EEB870E54
:101A00000CFB02779EED000A03EB870787ED000AC7
:101A10009442EEDB6D1C9542E9DB761C8E42E2DBE4
:101A2000F0BD0000F0B500238D1C9FED120A05FBF0
:101A300005F404E002EB83065B1C86ED000A9C4281
:101A4000F8DC002412E00023661C0CE004FB0137E4
:101A500000EB870797ED000A06FB053702EB8707C7
:101A60005B1C87ED010A8B42F0DB641C8C42EADBD5
:101A7000F0BD00000000000031B500F001F904469F
:101A800000F0FEF80099001B8842F9D338BD000031
:101A90002DE9F84FDFF8A091002209F1040A0AF1BC
:101AA000040B4FF00F080BF1040E01260B68964053
:101AB0003340B34271D14C68022C01D0122C11D1A9
:101AC000D40800EB84073D6A5407E40E08FA04FCCE
:101AD00025EA0C05D1F810C00CFA04FC4CEA050C00
:101AE000C7F820C007685400032591F804C0A5403A
:101AF0000CF0030CAF430CFA04FC4CEA070CC0F8E2
:101B000000C04F68012F05D0022F03D0112F01D044
:101B1000122F11D18768D1F80CC0AF430CFA04FC26
:101B20004CEA070CC0F808C04768B7430E79C6F303
:101B3000001696403E434660C668AE438D68A54099
:101B40003543C5604C68E4006FD53C4C256845F4CE
:101B500080452560246822F0030504F48044009445
:101B6000374C2E19D6F808789407250F08FA05F493
:101B7000A743344CA04201D100242EE0324CA042B5
:101B800001D1012429E0314CA04201D1022424E0FA
:101B90002F4CA04202D103241FE046E02D4CA0426E
:101BA00001D1042419E02C4CA04201D1052414E0F9
:101BB0002A4CA04201D106240FE0294CA04201D1B9
:101BC00007240AE0274CA04201D1082405E0264C56
:101BD000A04201D1092400E00A24AC403C43C6F8ED
:101BE0000848D9F800404D464E689C43F60300D59E
:101BF0001C432C60DAF8004055464E689C43B603FF
:101C000000D51C432C60DBF800405D464E689C43C9
:101C1000F60200D51C432C60DEF8004075464E6885
:101C20009C43B60200D51C432C60521C102AFFF4C2
:101C30003CAFBDE8F88F0000003C01404438024052
:101C40000030014000000240000402400008024051
:101C5000000C024000100240001402400018024034
:101C6000001C02400020024000240240006908409D
:101C700000D0012070470AB1816170470904FBE779
:101C80000148006870470000140000200248016805
:101C9000491C016070470000140000200B4810B57B
:101CA000016841F400710160016841F480610160E4
:101CB000016841F480710160052000F049FA0F20AD
:101CC00000F006F800F08AF9002010BD003C024048
:101CD00010B5044600F0EAFC4FF47A71B0FBF1F065
:101CE00001F0B8FD00222146501E00F011FA00203C
:101CF00010BD2DE9F041044690F8A00015460F46AE
:101D000001281DD0012684F8A060022084F8A100DB
:101D100005EB850000EBC50004EB80003422383071
:101D2000FEF799FA2A463946204605F093F92068CD
:101D3000466284F8A160002084F8A000BDE8F0812C
:101D40000220FBE770B5040004D094F8A100002540
:101D500010B106E0012070BD84F8A050204600F0CC
:101D60006FF8022084F8A1002068816921F0704199
:101D70008161D4E901100143D4E903021043014316
:101D80002068826911438161206882682B490A407A
:101D90008260A08A020420688368A66933431343E3
:101DA00083602068C2680A40C260A08B0204206879
:101DB000C368266A33431343C360206802690A403C
:101DC0000261A08C020420680369A66A33431343AE
:101DD0000361206842690A404261A08D01042068C5
:101DE0004269236B1A430A43426194F835000202A8
:101DF00094F8360001042068C36A03F07F43C3628D
:101E00002068C36A94F83460114333430B43C362C0
:101E10002068416B41F0040141632068416B41F04F
:101E2000020141632068816941F001018161C4F8C8
:101E3000A450012084F8A100002070BD00F800F03B
:101E400030B5364887B00025016841F080610160F7
:101E5000006800F08060059030481438016841F453
:101E600000010160016801F400010591016841F081
:101E700002010160016801F002010591016841F071
:101E800020010160016801F020010591016841F025
:101E900040010160016801F040010591016841F0D5
:101EA00080010160016801F080010591016841F441
:101EB000807101600068032400F480700590202088
:101EC00000900120CDE90204019069461448FFF713
:101ED000DFFD4FF4806000900220CDE901050E2067
:101EE000CDE9034069460F48FFF7D2FD4FF40C607F
:101EF000009069460C48FFF7CBFD4FF47E40009000
:101F000069460A48FFF7C4FD40F2F7600090694651
:101F10000748FFF7BDFD07B030BD00004438024060
:101F2000000402400014024000180240001C02405D
:101F30000020024070B5044690F8A0000E4601282B
:101F400020D0012584F8A050022084F8A10003EBE2
:101F5000830000EBC30004EB800141F8386F886A0E
:101F60003044C1E90102C86A1044C8601A462046DC
:101F700005F070F82068456284F8A150002084F8CC
:101F8000A00070BD022070BD2DE9F041044690F81C
:101F9000A0000F4601281FD0012584F8A050022080
:101FA00084F8A10003EB830000EBC30004EB800185
:101FB0000026E1E90E672046C1E90262C1E90A7222
:101FC0001A4605F047F82068456284F8A15084F865
:101FD000A0600020BDE8F0810220FBE708B50020EA
:101FE000009008BD70B515460E46040003D094F865
:101FF000210010B107E0012070BD002084F820000E
:10200000204600F021F8211D2068FEF7F1FFD4E9F9
:1020100000023146FEF7D3FFD4E900022946FEF75D
:10202000B6FF60681028206808D0016A41F00401FA
:102030000162012084F82100002070BD016841F098
:1020400004010160F5E7000070B5274886B0002460
:10205000016841F001010160006800F00100059095
:1020600021480838016841F008010160016801F069
:1020700008010591016841F010010160016801F05B
:1020800010010591016841F04001016000680325DD
:1020900000F0400005904020CDE900040120CDE98A
:1020A0000205124E69463046FFF7F2FC70150090AB
:1020B00001A9022081E831000C20049069460C48F7
:1020C000FFF7E6FC4DF63300009069460294304677
:1020D000FFF7DEFC4FF4F060009069460548FFF71B
:1020E000D7FC06B070BD000038380240000C02403A
:1020F000001802400010024000F01F020121914030
:102100004009800000F1E020C0F800117047000095
:10211000F0B40E4B1B68C3F30223C3F10704042C75
:1021200000D904241D1D072D01D2002300E0DB1E71
:10213000012606FA04F56D1E0D409D409E40761E58
:10214000164045EA0601F0BC05F035BD0CED00E097
:10215000064A00F0070110684FF6FF03184040EAF6
:102160000120034908431060704700000CED00E0B7
:102170000000FA052DE9F8431D48016841F080513F
:1021800001600068012700F080500090380490FA48
:10219000A0F0DFF86080B0FA80F048F82070FFF718
:1021A0006FFD04464FF47A75134E04E0FFF768FDA7
:1021B000001BA84213D87068C003F7D54FF4003055
:1021C00090FAA0F0B0FA80F048F82070FFF758FDC0
:1021D000044607E0FFF754FD001BA84202D9032084
:1021E000BDE8F88370688003F4D50020F8E70000AC
:1021F0004038024000000E42007000402DE9F84FC8
:1022000004460068DFF878829E4DC10747F6C07A21
:102210004FF0E0464FF0010B4FF0000901D180076D
:102220004BD59949C1F86890FFF72AFD074604E0AD
:10223000FFF726FDC01B64287ED828680001F7D46C
:1022400020789249C0070DD09AFAAAF26068B2FAD3
:1022500082F2904096FAA6F3A268B3FA83F39A400A
:10226000104308602078800718D5086896FAA6F20F
:1022700000F0E040B2FA82F2D0406268237B920123
:1022800042EA036242EA00700860D8F80010E2698E
:1022900021F01F01521E1143C8F800107A49C1F8FD
:1022A00068B0FFF7EDFC074604E0FFF7E9FCC01B50
:1022B000642841D828680001F7D52068410701D477
:1022C000000776D57049C1F87090FFF7D9FC074632
:1022D00004E0FFF7D5FCC01B64282DD82868C04354
:1022E0008000F6D520786A4F40074FF0706C29D5F2
:1022F000386896FAA6F100F0E040B1FA81F1C840E2
:102300009AFAAAF22169B2FA82F291409CFAACF3ED
:102310006269B3FA83F39A40114396FAA6F2B2FACD
:1023200082F2904001433960D8F800106FF0FF034B
:1023300021F4F851226A00E079E003EB0222114314
:10234000C8F800102078000723D538689CFAACF153
:1023500000F07060B1FA81F1C8409AFAAAF22169DE
:10236000B2FA82F291409CFAACF2B2FA82F2904058
:10237000014396FAA6F2A069B2FA82F290400143B4
:102380003960D8F80010626A21F440311143C8F86E
:1023900000103D49C1F870B0FFF772FC064604E03A
:1023A000FFF76EFC801B642841D82868C04380007A
:1023B000F6D42078800651D532484F464030016827
:1023C00041F0805101600068324E00F08050009072
:1023D000306840F480703060FFF752FC054604E03E
:1023E000FFF74EFC401B642821D83068C005F7D5A4
:1023F000264E143E3068218D00F4407001F4407187
:1024000088422BD03068244920F44070C1F800B0D5
:102410000F603060800710D5FFF732FC054641F2AF
:10242000883707E0FFF72CFC401BB84202D9032095
:10243000BDE8F88F30688007F4D5A06A1149C0F371
:1024400001220831032A13D0086820F4F81008602C
:102450003068218DC1F30B01084330602078C0063D
:1024600004D50E4994F82C00C1F8E0010020DFE704
:102470000A680B4B22F4F812184002430A60E7E79F
:102480008C38024000380240000047428438024045
:102490008838024000700040400E4742001047421A
:1024A000FFFCFF0F2DE9F05FDFF8F8A104460F46AF
:1024B000DAF80000DFF8F08100F00F02C8B27A49C4
:1024C000814641F2883608F10808BA4261D20246D4
:1024D0008AF80020DAF8000000F00F00B8427DD141
:1024E0002078800707D5D8F80020A36822F0F002F2
:1024F0001A43C8F800202078C0072DD06068012852
:102500001AD002281BD0032819D00968890700298E
:1025100064DAD8F80010474621F003010143C8F8F7
:102520000010FFF7ADFB0546606801280FD00228B8
:1025300018D003281CD027E009688903E7E7096859
:102540008901E4E7FFF79CFB401BB04258D838688C
:10255000C0F381000128F5D188E0FFF791FB401B13
:10256000B0424DD83868C0F381000228F5D17DE033
:102570003868FFF785FB401BB042F9D940E0FFF710
:102580007FFB401BB0423BD8386810F00C0FF6D1EF
:102590006CE02078800707D5D8F80020A36822F0E7
:1025A000F0021A43C8F800202078C0074CD06068B9
:1025B000012828D0022829D0032827D009688907B4
:1025C000002949DAD8F8002022F003020243C8F8B3
:1025D0000020FFF755FB0546606800E03CE001285D
:1025E0001DD0022829D0032838D0B346464630688B
:1025F00010F00C0F28D0FFF743FB411B5945F6D9CB
:102600000320BDE8F09F09688903D9E709688901BB
:10261000D6E7FFF735FB411B594502D9F0E7B34632
:1026200046463068C0F381000128F2D10CE0FFF784
:1026300027FB411B594502D9E2E7B34646463068BD
:10264000C0F381000228F2D18AF80090DAF8000085
:1026500000F00F00B84209D00120D2E744462068BC
:10266000FFF70EFB401BB042F9D9C9E720784007BD
:1026700007D5D8F80010E26821F4E0511143C8F8FA
:1026800000102078000708D5D8F80010226921F43E
:10269000604141EAC201C8F800100F20FFF718FBA3
:1026A0000020AEE7003C02400038024010B500F0C8
:1026B00043F808490968F02292FAA2F201F0F00109
:1026C000B2FA82F2D140044A515CC8400349086022
:1026D00010BD0000083802402E0C01080000002048
:1026E00010B5FFF7E3FF074909684FF4E05292FA8B
:1026F000A2F201F4E051B2FA82F2D140024A515CF6
:10270000C84010BD083802402E0C010810B5FFF774
:10271000CDFF074909684FF4604292FAA2F201F432
:102720006041B2FA82F2D140024A515CC84010BD09
:10273000083802402E0C010830B51948006810F026
:102740000C01184812D0184C04290ED008290DD1BC
:10275000134A121F1168136801F03F015D0247F62A
:10276000C07304D5B4FBF1F003E0204630BDB0FBEC
:10277000F1F01168194093FAA3F3B3FA83F3D94047
:10278000484311684FF4403292FAA2F201F440310A
:10279000B2FA82F2D140491C4900B0FBF1F030BDE1
:1027A000083802400024F40040787D012DE9F84FFC
:1027B00004460078DFF8FCA2BF4DC0074FF00006CA
:1027C00048D0DAF800105046C1F38101012908D041
:1027D0000068C0F3810002280AD1281D0068400269
:1027E00006D52868800335D56068002873D031E0AD
:1027F000DFF8C49209F1020989F80060FFF740FA96
:10280000074641F2883804E0FFF73AFAC11B414518
:102810007AD828688003F7D4207989F800006068A6
:1028200060B1FFF72DFA074604E0FFF729FAC11B54
:102830004145EDD828688003F7D50BE0FFF720FA73
:10284000074604E0FFF71CFAC11B4145E0D82868A1
:102850008003F7D42078DFF86492800744D5DAF853
:102860000010504611F00C0F4FF0F80809D0006826
:10287000C0F3810002280BD18E48001F006840027F
:1028800006D42868800714D5E068012823D110E019
:10289000E068D0B10120C9F80000FFF7F1F9074660
:1028A00004E0FFF7EDF9C01B6428B1D82868800761
:1028B000F7D5286898FAA8F22169B2FA82F220F0D6
:1028C000F8009140084328600EE0C9F80060FFF767
:1028D000D7F9074605E0EAE0FFF7D2F9C01B642804
:1028E00012D828688007F7D42078000725D5DFF8AC
:1028F000C4817348616908F16C0881B101210160EC
:10290000FFF7BEF9074605E07EE0FFF7B9F9C01B07
:10291000642879D8D8F800008007F6D50DE0066065
:10292000FFF7AEF9074604E0FFF7AAF9C01B6428D9
:102930006AD8D8F800008007F6D42078400753D52D
:102940005C483830016841F0805101600068DFF870
:10295000748100F080500090D8F8001041F480712C
:10296000C8F80010FFF78CF9074604E0FFF788F974
:10297000C01B642848D8D8F80000C005F6D5DFF899
:1029800034B10BF1680B8BF80060FFF779F907465B
:1029900041F2883804E0FFF773F9C11B41457ED846
:1029A000DBF800008007F6D4207A8BF80000A068DE
:1029B00068B1FFF765F9074604E0FFF761F9C11B4D
:1029C00041456CD8DBF800008007F6D50CE0FFF736
:1029D00057F9074604E0FFF753F9C11B41455ED89C
:1029E000DBF800008007F6D4A069E8B3DAF800103D
:1029F000C1F3810102295AD0022806D0C9F86060CB
:102A0000FFF73EF904464DE049E04F46C9F86060E3
:102A1000FFF736F9064604E0FFF732F9801B642819
:102A20003DD828688001F7D4D4E90701084347F668
:102A3000C07191FAA1F1626AB1FA81F18A40A16A8A
:102A40004FF0FF3303EB51014FF4403393FAA3F3FC
:102A5000B3FA83F399400A4310434FF0706292FA3D
:102A6000A2F2B2FA82F200E01FE0E16A914008436C
:102A70001049091F086001203866FFF701F9044674
:102A800004E0FFF7FDF8001B642808D828688001DF
:102A9000F7D50AE0FFF7F4F8001B642802D90320F9
:102AA000BDE8F88F28688001F4D40020F8E7012001
:102AB000F6E70000083802400038024000004742B4
:102AC000800E47420070004070B50D46040003D0F0
:102AD00094F82C0010B107E0012070BD002084F8AC
:102AE0002D00204600F012F8022084F82C00211D51
:102AF0002068FEF72FFBD4E900022946FEF77AFB97
:102B0000012084F82C00002070BD0000304800B582
:102B1000016887B041F001010160006800F0010028
:102B200005902B480838016841F0040101600168F4
:102B300001F004010591016841F00801016001689C
:102B400001F008010591016841F010010160016880
:102B500001F010010591016841F020010160016858
:102B600001F020010591016841F040010160006819
:102B7000694600F0400005900D2000900220019071
:102B800001200290032003900C2004901148FEF7CE
:102B90007FFF4CF20370009069460F48FEF778FF04
:102BA0004FF68370009069460C48FEF771FF4FF6B0
:102BB0003F00009069460A48FEF76AFF48F2371066
:102BC000009069460748FEF763FF07B000BD0000AC
:102BD0003838024000080240000C02400010024059
:102BE000001402400018024010B5044690F82C0072
:102BF000022809D0022084F82C002068FEF7D0FAC1
:102C0000012084F82C00002010BD70B5044690F817
:102C10002C000D4602280CD0022084F82C002068DD
:102C2000FEF7C4FA2868022804D0012084F82C009A
:102C3000002070BD0520F9E72DE9F04790F820202D
:102C400081F85620828CA1F85420826A0023120E4B
:102C500094090C70C2F383044C7002F003028A7072
:102C6000826A120CCA70028D120A0A7190F828202A
:102C70004A71C26A4FF6FF7A120E0AEA0212CA803D
:102C8000C26ACC88C2F3074244EA1214CC8002F034
:102C90000F020A72828DC2F30722D4094C72C2F36A
:102CA00080148C72C2F34014CC72C2F300140C7303
:102CB00000264E73046A4FF00109002C7DD0012CD0
:102CC000FCD0022C7AD02923C2F380144C769206D1
:102CD000520E01F81A2F10F8302F0C7844EAD21453
:102CE00001F8014B02F07F0201F8012B50F8042F8C
:102CF000120ED4090C70C2F341144C70C2F382045A
:102D00008C709207120FCA7004C8CC78C2F30742C5
:102D100044EA9214CC70C2F340140C714E7102F06C
:102D200001028A7130F8042CC2F30722D409CC7155
:102D3000C2F380140C72C2F340144C72C2F300143C
:102D40008C72C2F38104CC7202F003020A7310F891
:102D5000042C52084A734C4681F80E9050F8082B08
:102D6000120E0A7450F8082C120C0AEA02224A8247
:102D700030F8082C4D8AC2F3072215434D8210F813
:102D8000082C120641F8142F50F8042C0D68120E6E
:102D900045EA02420A6050F8042C0D68C2F307426B
:102DA00045EA02220A6030F8042C0D68C2F30722BB
:102DB000154320C110F8042C01E034E076E001F85E
:102DC000012B0268120E01F8032B0268120C120686
:102DD0000A6002880D68C2F3072245EA02420A60CF
:102DE00002780D6845EA02220A6042680D6845EAE9
:102DF000126520C142680D78C2F3074245EA1215F8
:102E000001F8025B1207120D0A8082880D88C2F356
:102E10000722154321F8025B0079400808704C70C6
:102E20001846BDE8F0879207120D0A6190F82C2031
:102E30000C6944EA82020A61026B0C69120E44EAD0
:102E400092140C61C2F3C2040C7502F007024A75B9
:102E5000026BC2F3074254098C75C2F38204CC752D
:102E60009207520F0A76028E0C7EC2F3072244EAC2
:102E7000D2140C760C690F7EBF1C09FA07F5641C8E
:102E8000A4FB05784FEAE57C06FB058504FB0C55A1
:102E900091F808C009FA0CF4A7FB04C80C6505FBFF
:102EA000048407FB0644C1E912C40DE790F82C2006
:102EB0009206920A0A61026B0C69120E44EA02221F
:102EC0000A61026B0C69C2F3074214430C61028E63
:102ED0000C69C2F30722641C46F10005ED0445EAC3
:102EE0005435E404C1E912454FF400740C65EBE677
:102EF00070B586B000250E4604468DF80C50057757
:102F000000F046F876200095CDE901502B462A4680
:102F10002946206804F012FF204605F0A1FA8DF83A
:102F20000C009DF80C0038B9204605F08DF98DF89D
:102F30000C009DF80C0018B19DF80C0006B070BD97
:102F400031462046FFF778FE8DF80C009DF80C0006
:102F5000A0B9B6F85400694600040090072001901B
:102F60004020CDE9020500010490206804F0FFFE36
:102F70000721204604F0DAFF8DF80C0004F1100060
:102F800007C88DE8070094E80F0004F0D7FED3E7E8
:102F90001D4800B5016887B041F400610160006818
:102FA00000F40060059018481438016841F480016D
:102FB0000160016801F480010591016841F004019C
:102FC0000160016801F004010591016841F0080108
:102FD00001600068694600F0080005904FF4F85061
:102FE00000900220019001200290032003900C2009
:102FF00004900648FEF74CFD042000906946044802
:10300000FEF746FD07B000BD44380240000802400C
:10301000000C02402DE9F04F8BB004460D46DDE96F
:103020001478216800201646C862216A022903D15B
:103030000F02560A46EAC3561021CDE9007140211D
:10304000834608010291CDE903B06946206804F087
:103050008EFE1021204604F069FF00286DD14FF04C
:10306000FF3A08FB07F0CDE905A007A990204FF033
:10307000020981E8010A01200A9005A9206804F0EC
:103080003BFEB8F1010F01D9122000E01120CDE97B
:1030900000606946206804F06AFEB8F1010F1AD991
:1030A0001221204604F042FF070046D140F22A3B9D
:1030B0002068416B11EA0B0F28D1406B0004F7D553
:1030C0000026206804F050FE45F82600761C082EE5
:1030D000F7D32035ECE71121204604F027FF070045
:1030E0002BD140F22A6B2068416B11EA0B0F0DD1F6
:1030F000406B0004F7D50026206804F035FE45F843
:103100002600761C082EF7D32035ECE7406BC0056F
:103110000CD5B8F1010F09D9206A18B1012801D0E6
:10312000022803D1204600F033F807462168486B97
:10313000000705D50820886304200BB0BDE8F08F98
:10314000486B800703D54846C1F83890F5E7486BCF
:10315000800603D5202088630620EEE7486B8005B3
:1031600004D54FF4007088630720E6E7564603E075
:1031700004F0FAFD01C5761E2068416B890201D575
:10318000002EF5D1216840F2FF5088633846D4E71D
:1031900010B586B0044600200C21CDE90001402185
:1031A000CDE90210080104906946206804F0DFFDB3
:1031B0000C21204604F0BAFE06B010BDFEB5044650
:1031C000006A00250E46032805D030B1012804D03E
:1031D000022802D01FE02720FEBDB6F5805F05D093
:1031E000B6F5006F04D03EB1262514E0272512E085
:1031F000204605F070FA02E0204605F033FA05009B
:1032000009D1211DD4E905070EC9CDE90060029757
:10321000206804F093FD2846FEBD2DE9F04F8DB0E7
:10322000064600250C468DF82C50DDE916983168CD
:1032300017462846CD62316A4FF4007B022903D13C
:10324000570AD94647EAC3571021CDE900914021DA
:10325000824608010291CDE903A06946306804F076
:1032600086FD1021304604F061FE00286ED1B8F1D1
:10327000010F01D9192000E01820CDE9007069463E
:10328000306804F074FDB8F1010F01D9192100E094
:103290001821304604F04AFE00287FD1411E09FB68
:1032A00008F99020CDE906900591CDF820A00120E5
:1032B000CDE909A005A9306804F01EFDB8F1010FA1
:1032C00024D84FE0406B400420D5A9EB050020280E
:1032D00011D281074FEA900000D0401C824600279F
:1032E00006E02146306804F052FD241D2D1D7F1C90
:1032F00057450BD2F5E7002704EB8701306804F04F
:1033000046FD7F1C082FF7D3203420353068416BF1
:1033100040F21A321142D5D02AE0406B400421D548
:10332000A9EB0500202812D281074FEA900000D0B7
:10333000401C8246002706E02146306804F027FD45
:10334000241D2D1D7F1C57450CD2F5E726E00027D4
:1033500004EB8701306804F01AFD7F1C082FF7D3B7
:10336000203420353068416B40F21A621142D4D0CB
:10337000406BC0050BD5B8F1010F08D9306A18B100
:10338000012801D0022802D13046FFF701FF316841
:10339000486B000705D50820886304200DB0BDE800
:1033A000F08F486B800702D502208863F6E7486BF0
:1033B000C00603D5102088630520EFE7486B800521
:1033C00003D5C1F838B00720E8E740F2FF50886322
:1033D0000BA9304604F0A6FF0028DFD19DF82C1081
:1033E0000729F5D00629F3D0D8E770B5040004D03A
:1033F00094F85100002510B106E0012070BD84F85A
:103400005050204600F034F8022084F85100206823
:10341000016821F040010160D4E901010843D4E9C9
:1034200003121143084361690843218B01F40071C1
:103430000843E1690843216A0843A16A08432168F7
:103440000860A069042101EA1040616A084321680C
:1034500048602168E06A08612068C16921F4006160
:10346000C1616565012084F85100002070BD000035
:10347000124800B5016887B041F020010160006882
:1034800000F0200005900D481430016841F48011CF
:1034900001600068012100F4801005904FF4607015
:1034A00000900220CDE901010390052004906946B7
:1034B0000348FEF7EDFA07B000BD000030380240C7
:1034C000001402402DE9F843044690F85100DDF85D
:1034D0002080012801D022287ED169B162B15BB180
:1034E00094F85000012877D0012784F8507094F8A0
:1034F0005100012803D005E00120BDE8F883322007
:1035000084F8510000266665A263A387E3872163E0
:10351000A386E386A664E664A06A4FF40055A84239
:1035200009D12068016821F4005101602068016818
:1035300041F40051016020680168490603D4016824
:1035400041F040010160E0684FF48271B0F5006F16
:10355000606807D0002867D088426ED1E08E0128CD
:1035600062D06AE020B188420CD1E08E012809D1F6
:10357000206B21680088C860206B801C2063E08E6F
:10358000401EE086E08E80B9A06AA84244D120683F
:10359000016841F4805101603EE02068C068A16B81
:1035A0000880A06B801CA0639EE04346002202219D
:1035B000204605F05BF9002874D1206B2168008853
:1035C000C860206B801C2063E08E401E0004000C4D
:1035D000E08609D1A06A00E0C7E0A84204D12068D3
:1035E000016841F4805101604346002201212046D8
:1035F00005F03CF900286FD12068C068A16B0880F5
:10360000A06B801CA063E08F401EE087E08E002846
:10361000CBD1606800286AD14346002201212046B0
:1036200005F024F9F0BBB8E7206B411C2163216849
:103630000078C860E08E401EE086E08E98B9A06AEF
:10364000A84204D12068016841F4805101604346DA
:1036500000220121204605F009F918BB2068C06846
:10366000A16B087040E0434600220221204605F08D
:10367000FDF8B8B9206B411C216321680078C8604F
:10368000E08E401E0004000CE08607D1A06AA8422C
:1036900004D12068016841F4805101600022434652
:1036A000012100E018E0204605F0E0F8A0B920680C
:1036B000C168A06B421CA2630170E08F401EE087CE
:1036C000E08E0028CFD1606888B9434600220121EE
:1036D000204605F0CBF808B103200EE72068C1684A
:1036E000A06B421CA2630170E08F401EE087A06ABD
:1036F000A84210D1434600220121204605F0B6F829
:1037000018B1606D40F002000FE02068C068ADF8AD
:103710000000BDF80000434601228021204605F04C
:10372000A5F820B1606D40F020006065D4E784F812
:10373000517020688168A26AC1F30011AA4210D1B9
:1037400079B1616D41F002016165016821F40051B8
:1037500001602068016841F40051016084F8506004
:10376000CAE684F850600020C7E60220C5E670B5BE
:1037700015460E46040003D094F8490010B107E046
:10378000012070BD002084F84800204600F01AF89F
:1037900004F108012068FDF773FC3146A268206837
:1037A000FDF7AAFCD4E901022946236BFDF748FC8A
:1037B000A168206850F8212042F0010240F8212041
:1037C000002070BD1A4800B5016887B041F00101C2
:1037D0000160006800F00100059015480838016894
:1037E00041F008010160016801F0080105910168DC
:1037F00041F0100101600068694600F0100005907A
:103800004EF2B3700090022001900120029003203C
:1038100003900C2004900748FEF73AF94FF68070A9
:10382000009069460448FEF733F907B000BD000078
:1038300038380240000C0240001002404FF0E021F6
:103840000428086903D020F004000861704740F0A4
:103850000400FAE710B5401EB0F1807F01D30120CB
:1038600010BD4FF0E02460610F21601704F0A3F950
:103870000020A06107202061002010BD7047704724
:1038800010B5040003D094F8390010B107E001200E
:1038900010BD002084F83800204600F00DF802200A
:1038A00084F83900211D206805F0D4F8012084F83F
:1038B0003900002010BD000008B500680B4988429F
:1038C00012D10B48016841F0020101600068032237
:1038D00000F00200009001211D20FEF719FCBDE858
:1038E00008401D20FEF708BC08BD00000004004091
:1038F000403802400168CA6842F00102CA600068AC
:10390000016841F00101016000207047704770B507
:103910000446006801694FF00005C943890715D4C2
:10392000C168C943890711D4E91E016101202076CD
:10393000206880698007204602D0FFF7E7FF04E097
:1039400000F098F8204600F096F825762068016986
:10395000C943490717D4C168C943490713D46FF055
:1039600004010161022020762068806910F4407F04
:10397000204602D0FFF7CAFF04E000F07BF82046A3
:1039800000F079F8257620680169C943090716D443
:10399000C168C943090712D46FF00801016104200E
:1039A00020762068C0698007204602D0FFF7AEFF6E
:1039B00004E000F05FF8204600F05DF8257620680E
:1039C0000169C943C90617D4C168C943C90613D4DC
:1039D0006FF010010161082020762068C06910F4A2
:1039E000407F204602D0FFF791FF04E000F042F84C
:1039F000204600F040F8257620680169C943C907D0
:103A000008D1C168C943C90704D1891E0161204694
:103A100000F032F820680169C943090609D4C16879
:103A2000C943090605D46FF0800101612046FFF704
:103A300025FF20680169C943490609D4C168C94303
:103A4000490605D46FF040010161204600F026F8D8
:103A500020680169C94389060BD4C168C943890636
:103A600007D46FF0200101612046BDE87040FFF7E8
:103A700006BF70BD704770470649884206D10649A7
:103A8000D1F8800218B10020C1F8800270470120EF
:103A9000FAE70000B0C30220008040427047704740
:103AA00038B5016804460868CA68C0F3000002F42B
:103AB000807238B132B1086848680090E06B40F01D
:103AC0000100E06308684A69C0F3400002F00102A7
:103AD00038B132B1086848680090E06B40F00400EB
:103AE000E06308684A69C0F3800002F0010238B15F
:103AF00032B1086848680090E06B40F00200E06373
:103B000008684A69C0F3C00002F0010238B132B15E
:103B1000086848680090E06B40F00800E0630868BF
:103B2000C968C0F3401001F0200118B111B120465E
:103B300005F01AF820680168C068C1F3C01100F0F0
:103B4000800019B110B1204605F01CF92168086801
:103B5000CA68C0F3801002F04002012568B162B16A
:103B6000CA68204622F04002CA6094F8391032290F
:103B70000CD080F8395000F0EDF8E06B002804D04C
:103B800084F839502046FFF78AFF38BD222180F89B
:103B90003910F0E770B5040004D094F8390000251E
:103BA00010B106E0012070BD84F83850204600F0C6
:103BB00021F8022084F839002068C16821F40051FE
:103BC000C160204605F024F82068016921F4904185
:103BD00001612068416921F02A0141612068C168C2
:103BE00041F40051C160E563012084F839000020F0
:103BF00070BD000030B504460068204987B0884297
:103C000039D11F48016841F001010160006800F0EE
:103C1000010005901A481430016841F0100101605C
:103C20000068012100F0100005904FF40070009032
:103C30000220CDE9010103900720124D049069464E
:103C40002846FDF725FF2815009069462846FDF710
:103C50001FFF2068C16821F04001C1602068C16871
:103C600041F02001C1602520FEF746FA03221146EB
:103C70002520FEF74DFA07B030BD000000100140CE
:103C800030380240000002402DE9F047044690F829
:103C9000390099460D46012801D0122857D125B385
:103CA0001AB394F83800012851D0012684F83860FE
:103CB0000027E76394F83900122819D0222084F8ED
:103CC0003900A285E2854FF48058E08D4B46401EB6
:103CD000E085A0684FF0000240454FF020012046EB
:103CE00016D105F082F8B0B904E00120BDE8F087F4
:103CF0003220E4E7206900282068406803D0C1B280
:103D000025F8011B12E0C0F3080125F8021B0DE0A5
:103D100005F06BF808B10320E8E720690028206867
:103D2000406801D000F07F0005F8010BE08D00280D
:103D3000CBD194F83900322805D084F8396084F862
:103D400038700020D2E7122084F83900F7E702200B
:103D5000CCE770477047FEE770B51B4886B000257A
:103D6000016841F001010160016801F00101059164
:103D7000016841F004010160016801F0040105914E
:103D8000016841F0800101600068032400F08000B8
:103D9000059002200126CDE90204CDE900656946BF
:103DA0000A48FDF775FE700303948DE861006946CB
:103DB0000748FDF76DFE0C20009069460548FDF7A9
:103DC00067FE06B070BD00003038024000000240BF
:103DD00000080240001C024070B50E490E4A06461B
:103DE00008881268002422B13046BDE8704002F015
:103DF000E5BE4D8800214543084602F031FD02F042
:103E0000A5FEB1B2054801E00180641CAC42FBD3C1
:103E100070BD0000800400206C05002000000860D8
:103E20002DE9F05F3C4C3D4DA071296839B102F09D
:103E3000E5FEE88A2080288B6080BDE8F09F364947
:103E40002C232A2589884FF0F00949F2413A47F29C
:103E5000897B2B2645F2105E4FF448774FF4A0780B
:103E600045F2103C4FF4F07268B1A4F80080A4F859
:103E70000290514503D0614501D059452CD1238191
:103E80006581A6813DE0A4F80090A4F80280514528
:103E900003D0614501D0594508D123816581A681B0
:103EA000614533D1A4F8008062802FE0714509D1CB
:103EB0004FF4305020814FF4285060814FF42C5043
:103EC000A08106E0A1F5C85063381FD12381668127
:103ED000A5812280678019E0714509D14FF43050E7
:103EE00020814FF4285060814FF42C50A08106E0CF
:103EF000A1F5C850633804D123816581A68127804C
:103F00006280614502D12280A4F80280BDE8F05FA2
:103F1000002002F0C5BB0000800400206C050020DA
:103F20002DE9F04104463C480D46006820B120468A
:103F3000BDE8F04102F076BE384E270A3146B0881F
:103F40004989A0F513434FEA1528413B10D0A0F54D
:103F5000A643103B0CD0A0F5EE43893B08D0A0F55A
:103F6000AA43103B11D0A0F5C853633B27D04BE0C8
:103F7000084602F0DFFD384602F0D0FDE0B202F064
:103F8000CDFDB08902F0D6FD38E0084602F0D2FD42
:103F9000384602F0C3FD7089401C80B202F0CAFDB1
:103FA000E0B202F0BBFDB08902F0C4FD404602F071
:103FB000B5FDB089401C80B202F0BCFD21E0B079B3
:103FC00018B93088001B401E84B2084602F0B2FDCA
:103FD000270A384602F0A2FDE0B202F09FFD384603
:103FE00002F09CFDE0B202F099FDB08902F0A2FD62
:103FF000404602F093FDE8B202F090FD404602F028
:104000008DFDE8B202F08AFD054930890880881CE0
:104010000280BDE8F08100006C05002080040020D3
:10402000FEFF07602DE9F8431F46144B80460898B1
:104030001B6833B100903B46404602F011FEBDE8DC
:10404000F883A2EB0802521C96B20C4685B2DFF848
:1040500030900FE02146404602F002FC02F076FD6F
:104060000020494602E00D80401C80B2B042FAD3E5
:10407000641CA4B2BC42EDD9E1E700006C0500204D
:10408000000008602DE9F04F95B002F087FFFE4C6C
:104090004FF0010BA4F1500AA08047F2897545F258
:1040A000103845F2105641F6631918B102F032FE8D
:1040B00002F096BAF5480027016841F0020101605C
:1040C000006810A900F0020000902020CDE9100B3C
:1040D0000320CDE912B0EE48FDF7DAFC4FF02041A5
:1040E0005046CAF80010EB49C0E901171021CAF880
:1040F0000C70C0E90471CAF818700902CAF81C7083
:10410000C0E909718900C0E90B71CAF834708901EE
:10411000CAE90E7146210B910F20CDE90907CDE9BF
:1041200002070490D8480F9702AA09A908975038A7
:10413000FFF71DFB322006F09BFED32002F0FAFCB5
:1041400002F07CFAA08002F079FAA08002F076FA00
:104150004FF6FF7707EA0020A08002F06FFAA188EF
:104160000843A0F51341A08041397AD0042002F021
:10417000E1FC02F063FAA08002F060FAA08002F095
:104180005DFA07EA0020A08002F058FAA1880843EF
:10419000A0F50541A08052395FD0A84261D0D4205B
:1041A00002F0C8FC02F04AFAA08002F047FAA080B0
:1041B00002F044FA07EA0020A08002F03FFAA1884A
:1041C0000843A08040454CD055214FF4704002F088
:1041D000C7FCAA214FF2010002F0C2FC52214FF2AB
:1041E000020002F0BDFC08214FF2030002F0B8FC0F
:1041F00001214FF2040002F0B3FC4FF4454002F0FD
:1042000099FC02F01BFA07EA0020A0804CF2015052
:1042100002F090FC02F012FAA1880843A080052069
:1042200006F026FEA088B0F5004F7DD0B04218D031
:10423000A12002F07FFC02F001FAA08002F0FEF95A
:1042400007EA0020A08002F0F9F9A1880843A0F550
:10425000AE41A080613902D003E0A58001E0A4F85E
:104260000490A1888CA004F0EFFFA088A0F5134172
:1042700041397DD0A8427CD1112002F05BFC78202E
:1042800006F0F6FD362002F055FC002002F046FC58
:104290003A2002F04FFC052002F040FCB22002F070
:1042A00049FC0C2002F03AFC0C2002F037FC002004
:1042B00002F034FC332002F031FC332002F02EFCFB
:1042C000B72002F037FC352002F028FCBB2002F0BA
:1042D00031FC322002F022FCC02002F02BFC0C202A
:1042E00002F01CFCC22002F025FC012002F016FCAA
:1042F000C32002F01FFC102002F010FCC42002F0CA
:1043000019FC202002F00AFCC62002F013FC0F204A
:1043100002F004FCD02002F00DFCA42002F0FEFB11
:10432000A12002F0FBFB00E0A0E1E02002F002FC93
:10433000D02002F0F3FB002002F0F0FB022002F09C
:10434000EDFB072002F0EAFB0A2002F0E7FB282041
:1043500002F0E4FB322002F0E1FB442002F0DEFB3D
:10436000422002F0DBFB062002F0D8FB0E2001E029
:1043700059E07DE102F0D2FB122002F0CFFB1420C5
:1043800002F0CCFB172002F0C9FBE12002F0D2FBC7
:10439000D02002F0C3FB002002F0C0FB022002F09C
:1043A000BDFB072002F0BAFB0A2002F0B7FB282071
:1043B00002F0B4FB312002F0B1FB542002F0AEFB5E
:1043C000472002F0ABFB0E2002F0A8FB1C2002F0FD
:1043D000A5FB172002F0A2FB1B2002F09FFB1E2072
:1043E00002F09CFB2A2002F0A5FB002002F096FBC5
:1043F000002002F093FB002002F090FBEF2002F07F
:104400008DFB2B2002F096FB002002F087FB0020A2
:1044100002F084FB012002F081FB3F2002F07EFBD2
:10442000292002F020B8CF2002F084FB002002F007
:1044300075FBC12002F072FB302002F06FFBED2013
:1044400002F078FB642002F069FB032002F066FBB7
:10445000122002F063FB812002F060FBE82002F0F2
:1044600069FB852002F05AFB102002F057FB7A20EE
:1044700002F054FBCB2002F05DFB392002F04EFB32
:104480002C2002F04BFB0FE080040020303802406B
:1044900000040240040100A0204C43442049443A57
:1044A00025780D0A00000000002002F037FB3420C0
:1044B00002F034FB022002F031FBF72002F03AFB5D
:1044C000202002F02BFBEA2002F034FB002002F057
:1044D00025FB002002F022FBC02002F02BFB1B205A
:1044E00002F01CFBC12002F025FB012002F016FBAC
:1044F000C52002F01FFB302002F010FB302002F03C
:104500000DFBC72002F016FBB72002F007FB362098
:1045100002F010FB482002F001FB3A2002F00AFBF7
:10452000552002F0FBFAB12002F004FB002002F05B
:10453000F5FA1A2002F0F2FAB62002F0FBFA0A208D
:1045400002F0ECFAA22002F0E9FAF22002F0F2FA0C
:10455000002002F0E3FA262002F0ECFA012002F03B
:10456000DDFAE02002F0E6FA0F2002F0D7FA2A2066
:1045700002F0D4FA282002F0D1FA082002F0CEFA94
:104580000E2002F0CBFA082002F0C8FA542002F004
:10459000C5FAA92002F0C2FA432002F0BFFA0A20AD
:1045A00002F0BCFA0F2002F0B9FA002002F0B6FACD
:1045B000002002F0B3FA002002F0B0FA002002F06E
:1045C000ADFAE12002F0B6FA002002F0A7FA1520B9
:1045D00002F0A4FA172002F0A1FA072002F09EFAD6
:1045E000112002F09BFA062002F098FA2B2002F02C
:1045F00095FA562002F092FA3C2002F08FFA05203C
:1046000002F08CFA102002F089FA0F2002F086FAEC
:104610003F2002F083FA3F2002F080FA0F2002F0E0
:104620007DFA2B2002F086FA002002F077FA0020B3
:1046300002F074FA012002F071FA3F2002F06EFAE3
:104640002A2002F077FA002002F068FA002002F037
:1046500065FA002002F062FAEF2002F05FFA112002
:1046600002F068FA782006F003FCD9E6A680F8E5A7
:1046700040457CD1ED2002F05DFA012002F04EFAB7
:10468000FE2002F04BFAEE2002F054FADE2002F097
:1046900045FA212002F042FAF12002F04BFA012003
:1046A00002F03CFADF2002F045FA102002F036FA60
:1046B000C42002F03FFA8F2002F030FAC62002F048
:1046C00039FA002002F02AFAE22002F027FAE2206A
:1046D00002F024FAE22002F021FABF2002F02AFAC6
:1046E000AA2002F01BFAB02002F024FA0D2002F0FA
:1046F00015FA002002F012FA0D2002F00FFA002045
:1047000002F00CFA112002F009FA002002F006FA79
:10471000192002F003FA002002F000FA212002F032
:10472000FDF9002002F0FAF92D2002F0F7F900203F
:1047300002F0F4F93D2002F0F1F9002002F0EEF968
:104740005D2002F0EBF9002002F0E8F95D2002F0B4
:10475000E5F9002002F0E2F9B12002F0EBF9802047
:1047600002F0DCF9002002F0D9F98B2000E0FCE334
:1047700002F0D4F9002002F0D1F9962002F0CEF92F
:10478000002002F0CBF9B22002F0D4F9002002F0B0
:10479000C5F9002002F0C2F9022002F0BFF90020A2
:1047A00002F0BCF9032002F0B9F9002002F0B6F9DA
:1047B000B32002F0BFF9002002F0B0F9002002F0AF
:1047C000ADF9002002F0AAF9002002F0A7F90020BC
:1047D00002F0A4F9002002F0A1F9002002F09EF9F5
:1047E000002002F09BF9002002F098F9002002F06E
:1047F00095F9002002F092F9002002F08FF90020D4
:1048000002F08CF9002002F089F9002002F086F90C
:10481000002002F083F9002002F080F9002002F06D
:104820007DF9002002F07AF9002002F077F90020EB
:1048300002F074F9002002F071F9002002F06EF924
:10484000002002F06BF9B42002F074F98B2002F022
:1048500065F9002002F062F9962002F05FF900206D
:1048600002F05CF9A12002F059F9002002F056F99B
:10487000B52002F05FF9022002F050F9002002F0AA
:104880004DF9032002F04AF9002002F047F9042014
:1048900002F044F9002002F041F9B62002F04AF992
:1048A000002002F03BF9002002F038F9B72002F0B6
:1048B00041F9002002F032F9002002F02FF93F20E8
:1048C00002F02CF9002002F029F95E2002F026F90E
:1048D000002002F023F9642002F020F9002002F009
:1048E0001DF98C2002F01AF9002002F017F9AC2013
:1048F00002F014F9002002F011F9DC2002F00EF9A8
:10490000002002F00BF9702002F008F9002002F0FC
:1049100005F9902002F002F9002002F0FFF8EB20E8
:1049200002F0FCF8002002F0F9F8DC2002F0F6F8C2
:10493000002002F0F3F8B82002F0FCF8002002F0AA
:10494000EDF8002002F0EAF8002002F0E7F800207D
:1049500002F0E4F8002002F0E1F8002002F0DEF8B6
:10496000002002F0DBF8002002F0D8F8BA2002F0B4
:10497000E1F8242002F0D2F8002002F0CFF8002065
:1049800002F0CCF8002002F0C9F8C12002F0D2F801
:10499000202002F0C3F8002002F0C0F8542002F0FA
:1049A000BDF8002002F0BAF8FF2002F0B7F80020AE
:1049B00002F0B4F8C22002F0BDF80A2002F0AEF80E
:1049C000002002F0ABF8042002F0A8F8002002F06A
:1049D000A5F8C32002F0AEF83C2002F09FF80020BA
:1049E00002F09CF83A2002F099F8002002F096F8C4
:1049F000392002F093F8002002F090F8372002F0FE
:104A00008DF8002002F08AF83C2002F087F80020A0
:104A100002F084F8362002F081F8002002F07EF8DF
:104A2000322002F07BF8002002F078F82F2002F00C
:104A300075F8002002F072F82C2002F06FF80020C8
:104A400002F06CF8292002F069F8002002F066F804
:104A5000262002F063F8002002F060F8242002F023
:104A60005DF8002002F05AF8242002F057F80020E8
:104A700002F054F8232002F051F8002002F04EF822
:104A80003C2002F04BF8002002F048F8362002F0FB
:104A900045F8002002F042F8322002F03FF80020F2
:104AA00002F03CF82F2002F039F8002002F036F82E
:104AB0002C2002F033F8002002F030F8292002F018
:104AC0002DF8002002F02AF8262002F027F8002016
:104AD00002F024F8242002F021F8002002F01EF851
:104AE000242002F01BF8002002F018F8232002F026
:104AF00015F8002002F012F8C42002F01BF8622022
:104B000002F00CF8002002F009F8052002F006F887
:104B1000002002F003F8842002F000F8002001F0E9
:104B2000FDFFF02001F0FAFF002001F0F7FF182050
:104B300001F0F4FF002001F0F1FFA42001F0EEFFEE
:104B4000002001F0EBFF182001F0E8FF002001F049
:104B5000E5FF502001F0E2FF002001F0DFFF0C2014
:104B600001F0DCFF002001F0D9FF172001F0D6FF93
:104B7000002001F0D3FF952001F0D0FF002001F0CC
:104B8000CDFFF32001F0CAFF002001F0C7FFE620AF
:104B900001F0C4FF002001F0C1FFC52001F0CAFFF1
:104BA000322001F0BBFF002001F0B8FF442001F0EB
:104BB000B5FF002001F0B2FF652001F0AFFF00203B
:104BC00001F0ACFF762001F0A9FF002001F0A6FF64
:104BD000882001F0A3FF002001F0A0FFC62001F013
:104BE000A9FF202001F09AFF002001F097FF172075
:104BF00001F094FF002001F091FF012001F08EFFF1
:104C0000002001F08BFFC72001F094FF002001F08D
:104C100085FF002001F082FF002001F07FFF0020CF
:104C200001F07CFFC82001F085FF002001F076FF35
:104C3000002001F073FF002001F070FF002001F060
:104C40006DFFC92001F076FF002001F067FF002012
:104C500001F064FF002001F061FF002001F05EFF21
:104C6000002001F05BFF002001F058FF002001F060
:104C700055FF002001F052FF002001F04FFF0020FF
:104C800001F04CFF002001F049FF002001F046FF39
:104C9000002001F043FF002001F040FF002001F060
:104CA0003DFF002001F03AFFE02001F043FF162015
:104CB00001F034FF002001F031FF1C2001F02EFF35
:104CC000002001F02BFF212001F028FF002001F03F
:104CD00025FF362001F022FF002001F01FFF4620B3
:104CE00001F01CFF002001F019FF522001F016FF17
:104CF000002001F013FF642001F010FF002001F0FC
:104D00000DFF7A2001F00AFF002001F007FF8B2041
:104D100001F004FF002001F001FF992001F0FEFEE8
:104D2000002001F0FBFEA82001F0F8FE002001F0B9
:104D3000F5FEB92001F0F2FE002001F0EFFEC420E4
:104D400001F0ECFE002001F0E9FECA2001F0E6FED1
:104D5000002001F0E3FED22001F0E0FE002001F08F
:104D6000DDFED92001F0DAFE002001F0D7FEE020C0
:104D700001F0D4FE002001F0D1FEF32001F0CEFEC0
:104D8000002001F0CBFEE12001F0D4FE162001F05E
:104D9000C5FE002001F0C2FE1C2001F0BFFE002075
:104DA00001F0BCFE222001F0B9FE002001F0B6FEA9
:104DB000362001F0B3FE002001F0B0FE452001F0E6
:104DC000ADFE002001F0AAFE522001F0A7FE002057
:104DD00001F0A4FE642001F0A1FE002001F09EFE7F
:104DE0007A2001F09BFE002001F098FE8B2001F05C
:104DF00095FE002001F092FE992001F08FFE002028
:104E000001F08CFEA82001F089FE002001F086FE52
:104E1000B92001F083FE002001F080FEC42001F0E3
:104E20007DFE002001F07AFECA2001F077FE00200E
:104E300001F074FED22001F071FE002001F06EFE40
:104E4000D82001F06BFE002001F068FEE02001F0A8
:104E500065FE002001F062FEF32001F05FFE0020FD
:104E600001F05CFEE22001F065FE052001F056FE37
:104E7000002001F053FE0B2001F050FE002001F055
:104E80004DFE1B2001F04AFE002001F047FE3420B9
:104E900001F044FE002001F041FE442001F03EFEFE
:104EA000002001F03BFE4F2001F038FE002001F011
:104EB00035FE612001F032FE002001F02FFE792046
:104EC00001F02CFE002001F029FE882001F026FED2
:104ED000002001F023FE972001F020FE002001F0C9
:104EE0001DFEA62001F01AFE002001F017FEB720DB
:104EF00001F014FE002001F011FEC22001F00EFEB0
:104F0000002001F00BFEC72001F008FE002001F098
:104F100005FED12001F002FE002001F0FFFDD620A9
:104F200001F0FCFD002001F0F9FDDD2001F0F6FDAF
:104F3000002001F0F3FDF32001F0F0FD002001F06E
:104F4000EDFDE32001F0F6FD052001F0E7FD002076
:104F500001F0E4FD0A2001F0E1FD002001F0DEFD9A
:104F60001C2001F0DBFD002000E0FDE201F0D6FD99
:104F7000332001F0D3FD002001F0D0FD442001F0EA
:104F8000CDFD002001F0CAFD502001F0C7FD00203A
:104F900001F0C4FD622001F0C1FD002001F0BEFD62
:104FA000782001F0BBFD002001F0B8FD882001F061
:104FB000B5FD002001F0B2FD972001F0AFFD00200B
:104FC00001F0ACFDA62001F0A9FD002001F0A6FD36
:104FD000B72001F0A3FD002001F0A0FDC22001F0E8
:104FE0009DFD002001F09AFDC72001F097FD0020F3
:104FF00001F094FDD12001F091FD002001F08EFD23
:10500000D52001F08BFD002001F088FDDD2001F0AE
:1050100085FD002001F082FDF32001F07FFD0020DE
:1050200001F07CFDE42001F085FD012001F076FD1A
:10503000002001F073FD012001F070FD002001F05F
:105040006DFD022001F06AFD002001F067FD2A20BD
:1050500001F064FD002001F061FD3C2001F05EFDE7
:10506000002001F05BFD4B2001F058FD002001F015
:1050700055FD5D2001F052FD002001F04FFD742030
:1050800001F04CFD002001F049FD842001F046FDB7
:10509000002001F043FD932001F040FD002001F0CD
:1050A0003DFDA22001F03AFD002001F037FDB320C4
:1050B00001F034FD002001F031FDBE2001F02EFD95
:1050C000002001F02BFDC42001F028FD002001F09C
:1050D00025FDCD2001F022FD002001F01FFDD32091
:1050E00001F01CFD002001F019FDDD2001F016FD8E
:1050F000002001F013FDF32001F010FD002001F06D
:105100000DFDE52001F016FD002001F007FD002057
:1051100001F004FD002001F001FD002001F0FEFC83
:10512000022001F0FBFC002001F0F8FC292001F036
:10513000F5FC002001F0F2FC3C2001F0EFFC002027
:1051400001F0ECFC4B2001F0E9FC002001F0E6FC52
:105150005D2001F0E3FC002001F0E0FC742001F090
:10516000DDFC002001F0DAFC842001F0D7FC0020F7
:1051700001F0D4FC932001F0D1FC002001F0CEFC22
:10518000A22001F0CBFC002001F0C8FCB32001F00C
:10519000C5FC002001F0C2FCBE2001F0BFFC0020D5
:1051A00001F0BCFCC42001F0B9FC002001F0B6FC09
:1051B000CD2001F0B3FC002001F0B0FCD32001F0C1
:1051C000ADFC002001F0AAFCDC2001F0A7FC0020CF
:1051D00001F0A4FCF32001F0A1FC002001F09EFCF2
:1051E000E62001F0A7FC112001F098FC002001F05E
:1051F00095FC342001F092FC002001F08FFC562039
:1052000001F08CFC002001F089FC762001F086FC86
:10521000002001F083FC772001F080FC002001F0E9
:105220007DFC662001F07AFC002001F077FC8820EC
:1052300001F074FC002001F071FC992001F06EFC7B
:10524000002001F06BFCBB2001F068FC002001F0A5
:1052500065FC992001F062FC002001F05FFC6620F3
:1052600001F05CFC002001F059FC552001F056FCD7
:10527000002001F053FC552001F050FC002001F00B
:105280004DFC452001F04AFC002001F047FC432082
:1052900001F044FC002001F041FC442001F03EFC00
:1052A000002001F03BFCE72001F044FC322001F03B
:1052B00035FC002001F032FC552001F02FFC0020CD
:1052C00001F02CFC762001F029FC002001F026FCE6
:1052D000662001F023FC002001F020FC672001F093
:1052E0001DFC002001F01AFC672001F017FC0020D3
:1052F00001F014FC872001F011FC002001F00EFCED
:10530000992001F00BFC002001F008FCBB2001F00B
:1053100005FC002001F002FC992001F0FFFB0020B9
:1053200001F0FCFB772001F0F9FB002001F0F6FB17
:10533000442001F0F3FB002001F0F0FB562001F0C7
:10534000EDFB002001F0EAFB232001F0E7FB002049
:1053500001F0E4FB332001F0E1FB002001F0DEFB73
:10536000452001F0DBFB002001F0D8FBE82001F034
:10537000E1FB002001F0D2FB002001F0CFFB9920DF
:1053800001F0CCFB002001F0C9FB872001F0C6FB37
:10539000002001F0C3FB882001F0C0FB002001F0D9
:1053A000BDFB772001F0BAFB002001F0B7FB6620BF
:1053B00001F0B4FB002001F0B1FB882001F0AEFB4E
:1053C000002001F0ABFBAA2001F0A8FB002001F0B7
:1053D000A5FBBB2001F0A2FB002001F09FFB992060
:1053E00001F09CFB002001F099FB662001F096FB88
:1053F000002001F093FB552001F090FB002001F00C
:105400008DFB552001F08AFB002001F087FB442032
:1054100001F084FB002001F081FB442001F07EFBC1
:10542000002001F07BFB552001F078FB002001F00B
:1054300075FBE92001F07EFBAA2001F06FFB002044
:1054400001F06CFB002001F069FB002001F066FB1D
:10545000002001F06FFBAA2001F060FBCF2001F0DB
:1054600069FB002001F05AFB002001F057FB0020EF
:1054700001F054FB002001F051FB002001F04EFB35
:10548000002001F04BFB002001F048FB002001F060
:1054900045FB002001F042FB002001F03FFB002013
:1054A00001F03CFB002001F039FB002001F036FB4D
:1054B000002001F033FB002001F030FB002001F060
:1054C0002DFB002001F02AFBF02001F033FB00202F
:1054D00001F024FB502001F021FB002001F01EFB15
:1054E000002001F01BFB002001F018FBF32001F06D
:1054F00021FB002001F012FBF92001F01BFB06202C
:1055000001F00CFB102001F009FB292001F006FB43
:10551000002001F003FB3A2001F00CFB552001F0C4
:10552000FDFA112001F006FB642005F0A1FC292002
:1055300001F000FB352001F0FDFA002001F0EEFA49
:10554000512001F0F7FAFF2001F0E8FA532001F0B2
:10555000F1FA2C2001F0E2FA552001F0EBFA82205A
:1055600001F0DCFA2C20FDE3B0427DD155214FF44F
:10557000704001F0F5FAAA214FF2010001F0F0FAB3
:1055800052214FF2020001F0EBFA4FF2030308211F
:10559000184601F0E5FA4FF204070121384601F000
:1055A000DFFA0D214FF4304001F0DAFA0D214BF211
:1055B000010001F0D5FA0D214BF2020001F0D0FA02
:1055C00034214FF4364001F0CBFA34214BF2016024
:1055D00001F0C6FA34214BF2026001F0C1FA0D214C
:1055E0004FF4314001F0BCFA0D214BF2011001F0F3
:1055F000B7FA0D214BF2021001F0B2FA34214FF448
:10560000374001F0ADFA34214BF2017001F0A8FAF5
:1056100034214BF2027001F0A3FA00214FF4324022
:1056200001F09EFA00214BF2012001F099FA0021CD
:105630004BF2022001F094FA24214FF4384001F09B
:105640008FFA24214BF6010001F08AFA24214BF64F
:10565000020001F085FA01214FF43F4001F080FA89
:105660000F214FF4334000E0FEE301F079FA0F21FF
:105670004BF2013001F074FA0F214BF2023001F0CD
:105680006FFA34214FF4394001F06AFA34214BF6B5
:10569000011001F065FA34214BF6021001F060FAB6
:1056A00008214FF4354001F05BFA08214BF201501C
:1056B00001F056FA08214BF2025001F051FA032191
:1056C0004FF4424001F04CFA24214FF43A4001F0EB
:1056D00047FA24214BF6012001F042FA24214BF62F
:1056E000022001F03DFA00214FF43C4001F038FA6D
:1056F00078214BF6014001F033FA00214BF60240CD
:1057000001F02EFA00214FF43D4001F029FA7821F2
:105710004BF6015001F024FA00214BF6025001F043
:105720001FFA00214FF43E4001F01AFA64214BF6B3
:10573000016001F015FA00214FF4514001F010FA18
:1057400033214DF2011001F00BFA00214DF202104D
:1057500001F006FA34214DF2031001F001FA0021A4
:105760004DF2041001F0FCF93A214DF2051001F060
:10577000F7F900214DF2061001F0F2F94A214DF23D
:10578000071001F0EDF900214DF2081001F0E8F9E1
:105790005C214DF2091001F0E3F900214DF20A10ED
:1057A00001F0DEF981214DF20B1001F0D9F9002151
:1057B0004DF20C1001F0D4F9A6214DF20D1001F0BC
:1057C000CFF900214DF20E1001F0CAF9E5214DF29A
:1057D0000F1001F0C5F901214DF2101001F0C0F9D0
:1057E00013214DF2111001F0BBF901214DF21210FD
:1057F00001F0B6F954214DF2131001F0B1F9012175
:105800004DF2141001F0ACF982214DF2151001F0A7
:10581000A7F901214DF2161001F0A2F9CA214DF2AB
:10582000171001F09DF902214DF2181001F098F9BE
:1058300000214DF2191001F093F902214DF21A10D6
:1058400001F08EF901214DF21B1001F089F90221BE
:105850004DF21C1001F084F934214DF21D1001F0BD
:105860007FF902214DF21E1001F07AF967214DF205
:105870001F1001F075F902214DF2201001F070F9AE
:1058800084214DF2211001F06BF902214DF222101A
:1058900001F066F9A4214DF2231001F061F9022113
:1058A0004DF2241001F05CF9B7214DF2251001F002
:1058B00057F902214DF2261001F052F9CF214DF295
:1058C000271001F04DF902214DF2281001F048F99E
:1058D000DE214DF2291001F043F902214DF22A1088
:1058E00001F03EF9F2214DF22B1001F039F90221BD
:1058F0004DF22C1001F034F9FE214DF22D1001F083
:105900002FF903214DF22E1001F02AF910214DF24A
:105910002F1001F025F903214DF2301001F020F98C
:1059200033214DF2311001F01BF903214DF23210F9
:1059300001F016F96D214DF2331001F011F900213B
:105940004FF4524001F00CF933214DF2012001F0E7
:1059500007F900214DF2022001F002F934214DF245
:10596000032001F0FDF800214DF2042001F0F8F8C9
:105970003A214DF2052001F0F3F800214DF2062006
:1059800001F0EEF84A214DF2072001F0E9F800217C
:105990004DF2082001F0E4F85C214DF2092001F0FD
:1059A000DFF800214DF20A2001F0DAF881214DF2F2
:1059B0000B2001F0D5F800214DF20C2001F0D0F8B9
:1059C000A6214DF20D2001F0CBF800214DF20E2062
:1059D00001F0C6F8E5214DF20F2001F0C1F80121D8
:1059E0004DF2102001F0BCF813214DF2112001F00E
:1059F000B7F801214DF2122001F0B2F854214DF216
:105A0000132001F0ADF801214DF2142001F0A8F8A7
:105A100082214DF2152001F0A3F801214DF216204C
:105A200001F09EF8CA214DF2172001F099F80221E9
:105A30004DF2182001F094F800214DF2192001F0E8
:105A40008FF802214DF21A2001F08AF801214DF25F
:105A50001B2001F085F802214DF21C2001F080F896
:105A600034214DF21D2001F07BF802214DF21E2061
:105A700001F076F867214DF21F2001F071F8022144
:105A80004DF2202001F06CF884214DF2212001F02C
:105A900067F802214DF2222001F062F8A4214DF2B4
:105AA000232001F05DF802214DF2242001F058F886
:105AB000B7214DF2252001F053F802214DF22620A6
:105AC00001F04EF8CF214DF2272001F049F80221D4
:105AD0004DF2282001F044F8DE214DF2292001F09A
:105AE0003FF802214DF22A2001F03AF8F2214DF25E
:105AF0002B2001F035F802214DF22C2001F030F876
:105B0000FE214DF22D2001F02BF803214DF22E2025
:105B100001F026F810214DF22F2001F021F8032189
:105B20004DF2302001F01CF833214DF2312001F00C
:105B300017F803214DF2322001F012F86D214DF2D9
:105B4000332001F00DF800214FF4534001F008F824
:105B500033214DF2013001F003F800214DF2023003
:105B600000F0FEFF34214DF2033000F0F9FF002178
:105B70004DF2043000F0F4FF3A214DF2053000F010
:105B8000EFFF00214DF2063000F0EAFF4A214DF20E
:105B9000073000F0E5FF00214DF2083000F0E0FF93
:105BA0005C214DF2093000F0DBFF00214DF20A309C
:105BB00000F0D6FF81214DF20B3000F0D1FF002123
:105BC0004DF20C3000F0CCFFA6214DF20D3000F06C
:105BD000C7FF00214DF20E3000F0C2FFE5214DF26B
:105BE0000F3000F0BDFF01214DF2103000F0B8FF82
:105BF00013214DF2113000F0B3FF01214DF21230AC
:105C000000F0AEFF54214DF2133000F0A9FF012146
:105C10004DF2143000F0A4FF82214DF2153000F057
:105C20009FFF01214DF2163000F09AFFCA214DF27C
:105C3000173000F095FF02214DF2183000F090FF70
:105C400000214DF2193000F08BFF02214DF21A3085
:105C500000F086FF01214DF21B3000F081FF022190
:105C60004DF21C3000F07CFF34214DF21D3000F06D
:105C700077FF02214DF21E3000F072FF67214DF2D6
:105C80001F3000F06DFF02214DF2203000F068FF60
:105C900084214DF2213000F063FF02214DF22230C9
:105CA00000F05EFFA4214DF2233000F059FF0221E5
:105CB0004DF2243000F054FFB7214DF2253000F0B2
:105CC0004FFF02214DF2263000F04AFFCF214DF266
:105CD000273000F045FF02214DF2283000F040FF50
:105CE000DE214DF2293000F03BFF02214DF22A3037
:105CF00000F036FFF2214DF22B3000F031FF02218F
:105D00004DF22C3000F02CFFFE214DF22D3000F032
:105D100027FF03214DF22E3000F022FF10214DF21B
:105D20002F3000F01DFF03214DF2303000F018FF3E
:105D300033214DF2313000F013FF03214DF23230A8
:105D400000F00EFF6D214DF2333000F009FF00210D
:105D50004FF4544000F004FF33214DF2014000F0B5
:105D6000FFFE00E07FE300214DF2024000F0F8FE6C
:105D700034214DF2034000F0F3FE00214DF20440C7
:105D800000F0EEFE3A214DF2054000F0E9FE002160
:105D90004DF2064000F0E4FE4A214DF2074000F0CB
:105DA000DFFE00214DF2084000F0DAFE5C214DF2EA
:105DB000094000F0D5FE00214DF20A4000F0D0FE6F
:105DC00081214DF20B4000F0CBFE00214DF20C4042
:105DD00000F0C6FEA6214DF20D4000F0C1FE0021EC
:105DE0004DF20E4000F0BCFEE5214DF20F4000F0F8
:105DF000B7FE01214DF2104000F0B2FE13214DF22A
:105E0000114000F0ADFE01214DF2124000F0A8FE5D
:105E100054214DF2134000F0A3FE01214DF2144035
:105E200000F09EFE82214DF2154000F099FE012106
:105E30004DF2164000F094FECA214DF2174000F0DA
:105E40008FFE02214DF2184000F08AFE00214DF233
:105E5000194000F085FE02214DF21A4000F080FE4C
:105E600001214DF21B4000E000E300F079FE022129
:105E70004DF21C4000F074FE34214DF21D4000F044
:105E80006FFE02214DF21E4000F06AFE67214DF2C6
:105E90001F4000F065FE02214DF2204000F060FE40
:105EA00084214DF2214000F05BFE02214DF22240A0
:105EB00000F056FEA4214DF2234000F051FE0221D5
:105EC0004DF2244000F04CFEB7214DF2254000F089
:105ED00047FE02214DF2264000F042FECF214DF256
:105EE000274000F03DFE02214DF2284000F038FE30
:105EF000DE214DF2294000F033FE02214DF22A400E
:105F000000F02EFEF2214DF22B4000F029FE02217E
:105F10004DF22C4000F024FEFE214DF22D4000F009
:105F20001FFE03214DF22E4000F01AFE10214DF20B
:105F30002F4000F015FE03214DF2304000F010FE1E
:105F400033214DF2314000F00BFE03214DF232407F
:105F500000F006FE6D214DF2334000F001FE0021FD
:105F60004FF4554000F0FCFD33214DF2015000F09C
:105F7000F7FD00214DF2025000F0F2FD34214DF208
:105F8000035000F0EDFD00214DF2045000F0E8FD5B
:105F90003A214DF2055000F0E3FD00214DF206508C
:105FA00000F0DEFD4A214DF2075000F0D9FD00213E
:105FB0004DF2085000F0D4FD5C214DF2095000F084
:105FC000CFFD00214DF20A5000F0CAFD81214DF2B3
:105FD0000B5000F0C5FD00214DF20C5000F0C0FD4B
:105FE000A6214DF20D5000F0BBFD00214DF20E50E8
:105FF00000F0B6FDE5214DF20F5000F0B1FD01219A
:106000004DF2105000F0ACFD13214DF2115000F094
:10601000A7FD01214DF2125000F0A2FD54214DF2D6
:10602000135000F09DFD01214DF2145000F098FD39
:1060300082214DF2155000F093FD01214DF21650D2
:1060400000F08EFDCA214DF2175000F089FD0221AB
:106050004DF2185000F084FD00214DF2195000F06F
:106060007FFD02214DF21A5000F07AFD01214DF220
:106070001B5000F075FD02214DF21C5000F070FD28
:1060800034214DF21D5000F06BFD02214DF21E50E7
:1060900000F066FD67214DF21F5000F061FD022106
:1060A0004DF2205000F05CFD84214DF2215000F0B3
:1060B00057FD02214DF2225000F052FDA4214DF275
:1060C000235000F04DFD02214DF2245000F048FD18
:1060D000B7214DF2255000F043FD02214DF226502C
:1060E00000F03EFDCF214DF2275000F039FD022196
:1060F0004DF2285000F034FDDE214DF2295000F021
:106100002FFD02214DF22A5000F02AFDF2214DF21E
:106110002B5000F025FD02214DF22C5000F020FD07
:10612000FE214DF22D5000F01BFD03214DF22E50AB
:1061300000F016FD10214DF22F5000F011FD03214B
:106140004DF2305000F00CFD33214DF2315000F093
:1061500007FD03214DF2325000F002FD6D214DF29A
:10616000335000F0FDFC00214FF4564000F0F8FCE5
:1061700033214DF2016000F0F3FC00214DF202608A
:1061800000F0EEFC34214DF2036000F0E9FC002148
:106190004DF2046000F0E4FC3A214DF2056000F09D
:1061A000DFFC00214DF2066000F0DAFC4A214DF2DE
:1061B000076000F0D5FC00214DF2086000F0D0FC33
:1061C0005C214DF2096000F0CBFC00214DF20A6029
:1061D00000F0C6FC81214DF20B6000F0C1FC0021F3
:1061E0004DF20C6000F0BCFCA6214DF20D6000F0F9
:1061F000B7FC00214DF20E6000F0B2FCE5214DF23B
:106200000F6000F0ADFC01214DF2106000F0A8FC21
:1062100013214DF2116000F0A3FC01214DF2126038
:1062200000F09EFC54214DF2136000F099FC012116
:106230004DF2146000F094FC82214DF2156000F0E4
:106240008FFC01214DF2166000F08AFCCA214DF24C
:10625000176000F085FC02214DF2186000F080FC10
:1062600000214DF2196000F07BFC02214DF21A6012
:1062700000F076FC01214DF21B6000F071FC022160
:106280004DF21C6000F06CFC34214DF21D6000F0FA
:1062900067FC02214DF21E6000F062FC67214DF2A6
:1062A0001F6000F05DFC02214DF2206000F058FC00
:1062B00084214DF2216000F053FC02214DF2226056
:1062C00000F04EFCA4214DF2236000F049FC0221B5
:1062D0004DF2246000F044FCB7214DF2256000F03F
:1062E0003FFC02214DF2266000F03AFCCF214DF236
:1062F000276000F035FC02214DF2286000F030FCF0
:10630000DE214DF2296000F02BFC02214DF22A60C3
:1063100000F026FCF2214DF22B6000F021FC02215E
:106320004DF22C6000F01CFCFE214DF22D6000F0BF
:1063300017FC03214DF22E6000F012FC10214DF2EB
:106340002F6000F00DFC03214DF2306000F008FCDE
:1063500033214DF2316000F003FC03214DF2326035
:1063600000F0FEFB6D214DF2336000F0F9FB55218A
:10637000381F00F0F5FBAA21F81E00F0F1FB5221B6
:10638000B81E00F0EDFB0821184600F0E9FB0021E3
:10639000384600F0E5FBCC214FF4314000F0E0FB43
:1063A00000214BF2011000F0DBFB05214FF43640D9
:1063B00000F0D6FB70214FF4374000F0D1FB702184
:1063C0004BF2017000F0CCFB01214FF4384000F09B
:1063D000C7FB03214BF6010000F0C2FB03214BF683
:1063E000020000F0BDFB03214BF6030000F0B8FBF8
:1063F00002214FF43C4000F0B3FB00214BF601407A
:1064000000F0AEFB00214BF6024000F0A9FBD021CA
:106410004FF4494000F0A4FB02214CF6011000F0BB
:106420009FFB50214CF6021000F09AFB50214CF6D5
:10643000031000F095FB50214CF6041000F090FB87
:1064400000214FF4545000F08BFB55214FF468505D
:1064500000F086FB4FF4885000F06CFB782004F0CD
:1064600015FD4FF4245000F065FBB9E04845FCD120
:10647000E22000F05FFB1D2000F050FB022000F046
:106480004DFB042000F04AFB642004F0FFFCE020F8
:1064900000F050FB012000F041FB0A2004F0E8FC72
:1064A000E02000F047FB032000F038FB0C2004F054
:1064B000DFFC012000F03EFB0A2004F0D9FCE620BE
:1064C00000F038FB2F2000F029FBFF2000F026FB16
:1064D000FF2000F023FBB02000F02CFB202000F078
:1064E0001DFB002000F01AFB032000F017FB40F218
:1064F0001F3000F013FB012000F010FB40F2DF1012
:1065000000F00CFB002000F009FBB42000F012FBAF
:10651000042000F003FB40F21F4000F0FFFA0020CF
:1065200000F0FCFA2E2000F0F9FA002000F0F6FA54
:10653000002000F0F3FA002000F0F0FA002000F054
:10654000EDFAB62000F0F6FA022000F0E7FA4FF478
:10655000037000F0E3FA002000F0E0FA172000F0EA
:10656000DDFA152000F0DAFA002000F0D7FA00205A
:1065700000F0D4FAF02000F0DDFA032000F0CEFAAB
:10658000292000F0D7FAD02000F0D4FA002000F043
:10659000C5FABE2000F0CEFA052000F0BFFAFE20BA
:1065A00000F0BCFA012000F0B9FA002000F0B6FAC1
:1065B000002000F0B3FA002000F0B0FAB82000F09C
:1065C000B9FA032000F0AAFA012000F0A7FABA20D5
:1065D00000F0B0FA012000F0A1FA642000F038F8D1
:1065E000A088A0F51341413907D0404505D0B042FD
:1065F00003D0484501D0A84209D10420029004905C
:10660000DAE9010202A9DAF83030FAF719FD0020C0
:10661000FDF706FC0449C1F894B24FF6FF70FDF790
:10662000DBFB15B0BDE8F08F00804042034601203F
:1066300000E05843491EC9B2FBD27047034808B571
:106640000088ADF80000BDF8000008BD000008603B
:1066500010B50246BE2000F06DFA052000F05EFA8B
:106660001046F9F7A8FE9FED0C1B53EC112BF9F720
:1066700030FEF9F7ADFE80B200F050FA012000F0D4
:106680004DFAFF2000F04AFA002000F047FABDE87A
:106690001040002000F042BA6666666666660440F6
:1066A000F0B56E4D00232A46A979928841F663140D
:1066B000012901D019B11BE0A24202D118E0A24287
:1066C00016D1082814D2DFE800F00406080A0C0EE0
:1066D000101206200CE007200AE0042008E0052044
:1066E00006E0012004E0002002E0032000E0022098
:1066F000A2F5134745F2103145F21056413F09D03B
:106700008A4207D0B24205D0A24203D0A2F5EE479A
:10671000893F77D1082812D2DFE800F0110406087B
:106720000A0C0E1080230AE0402308E0C02306E094
:10673000202304E0602302E0A02300E0E023B24233
:1067400002D14FF4585000E036208A4205D0B242C0
:1067500003D0A24201D043F00803194600F000FA2A
:10676000A988A1420AD0980628886A8802D5904252
:1067700002D303E0904201D92A8068806889B1423F
:1067800041D100F0D7F9002000F0C8F96889401C19
:1067900080B200F0CFF9002000F0C0F96889801CB9
:1067A00080B200F0C7F92888401EC0F30F2000F027
:1067B000B5F96889C01C80B200F0BCF92878401E89
:1067C000C0B200F0ABF9A88900F0B4F9002000F0E5
:1067D000A5F9A889401C80B200F0ACF9002000F0B7
:1067E0009DF9A889801C80B200F0A4F96888401E39
:1067F000C0F30F2000F092F9A889C01C80B200F00D
:1068000099F922E028E000F095F9002000F086F9DF
:10681000002000F083F92888401EC0F30F2000F00C
:106820007DF92878401EC0B200F078F9A88900F000
:1068300081F9002000F072F9002000F06FF96888FB
:10684000401EC0F30F2000F069F9A878BDE8F040C1
:10685000401EC0B200F062B9F0BD0000800400200C
:10686000F0B5434D0C4602460F0AA8882946160A81
:106870004989A0F51343413B2DD0A0F5A643103B19
:1068800029D0A0F5EE43893B25D0A0F5C853633B42
:1068900031D0A0F5AA43103B68D1084600F04AF970
:1068A000304600F03BF96889401C80B200F042F9A4
:1068B000D0B200F033F9A88900F03CF9384600F076
:1068C0002DF9A889401C80B200F034F9E0B2BDE88F
:1068D000F04000F023B9084600F02CF9304600F0F3
:1068E0001DF9D0B200F01AF9A88900F023F9384652
:1068F00000F014F9EAE7A87930B3084600F01AF975
:10690000304600F00BF9D0B200F008F92888401E9C
:10691000C0F30F2000F002F92878401EC0B200F04A
:10692000FDF8A88900F006F9384600F0F7F8E0B263
:1069300000F0F4F86888401EC0F30F2000F0EEF875
:10694000A878401EC0B2C2E72888801A401E82B2D2
:10695000084600F0EFF8002000F0E0F8002000F01A
:10696000DDF8100A00F0DAF8D0B2D8E7F0BD000088
:10697000800400202DE9F84F82461F460E468B46C4
:10698000580700D0012000EBD700790810FB01F078
:10699000203AC0B202F0FF090025009047E00C2F1A
:1069A00010D0102F12D0182F14D0202F42D12249EE
:1069B00001EBC9104FF00008445D200610D51F48B8
:1069C000026811E009EB49001D4906E01D4901EB91
:1069D0000910EFE71C4909EBC90001EB8000E9E76A
:1069E0000A9828B91548426831465046FDF798FA8A
:1069F0006006040E1548761CB6B24088B04219D91C
:106A0000A6EB0B00B84209D10AF101001FFA80FA87
:106A10000E485E46018851450CD906E008F1010098
:106A200000F0FF08B8F1080FC7D36D1CEDB2009855
:106A30008542B4D3BDE8F88FFE230108240000206E
:106A40003E0C0108B2100108A216010880040020C3
:106A50002DE9FF4F81B00027DDF838B01D46924682
:106A600080463C46B9464FEA5B0627E0281B401E9D
:106A7000C1B20A20FFF7DAFDBAFBF0F00A21B0FB41
:106A8000F1F201FB120027B9691E8C4201DA48B10C
:106A900001273030C2B206FB048080B25B46CDF8DD
:106AA000009006E006FB048080B25B462022CDF811
:106AB00000900299FFF75EFF641CE4B2AC42D5D3AC
:106AC00005B0BDE8F08F2DE9F84F044600F0FF084F
:106AD00010190D46DDE90A761FFA80FA58191FFAD7
:106AE00080F94FF0000B11E0544502D3E8194446F9
:106AF00085B24D450FD23B4629462046CDF800B021
:106B0000FFF738FF04EB570084B2761C3278A2F10D
:106B100020005E28E8D9BDE8F88F000001B5BDF877
:106B20000000ADF80000BDF800000149088008BD74
:106B30000000086001B5BDF80000ADF80000BDF828
:106B400000000149088008BDFEFF076002480349B4
:106B5000008908807047000080040020FEFF076065
:106B6000024A1080901C018070470000FEFF076001
:106B7000104810B5016886B041F00201016000685C
:106B8000012100F0020005900320CDE90210CDE9BB
:106B90000001094C69462046FAF77AFF01221146A6
:106BA0002046FBF768F8012202212046FBF763F834
:106BB00006B010BD303802400004024008B5009015
:106BC0000548018BC08A491E8BB2401E82B200214B
:106BD000084600F045F808BD6C05002000B58DB0F2
:106BE000082309920490009306916846FBF706FB80
:106BF000002800D001200DB000BD000010B5084BEA
:106C00001C465875A1888AB2218889B220B1012812
:106C100001D1D9821A8310BDDA82198310BD000018
:106C20006C050020F0B50C4F94B23D46DFF82CC047
:106C30002B68EA692D7D7E7D5CF8255026B103FB2B
:106C400001004243AC52F0BD7E68301A401E03FB87
:106C5000001050432C52F0BD6C0500202C00002089
:106C60002DE9F843274EDDF820900024757D0DB105
:106C7000054606E077680D46B91A1A463B1A491EC2
:106C80005B1E306896F814C0DFF87C80521B871AB0
:106C900058F82CC0F66900FB015006FB00C51B48E4
:106CA0007F1EBFB2066846F400060660006800F466
:106CB000000000901648066826F0010606604FF4B2
:106CC00040360660022646630764C563591AF3031B
:106CD00003EB0242491C11434164C0F8389001683B
:106CE00041F0010101605A0102E0641C944202D2A9
:106CF00041688907F9D5816841F002018160BDE8EA
:106D0000F88300006C0500202C0000203038024081
:106D100000B002402DE9FF5F00F040F90446012673
:106D2000784DA0F586404FF4F0714FF0280941F2FC
:106D3000180A423847D03204A4F5E0434FF44870B3
:106D40004FF4C67B843B50D003238C27A4F5E04C42
:106D50004FF4B47EBCF1160C54D0A4F5E0484FF4C7
:106D6000A06CB8F118085DD0A4F58048B8F561783A
:106D70005BD054450CD1C5E900C0AF810A20288200
:106D80002881E88168826B8102217046FFF726FF27
:106D90005D482A685E4F0280696841800220E86190
:106DA0005A48386057485B4BA8384FF00008C0E994
:106DB0000038C0F80880C0F80C80544545D14FF029
:106DC0008053036143E04FF48870C5E900102E81C1
:106DD0006E810820A5F80C90E881052129828203A4
:106DE000688204214FF49070D0E7C5E900012E813C
:106DF0006E812E20A8811720E881D22028821620BB
:106E000068821FE04FF4806028604FF4167068605D
:106E1000142028816B81AF81E881A02028820C207A
:106E20006882B1E7C5E900C0B2E7C5E900015820B2
:106E3000A881A5F81090302028812020E8810D201D
:106E400068826B8103215846A0E7C0F810802C8926
:106E5000631E43616B89A3F1010CC0F818C0B5F83B
:106E60000CC06444A4F1010CC0F81CC0B5F80EC0FD
:106E70006344A3F1010CC0F820C0A2F1010CA444AA
:106E8000C0F824C0A1F1010C9C44C0F828C0B5F89A
:106E900010C062442244521EC2626A8A11441944DC
:106EA000491E016380F8368080F8358080F8348090
:106EB0001448A838FAF746FF07200621CDE9020852
:106EC000CDE90081FF2302220020396800F026F876
:106ED000A888002280B200902888114683B210460C
:106EE00000F04AF80020FFF789FE0B4885F814806F
:106EF000C0F8946204B04FF0FF30BDE8F05FFFF7D8
:106F00005DBE00006C05002080040020000000C071
:106F10002C00002000680140008040422DE9F04331
:106F20008DB0164614AA002492E88013114D0094E7
:106F300002942A6801926D68CDE904634FEA082340
:106F4000CDE9067303954FEA09230DF1240E08934A
:106F50008EE8260002468DF8324006488DF8314012
:106F60008DF830C06946A838FAF7C3FE0DB0BDE809
:106F7000F08300006C05002070B51E4604460346F1
:106F80000548049DFAF7D6FF23462A463146BDE858
:106F900070400148FAF7F8BFC404002030B52A4811
:106FA00087B00021026842F040020260026802F0ED
:106FB00040020592026842F4807202600068234C2D
:106FC00000F4807005904020CDE90001012002907E
:106FD0000320039069462046FAF75AFD84201C4D91
:106FE000009069462846FAF753FD40212046FAF7FB
:106FF0003DFE044604212846FAF738FE44EA4004E0
:1070000080212846FAF732FE44EA8000C0B2062802
:1070100017D2DFE800F003070A0D101344F24230E4
:1070200007B030BD47F28400FAE747F21600F7E7F1
:1070300047F21800F4E744F28430F1E741F2180017
:10704000EEE70020ECE70000303802400018024074
:1070500000200240F0B504688B88E568C5F30B4555
:107060002B441D04882303EBC213E65806F4704634
:10707000E65004680F68E668C6F30B46761C3E448B
:107080002E43E65003688C89DD68C5F30A052C445D
:1070900025048C2404EBC2141E5906F470461E51BC
:1070A00003688F68DE68C6F30A06761C3E442E43EA
:1070B0001E519423046803EBC213E55825F007051D
:1070C000E55005680C69EC5091F8313005681F02F5
:1070D00091F832301C040B7E1E069C2303EBC21376
:1070E00055F803C04FF0000C45F803C091F830503C
:1070F00034433D4325430468E5509823046803EB7B
:10710000C213E55825F0FF05E55005684C69EC50C1
:10711000A023046803EBC213E55840F20776B54399
:10712000E550D1E907452C430568EC50AC230468D1
:1071300003EBC213E55844F803C005684C6AEC50F1
:107140000B698BB3012B32D0042B32D0022B30D001
:10715000032B2ED0072B2CD00123B024056804EB81
:10716000C2142E5906F0E0262E51D1E90065AD1B60
:107170000E8D5D435E43ED1C45EA064305682B51C9
:10718000B423046803EBC213E5586FF30A05E55016
:107190000468C96AE1500068842101EBC2114258B9
:1071A00042F001024250F0BDFFE70423D5E703237C
:1071B000D3E70223D1E7FEE72DE9F84F1C46002371
:1071C0000A9E17460D46ADF8003062498979B0FB3A
:1071D000F1F2B5FBF1F1D207B2EBC17F7DD1DFF85F
:1071E0007891984689F80080DFF870B18BF80080BC
:1071F0008BF800808BF80000020A8BF80020000C4E
:107200008BF80000352089F80000002000F0D2FB48
:1072100020B9012000F0CEFB010002D00220BDE821
:10722000F88F852289F800208BF800703A0A8BF8D5
:1072300000208BF800502A0A8BF800202A0C8BF8CB
:1072400000201E2000F0CEF8F0054FF000450ED0D3
:10725000404605E014F8010B2870BDF80000401C02
:10726000ADF80000BDF80000B042F3D364E0760A48
:107270007A0A4FF02043C2464FF4007C354F27E096
:10728000D3F8800040F04000C3F88000504605E08D
:1072900014F8010B2870BDF80000401CADF8000088
:1072A000BDF800006045F3D3D3F884004006FBD559
:1072B000D3F8940001EB020807EB8808C8F81C001B
:1072C000D3F8800020F04000C3F88000491CC9B208
:1072D000B142D5D37988102000E037E000EB82007E
:1072E0000844ADF800001E2000F07CF8852189F8E4
:1072F0000010BDF800008BF80000BDF80000000A87
:107300008BF800001E2000F06DF807EB8201ADF84D
:1073100000A01C310CE0002011F8012B2A70401C49
:10732000C0B20428F8D3BDF80000401CADF800003E
:10733000BDF80000B042EED3102089F80000C8204C
:1073400003F0A4FD00F024FB402801D0012066E7F3
:10735000002064E7D81800200000018000000280AF
:107360002DE9F0410C461C498979B0FBF1F2B4FBE0
:10737000F1F1D207B2EBC17F29D1184F00263E7040
:10738000174D2E702E702870010A2970000C28707D
:1073900035203870304600F00DFB18B9012000F0A0
:1073A00009FB10B10220BDE8F081852038702E70F5
:1073B0002E702C70200A2870200C28701020387035
:1073C000C82003F063FD00F0E3FA402801D001205B
:1073D000E9E70020E7E70000D8180020000001805E
:1073E0000000028001B5009801E0401E00900028D6
:1073F000FBD108BD2DE9F041054690460E4601201F
:1074000000F042F804463146002000F03DF80746FF
:107410004146012000F038F806464146002000F0C1
:1074200033F884EA070272404240A2F57060FF38E8
:1074300005D00AA001F008FF0120BDE8F0817440EA
:1074400021460DA001F000FFE10804F00703685C8D
:1074500001229A40504068540020EEE7326269747D
:1074600020656363206572726F72206F72206D6F8A
:1074700072650D0A000000006572726F72706F73A2
:107480003A25640D0A00000070B5054600200C4640
:107490000246012602F00101A94208D124FA02F1B4
:1074A000C90704D0510806FA01F3184480B2521CEF
:1074B000D2B2182AEED370BD104910B50969104A2E
:1074C000914201D1C00103E00E4A914200D18001F6
:1074D0000D4A602111700D490870030A0B70000CF1
:1074E0000870D0201070042003F0C2FC00F050FAA5
:1074F000402801D0012010BD002010BDD818002068
:1075000089260048569590DC00000180000002802A
:1075100070B50024084D0AE02046FFF7CDFF0200B9
:1075200003D0214605A001F08FFE641CA4B2688937
:10753000A042F1D870BD0000D818002045726173D8
:107540006520256420626C6F636B206661696C2125
:1075500021A3ACB4EDCEF3C2EBCEAA25640D0A0094
:1075600010B5274888B0254901604FF4807141600B
:10757000002181604FF4C022C160C0E90412816122
:107580000121C16102200322CDE90402CDE90601F7
:10759000CDE90002CDE902016A4604A91848FAF7CC
:1075A00021FD00F0E7F9642003F062FC00F048F8E8
:1075B000134C38342061042000F028F8114B4FF4AC
:1075C000805220695110984207D14FF48750208093
:1075D0006280E020A080802008E00B4B98420BD115
:1075E0004FF40460208061804020A080A071218140
:1075F0006281002008B010BD0120FBE7600000A000
:10760000A018002089260048569590DC0A4A00B54B
:10761000EF211170094A01211170C907087000207B
:1076200008700870087000F0B3F9402801D00120FC
:1076300000BD002000BD00000000018000000280AD
:107640000CB50F49902008700E490020087088037F
:1076500001788DF8001001788DF8011001788DF80F
:10766000021001788DF8031000788DF80400DDF821
:1076700001009DF8041000BA20F0FF0008430CBD83
:1076800000000180000002802DE9F84F4FF0000853
:107690001C46154682468946ADF80080744A474626
:1076A00082F8008073480170090A017080F800A018
:1076B0004FEA1A2101704FEA1A4101703020107010
:1076C000002000F077F918B9012000F073F910B12B
:1076D0000220BDE8F88FE2054FF000410ED0404691
:1076E00005E0087805F8010BBDF80000401CADF876
:1076F0000000BDF80000A042F3D3B2E0660A4FEAF2
:107700005924AB464FF02042DFF86CE14FF4007C87
:107710002AE0D2F8801041F04001C2F88010002128
:10772000ADF800104FF0004307E0197805F8011B91
:10773000BDF80010491CADF80010BDF800106145FF
:10774000F3D3D2F884104906FBD5D2F8943000EB7D
:1077500004080EEB8801CB61D2F8801021F04001C3
:10776000C2F88010401CC0B2B042D2D3BEF80200B2
:10777000102101EB840108447546ADF80000232078
:10778000FFF730FE3A4805210170BDF80020394965
:107790000A70BDF80020120A0A70E0210170192059
:1077A000FFF720FE002205EB8400ADF800204FF02B
:1077B00000433C3007E0197800F8011BBDF80010C9
:1077C000491CADF80010BDF80010B1EB860FF2D3E4
:1077D000ADF8002041E0BDF80000BDF800102044E5
:1077E00005EB8000C06B214405EB8101C96988422B
:1077F0002ED0BDF80000204405EB8000C26BBDF820
:107800000000204405EB8000C1691CA001F01CFDB4
:10781000224631461FA001F017FD4A46514623A0DB
:1078200001F012FDBDF80000204405EB8000C269A4
:10783000BDF80000BDF80030204405EB8000C16BAE
:107840000BEB4320FFF7D6FD08B1042700E0032728
:10785000BDF80000401CADF80000BDF80000B042CB
:10786000B9D300F095F8402800D00127384630E71A
:107870000000018000000280D8180020657272208C
:1078800068642C72643A307825782C307825780D2D
:107890000A0000006563636E756D2C656363737425
:1078A0006172743A25642C25640D0A005061676585
:1078B0004E756D2C436F6C4E756D3A25642C2564A6
:1078C0000D0A0000F0B51D46164B0024059F164614
:1078D0001C70154A1170090A11701070010A11709C
:1078E000000C107030201870204600F063F818B9B2
:1078F000012000F05FF808B10220F0BD4FF0004019
:1079000004E00168B14203D1641CA4B2AC42F8D3D4
:107910003C8000F03DF8402801D00120F0BD00205F
:10792000F0BD0000000001800000028030B4064D70
:107930002C79641AE4B2A34200D923466C8821440E
:1079400030BC89B2FFF7A0BED818002008B50020CF
:107950008DF800000649702008701920FFF742FDDD
:107960004FF0004000788DF800009DF8000008BD41
:1079700000000180054900B5FF20087000F008F8FC
:10798000402801D0012000BD002000BD0000018082
:1079900008B500206FF060420090FFF7D7FF400667
:1079A00006D40098401C00909042F6D3022008BDF7
:1079B000402008BD01B581B00020009009486FF05B
:1079C0007E41009A521C0092D0F818229DF8043093
:1079D0009A4201D100200CBD009A8A42F1D30120C5
:1079E0000CBD0000008041422DE9F84F4FF0000827
:1079F0001D46ADF80080DFF83CA1802644468AF899
:107A00000060DFF834B18BF800100E0A8BF80060CC
:107A10008BF80000060A8BF80060000C8BF8000061
:107A20001E20FFF7DFFCE8054FF000460FD0ADF851
:107A3000008007E012F8010B3070BDF80000401C18
:107A4000ADF80000BDF80000A842F3D362E06D0A73
:107A5000490A4FF02043394FC1464FF4007C27E0DC
:107A6000D3F8800040F04000C3F88000484605E0AD
:107A700012F8010B3070BDF80000401CADF800009A
:107A8000BDF800006045F3D3D3F884004006FBD571
:107A9000D3F8940004EB010807EB8808C8F81C0031
:107AA000D3F8800020F04000C3F88000641CE4B2EA
:107AB000AC42D5D37A88102000EB81001044ADF899
:107AC00000001E20FFF78EFC85228AF80020BDF8FA
:107AD00000208BF80020BDF80020120A8BF800204F
:107AE0001E20FFF77FFC07EB8101ADF800901C31F1
:107AF0000CE0002011F8012B3270401CC0B20428A9
:107B0000F8D3BDF80000401CADF80000BDF800003F
:107B1000A842EED310208AF80000C82003F0B6F97E
:107B2000FFF736FF402802D00120BDE8F88F002083
:107B3000FBE700000000018000000280D818002050
:107B400070B5124E1D46002480233370104B1970FF
:107B5000090A19701870010A1970000C18701E209B
:107B6000FFF740FCF00302E00260641CA4B2AC42E8
:107B7000FAD310203070C82003F088F9FFF708FF0F
:107B8000402801D0012070BD002070BD00000180A0
:107B90000000028030B4064D2C79641AE4B2A3428E
:107BA00000D923466C88214430BC89B2FFF71CBF42
:107BB000D818002070470907090E002806DA00F0DF
:107BC0000F0000F1E02080F8141D704700F1E02064
:107BD00080F80014704770472DE9F04F8246881AEC
:107BE000B0FBF3F7002589467F1CDDF824B028E0C0
:107BF000002123E09FED150A002416E005FB034653
:107C000000200FE001FB030C06FB09CC0AEB8C0CF7
:107C1000DCED000AF4EEC00AF1EE10FA01DDB0EE80
:107C2000600A401C9042EDDB641C9442E6DB05FBDD
:107C300007100BEB8000491C80ED000AB942D9DB2C
:107C40006D1CBD42D4DBBDE8F08F000000000000D9
:107C50002DE9F04115460E460746002414E057F87A
:107C60002400F8F7CEFB41EC100B0FA053EC102BC7
:107C700001F0EAFA601C90FBF5F105FB110010B968
:107C80000AA001F0E1FA641CB442E8DB96FBF5F0CF
:107C900005FB1060002804D0BDE8F04103A001F00E
:107CA000D3BABDE8F0810000256620000A0000007C
:107CB00010B50023DFED0A0A0FE000EB830494ED1A
:107CC000000AB5EEC00AF1EE10FA01DCB0EE600A6F
:107CD00002EB83045B1C84ED000A8B42EDDB10BDDC
:107CE00000000000B5EEC00AF1EE10FA01DC9FEDD5
:107CF000010A7047000000000A6842624A68826216
:107D0000D1E902231A43D1E904310B43C16A1A4372
:107D100021F0F7011143C162002070470069C0B231
:107D20007047006800F003007047000008B5024982
:107D300008440090006808BD142C014070B50DF196
:107D4000100C11439CE870002343194329434268F7
:107D5000314347F6FF639A430A434260002070BDF7
:107D60000321016000207047D0F8800070470A6846
:107D70008260D1E901231A43D1E903310B43C16881
:107D80001A436FF30B011143C1600020704709686B
:107D9000C0F880100020704700B5164887B014491D
:107DA0000022C0E900120121816008211023C0E9EE
:107DB0000313402343614FF4C073C0E906320A0243
:107DC00002624A0242628A0282620220CDE9000116
:107DD00006210291CDE903100590069069460548F9
:107DE000FAF772FE034800F007F807B000BD000084
:107DF000400100A09004002010B50023012211468C
:107E0000184600F021F84FF4FA7003F03FF8002311
:107E100001220221184600F017F80023082203214E
:107E2000184600F011F84FF40C73012204210020D1
:107E300000F00AF8BDE8104040F2AB210148FAF723
:107E4000D3BE0000900400201FB5002410B101280B
:107E500002D002E0102400E00824CDE90014CDE9AE
:107E600002234FF4805269460348FAF7CEFE0028F9
:107E700000D0012004B010BD90040020F0B5002215
:107E800085B01746104607F013FB05460A24B0FBE1
:107E9000F4F0B5FBF4F204FB10531BA1684601F0AB
:107EA000E3F93A4601266B4629461AA001F0CCF9BF
:107EB000304607F0FDFA0546B0FBF4F0B5FBF4F2EE
:107EC00004FB105310A1684601F0CEF902276B465F
:107ED000324629460FA001F0B7F9384607F0E8FA14
:107EE0000546B0FBF4F0B5FBF4F204FB105306A119
:107EF000684601F0B9F96B463A46294605A001F0FB
:107F0000A3F905B0F0BD000025642E2530316425AD
:107F1000250000005B25645D202564CAB9D3C3C178
:107F2000BFCEAAA3BA25730D0A00000070B504469F
:107F300000680E460025416B11F0450FFBD0416BE8
:107F4000490703D503210422826304E0416BC9077A
:107F500003D001218163084670BDFFF7DFFEB04208
:107F60002BD1216840F2FF5088630020FFF7DEFE2E
:107F7000284908424BD0002801DA1C2070BD41007E
:107F800001D5092070BD810001D50A2070BDC10056
:107F900001D50B2070BD010101D50C2070BD410140
:107FA00001D50D2070BDC10101D50E2070BD0102AB
:107FB00001D50F2070BD410201D5102070BD810296
:107FC00001D5112070BDC10201D5122070BD010381
:107FD00001D5132070BD410301D5142070BD81036C
:107FE00001D5152070BDC10301D5162070BD010457
:107FF00001D5172070BD410401D5182070BD810442
:1080000001D5192070BD000701D51A2070BD284682
:1080100070BD000008E0FFFD0146002009684A6BC2
:1080200012F0450FFBD04A6B520702D50320042201
:1080300007E04A6BD20702D001208863704740F204
:10804000FF528A6370472DE9F041044600681546E7
:108050000E460027416B11F0450FFBD0416B4907DD
:1080600003D503210422826304E0416BC90704D0D5
:10807000012181630846BDE8F081FFF74FFEB04261
:1080800012D1216840F2FF5088630020FFF74EFEB6
:1080900010F4604F03D0810404D51320EBE7000CEB
:1080A000288007E0410401D51020E4E7000401D551
:1080B0000F20E0E73846DEE70246292012684FF439
:1080C0008031536B13F0450307D0012305E0536B58
:1080D00013F0450300D00123491E0BB90029F6D146
:1080E000536BC3F3800301B113B10320042104E0F7
:1080F000516B490602D500204021916370472DE95C
:10810000F04F8DB000250F460B9508261021CDE9C4
:10811000006140210C950446CDE902150801049048
:10812000A84669462068FFF722FE10212046FFF787
:10813000FDFE002844D1A08C694600040090372041
:1081400001902068FFF713FE37212046FFF7EEFE6F
:10815000002835D1401ECDE9050630204FF0020938
:10816000CDE907090120CDE90980B246464605A9B7
:108170002068FFF7C1FD3320CDE900606946206823
:10818000FFF7F5FD33212046FFF7D0FE060017D19B
:108190000DF12C0840F22A6B2068416B11EA0B0F9D
:1081A00008D1416B8902F7D5FFF7DEFD48F82500BD
:1081B0006D1CF1E7416B090705D5C0F838A0042014
:1081C0000DB0BDE8F08F416B890703D5C0F838903A
:1081D0004846F5E7416B890603D5202181630620D7
:1081E000EEE7416B890504D54FF4007181630720E8
:1081F000E6E740F2FF5181630B9800BA78600C9873
:1082000000BA38603046DBE70E4810B50C49016013
:10821000002141608160C16001614161816100F1C3
:108220006001FAF765FE08B1012010BD4FF400614E
:108230000448FAF7C3FF0028F7D0022010BD000061
:10824000002C01409005002070B586B00446012046
:10825000ADF8140000252068FFF763FD58B3206ACD
:1082600004285DD000200221C0268DE84300039041
:108270004802049069462068FFF779FD2046FFF721
:10828000CBFE050018D1FFF751FDA0630420FFF7D6
:108290004DFDE0630820FFF749FD20640C20FFF747
:1082A00045FD6064206A48B1012807D0062805D042
:1082B000022803D011E0252006B070BD03200190F4
:1082C0004020029069462068FFF751FD05AA03216E
:1082D0002046FFF7B8FE0500EED1206A04281FD023
:1082E000BDF814006062000400900920CDE9010689
:1082F00069462068FFF73BFD2046FFF78DFE05002D
:10830000DAD1FFF713FDA0620420FFF70FFDE06252
:108310000820FFF70BFD20630C20FFF707FD6063CB
:108320002846C9E770B586B0044600260D4600967B
:10833000A18C090401910D2102914021CDE9031680
:108340000801059001A92068FFF711FD2068416B25
:1083500011F0450FFBD0416B490703D503210422DF
:10836000826304E0416BC90704D0012181630846A0
:1083700006B070BDFFF7D2FC0D2838D1216840F25D
:10838000FF5088630020FFF7D1FC0090C0F343202A
:1083900028703249009808425DD00098002801DA20
:1083A0001C20E5E7400001D50920E1E700988000A6
:1083B00001D50A20DCE70098C00001D50B20D7E7E3
:1083C0000098000101D50C20D2E70098400101D5AA
:1083D0000D20CDE70098C00101D50E20C8E7009818
:1083E000000201D50F20C3E70098400201D51020FC
:1083F000BEE70098800201D51120B9E70098C002BD
:1084000001D51220B4E70098000301D51320AFE78F
:108410000098400301D51420AAE70098800301D5F5
:108420001520A5E70098C00301D51620A0E7009805
:10843000000401D517209BE70098400401D51820BF
:1084400096E70098800401D5192091E7009800076D
:1084500001D51A208CE730468AE7000008E0FFFDCE
:108460002DE9F04F87B04FF0000904468DF81490C5
:10847000DFF870A14F464D464E46C846CAF8A09058
:108480000068FFF76DFC0120F9F7F6FA4FF0010BD9
:10849000CAF8A0B0CDE90099CDF808904FF48060FB
:1084A000CDE9039069462068FFF761FC226800234C
:1084B0004FF48030516BC1F3C01104E0516B401E8A
:1084C000C1F3C0110CD00029F8D048B140F2FF50E0
:1084D00090638DF814309DF8140000287DD101E0E0
:1084E0000323F6E74FF4D570009008204FF04009C1
:1084F000CDE9010969462068FFF739FC2046FFF7FE
:10850000DBFD8DF814009DF8140018B94FF0804879
:10851000C4F820B04FF0000A3720CDE900A069462A
:108520002068FFF724FC37212046FFF7FFFC8DF879
:1085300014009DF814004FF6FF7180B34DE0372012
:10854000CDE900A0CDF808904FF48067CDE903A7EE
:10855000564669462068FFF70AFC37212046FFF798
:10856000E5FC8DF814009DF8140088BB1E4948EA0C
:10857000010000902920CDE90109CDE90367694692
:108580002068FFF7F4FB20680021426B12F0450FD2
:10859000FBD0426B520703D50321042202E00EE018
:1085A00040F2FF5282638DF814109DF8140078B9E0
:1085B0000020FFF7BBFBC60F07466D1C00E08B4693
:1085C0000EB95D45BBD35D4503D31B208DF8140068
:1085D00003E0780001D5022020629DF8140007B066
:1085E000BDE8F08F00802542000010802DE9FC5F7F
:1085F000924605464FF00008CE0D4F02F7F7E1FD19
:10860000A9074FF400701CD000244FF0010B8146E5
:1086100014E06002C2191249CDE9009B46EBE073F9
:10862000A1F1B800FAF7F6FC80464A460C49284604
:10863000F7F711FE641CE4B205F500755445E8D364
:1086400009E0CDE9000A06483A4633462946B838DB
:10865000FAF7E0FC8046F7F7B6FD4046BDE8FC9F20
:108660004806002030B587B0002504460595284609
:108670000695FFF75BFB800102D50E2007B030BDE9
:1086800005A92046FFF73BFD0028F7D10698C00357
:108690001FD5A08C6946000400903720019040202F
:1086A000CDE90205000104902068FFF760FB372147
:1086B0002046FFF73BFC0028E0D10620CDE9005022
:1086C00069462068FFF753FB06212046FFF72EFC82
:1086D000D4E72520D2E730B587B0002504460595BC
:1086E00028460695FFF722FB800102D50E2007B031
:1086F00030BD05A92046FFF702FD0028F7D10698F6
:10870000400320D5A08C69460004009037200190DA
:108710004020CDE90205000104902068FFF727FB07
:1087200037212046FFF702FC0028E0D1022000900C
:108730000620019069462068FFF719FB06212046B4
:10874000FFF7F4FBD3E72520D1E700002DE9FC5F1C
:10875000914605464FF00008CE0D4F02F7F731FD68
:10876000A8074FF400711DD000248A464FF0010B7A
:1087700015E0D046524629461248F7F76CFD6002D4
:10878000C2191049CDE9008B46EBE073A1F1B800A6
:10879000FAF743FD641C8046E4B205F500754C45CC
:1087A000E7D309E0CDE9001906483A4633462946A1
:1087B000B838FAF732FD8046F7F705FD4046BDE8C8
:1087C000FC9F00004806002010B5124C1048022102
:1087D00020604FF4827060600020A060C4E9030153
:1087E000012161614902A1613821C4E90710606279
:1087F000A0620720E0622046FAF7F7FD20680168D2
:1088000041F040010160BDE81040FF2000F004B8D5
:10881000005001404808002001B582B04FF47A7042
:108820000090012301AA02A90248FAF74BFE9DF825
:1088300004000EBD480800200B4A10B511680B68F3
:1088400023F040030B6011680B684FF6C774234098
:108850000B6011680B6803430B601068016841F0FE
:108860004001016010BD0000480800202DE9F047DC
:108870001D4690460F460446F9F702FA06465FEA9F
:1088800008004FF000084FF4005A4FF0010926D0BD
:1088900034E0681C23D025B1F9F7F2F9801BA84217
:1088A0001DD92068416821F0E0014160206801681D
:1088B00021F040010160A06A504509D1206801689B
:1088C00021F4005101602068016841F40051016009
:1088D00084F8519084F850800320BDE8F087206828
:1088E000806837EA0000D4D10DE0681C06D0002D66
:1088F000D7D0F9F7C5F9801BA842D2D82068806884
:1089000037EA0000F1D00020E7E7704770B51E4C51
:1089100092B00025266846F080562660246804F050
:1089200080541194194C266846F440462660246809
:108930000DF1240C04F4404411940124009401949A
:10894000022406948CE80D006605CDE907616846AF
:10895000F9F72CFF00B1FEE7F9F70CFC00B1FEE7D8
:108960000CA90F2081E831004FF4A0500F904FF474
:108970008050109005210CA8F9F794FD002800D034
:10898000FEE712B070BD00004038024000700040A9
:10899000F9F77CB91048016841F4700101600F4893
:1089A000016841F0010101600C4A002108321160A8
:1089B00002680B4B1A400260031D0A4A1A600268E3
:1089C00022F48022026005480C30016002495806FA
:1089D000803908607047000088ED00E000380240F0
:1089E000FFFFF6FE103000240148FAF790BF0000A8
:1089F000B0C30220094A10B5074BC2E9003100217B
:108A0000C2E9021010461161FAF73AFFBDE81040C2
:108A10000248FAF76FBF000000040040B0C3022014
:108A200010B50A4C2068C068C043C00709D1084887
:108A30000069804721680020486221686420C8627C
:108A4000E06021686FF00100086110BD40C10220A4
:108A50000C020020F0B50268234D244E244FDFF8AD
:108A600094C0254B4FF0804EA84209D0704507D0E6
:108A7000B04205D0B84203D0604501D0984203D13E
:108A800022F070044A682243A8421BD0704519D0D6
:108A9000B04217D0B84215D0604513D0984211D0DB
:108AA000164CA0420ED0164CA0420BD0154CA04242
:108AB00008D0154CA04205D0144CA04202D0144C52
:108AC000A04203D122F44074CA68224302608A683B
:108AD000C2620A688262A84201D0984201D1096943
:108AE000016301214161F0BD00000140000400402C
:108AF00000080040000C004000040140004001401C
:108B0000004401400048014000180040001C0040A3
:108B100000200040F8B5064610480D4600240168C4
:108B200041F0040101600068032200F0040000909D
:108B300011461E20F9F7ECFA1E20F9F7DDFA094A72
:108B400007481060C2E90154C2E903641046FAF70D
:108B500097FEBDE8F8400348FAF7CCBE4038024023
:108B60000008004040C1022010B590F839102229B9
:108B700003D0322901D0022010BD8168B1F5805F99
:108B800011D00169002901681FD0496801F07F03F5
:108B9000816A4A1C82620B70C18D491E0904090C4E
:108BA000C18518D02FE00269816A002A02685268E4
:108BB00005D0D2B20A80816A491C8162ECE7C2F317
:108BC00008020A80816A891CF7E74A68816A4B1C9F
:108BD00083620A70E0E70168CA6822F02002CA6076
:108BE00090F83910322910D00168CA6822F48072D6
:108BF000CA6001684A6922F001024A61012180F8D5
:108C00003910FBF7A6F8002010BD1221F7E700008D
:108C10002DE9F041044600680169E26821F4405101
:108C20000A4302612068C16849F20C6291432369DA
:108C3000A268E5691A4363692B431A430A43C26079
:108C40002068416921F44072A16911434161E069E2
:108C500064263225B0F5004F484A494920681DD0A6
:108C6000884201D0904269D1F9F750FD00EBC00174
:108C700001EB00106168B0468900B0FBF1F1B1FB77
:108C8000F8F6F9F743FD00EBC00101EB0010616855
:108C90008900B0FBF1F7F9F739FD68E0884201D0AF
:108CA000904219D1F9F732FD00EBC00101EB001041
:108CB0006168B0464900B0FBF1F1B1FBF8F6F9F795
:108CC00025FD00EBC00101EB001061684900B0FB1D
:108CD000F1F7F9F71BFD18E0F9F702FD00EBC00111
:108CE00001EB00106168B0464900B0FBF1F1B1FB47
:108CF000F8F6F9F7F5FC00EBC00101EB0010616834
:108D00004900B0FBF1F7F9F7EBFC00EBC00101EB18
:108D1000001061684900B0FBF1F1B1FBF8F06FF0B1
:108D20001801484307EB800005EB0011B1FBF8F098
:108D3000216866F31F108860BDE8F081F9F7D0FC68
:108D400000EBC00101EB00106168B0468900B0FB88
:108D5000F1F1B1FBF8F6F9F7C3FC00EBC00101EB50
:108D6000001061688900B0FBF1F7F9F7B9FC00EB7E
:108D7000C00101EB001061688900CCE700140140DC
:108D80000010014090F83910122903D0322901D087
:108D9000022070478168B1F5805F016A0BD04A1CE0
:108DA0000262026809785160C18C491E0904090CED
:108DB000C1840ED017E009880268C1F30801516030
:108DC00001690029016A02D0491C0162ECE7891C93
:108DD000FBE70168CA6822F08002CA600068C168C7
:108DE00041F04001C160002070472DE9F0471D4669
:108DF00090460F460446F8F743FF06465FEA080030
:108E00004FF000094FF0010808D030E0681C05D091
:108E100095B1F8F735FF801BA8420DD8206800688F
:108E200037EA0000F2D127E0681C20D025B1F8F71E
:108E300027FF801BA8421AD92068C16821F0800151
:108E4000C1602068C16821F02001C1602068C1684C
:108E500021F48071C1602068416921F00101416104
:108E600084F8398084F838900320BDE8F0872068C2
:108E7000006837EA0000D7D00020F6E738B5184878
:108E800000680068C043800622D44FF47A73012240
:108E900069461348FAF7F8FE124A1088010417D4FD
:108EA00041049DF800104FF0000304D50A290ED1AB
:108EB00040F4004012E00D290ED0C0F30D04084D1F
:108EC000401CC83D80B229551080C72800D91380A6
:108ED0000348FAF7E5FD38BD40F480401080F7E71D
:108EE000F00300201C000020FEE7000010B500F099
:108EF00045F900F0EDF8074C0020C4F89802C720AF
:108F000004F52674FFF788FC01202060BDE81040BE
:108F100000F0DEB80080424270B5040300F02EF984
:108F200000F0D6F8104D0020C5F898022020FFF779
:108F300073FC0E480088A0F56F41183902D1200E4D
:108F4000FFF76AFCC4F30740FFF766FCC4F3072091
:108F5000FFF762FCE0B2FFF75FFC0120C5F8980262
:108F6000BDE8704000F0B4B80080424234000020F8
:108F700070B51A4886B00025016841F020010160F3
:108F80000068012400F0200005904020CDE9000495
:108F90000220CDE9024069461148F8F779FD114EEB
:108FA000C6F89842FFF710FC0020FFF745FC00F0E0
:108FB00051F80D490880A0F56F4118390BD10320F5
:108FC00000F06AF8C00706D1C6F89852B720FFF73C
:108FD00023FCC6F8984206B070BD0000303802404D
:108FE0000014024000804242340000202DE9F0418C
:108FF000164F0646002015460C46C7F89802032077
:10900000FFF70AFC12480088A0F56F41183902D119
:10901000200EFFF701FCC4F30740FFF7FDFBC4F38C
:109020000720FFF7F9FBE0B2FFF7F6FB002405E0AD
:10903000FF20FFF7F1FB3055641CA4B2AC42F7D31C
:109040000120C7F89802BDE8F0810000008042428C
:109050003400002070B50F4D0024C5F898429020D0
:1090600005F52675FFF7D8FB0020FFF7D5FB00209C
:10907000FFF7D2FB0020FFF7CFFBFF20FFF7CCFB71
:1090800044EA0024FF20FFF7C7FB204301212960A9
:1090900070BD00000080424210B5012803D00228B4
:1090A00003D0032803D0052002E0352000E015207E
:1090B000064C0021C4F8981204F52674FFF7ACFBA7
:1090C000FF20FFF7A9FB0121216010BD0080424273
:1090D00010B50120FFF7E0FFC007FAD110BD000076
:1090E0002DE9F05FC1F30B06DFF88C800F0BC6F59E
:1090F00080548A4681461546A24200D81446390358
:109100008B464FF480524046FFF770FF002006E088
:10911000321818F80210FF2903D1401C80B2A04277
:10912000F6D3A04221D23846FFF7F6FE002006E033
:1091300019F800208319401C08F8032080B2A042CF
:10914000F6D359464FF48052404600F027F8A54226
:109150000FD0281BA144A244002685B24FF48054AE
:109160007F1CA542CBD82C46C9E72246514648462B
:10917000EBE7BDE8F09F0000A008002010B5064C0A
:109180000020C4F89802062004F52674FFF744FB7B
:109190000120206010BD0000008042422DE9F04116
:1091A0000746C8B2C0F580740E461546A24200D8E4
:1091B00014464FF4807822463146384600F00EF8C7
:1091C000A54208D0281B2744264485B24446A54220
:1091D000F1D82C46EFE7BDE8F08100002DE9F04121
:1091E00015460C460646FFF7C9FF154F0020C7F885
:1091F00098020220FFF710FB12480088A0F56F418B
:10920000183902D1200EFFF707FBC4F30740FFF720
:1092100003FBC4F30720FFF7FFFAE0B2FFF7FCFA05
:10922000002404E0305DFFF7F7FA641CA4B2AC42FE
:10923000F8D30120C7F89802BDE8F041FFF748BF16
:1092400000804242340000200FB4054B10B503A942
:10925000044A029800F092FB10BC5DF814FB000079
:10926000A1D60008200000200FB4084B10B504A9B7
:1092700002AA039800F082FB044602A9002000F035
:1092800014FF204610BC5DF814FB0000ABA00008E2
:10929000014B024A00F072BBA1D60008200000205A
:1092A00003B401984100009850EAC12018BF04207F
:1092B0004A0D18BF40F0010040F2FF72B2EB515F5F
:1092C00008BF40F00200012808BF052002B0704727
:1092D00030B583B0044600F06BFA9FED090B0546EC
:1092E0008DED000B002221466846F7F70AF9284663
:1092F00000F074FA9DED000B03B030BD00000000DB
:10930000000000000000000070B52DED020B2DEDF7
:109310000A8B82B00D98C40F20F00045AE488542FC
:1093200048D3AE48854219D30C99C5F313000843BE
:1093300009D09DED0C0B02B0BDEC0A8B02B0BDE86C
:10934000704000F009BA002C14BF9FEDA50B9DEDF5
:109350000C0B02B0BDEC0A8B02B070BD9FEDA20BEE
:1093600053EC102B9DED0C0B51EC100BF7F706FB9B
:109370000AD2022000F032FA02B0BDEC0A8B02B031
:10938000BDE8704000F0F4B99FED990B53EC102B41
:109390009DED0C0B51EC100BF7F7D8FA0AD2022016
:1093A00000F01CFA02B0BDEC0A8B02B0BDE87040C0
:1093B00000F0EEB990489FED92BBA8425CD2924873
:1093C000854219D29148784400EBC40090ED000B1F
:1093D00053EC102B9DED0C0B51EC100BF7F7F9F93A
:1093E00041EC1A0B8A48784400EBC40090ED009BD6
:1093F000C4F10100041B36E09FED870B53EC102BEA
:109400009DED0C0B51EC100BF6F763FF41EC100BCC
:109410008348784400EBC40090ED001B51EC100B26
:1094200053EC112BF7F734F9F7F759FA0446F7F72D
:1094300045FA41EC180B9FED7C0B53EC102BF6F723
:1094400048FF9DED0C1B53EC112BF7F7C5F941ECD0
:109450001A0B9FED770B51EC180B53EC102BF6F712
:1094600038FF41EC190B51EC1A0B53EC192BF7F7A1
:10947000B0F9CDE90C011BE06F48854217D29FED92
:10948000700B53EC102B9DED0C0B51EC100BF7F700
:10949000FFF853EC1B2BF7F771FA08D29DED0C0B7C
:1094A00053EC1B2B51EC100BF7F7F2F86EE0002495
:1094B0009DED0C0B53EC102B51EC100BF6F709FF44
:1094C00041EC180B60480521B0EE480AF0EE680A3E
:1094D000784400F0C5F853EC182B51EC100BF6F75C
:1094E000F8FE9DED0C1B53EC112BF7F775F941ECD1
:1094F000180B9FED570B5CB353EC182B51EC100B72
:10950000F7F767F99DED0C0B41EC1C0B53EC182B96
:1095100051EC100BF6F7DDFE53EC1C2BF7F75FF95F
:1095200053EC192BF7F758F953EC1A2BF7F751F9BD
:1095300053EC1B2BF7F750F9CDE900016FF47F7066
:10954000844226DB01EB045001909DED000B00E707
:1095500053EC102B51EC180BF7F73BF99DED0C0B6E
:1095600041EC190B53EC182B51EC100BF6F7B1FE34
:1095700053EC192BF7F733F99DED0C1B53EC112B22
:10958000F7F727F953EC1B2BF7F726F941EC100BF3
:10959000DFE608464FF07A5101EB04519FED2E0BA8
:1095A000084453EC102B01909DED000B51EC100B77
:1095B000F6F78FFE0D4645EC100B044651EC100BF0
:1095C000FFF76EFE042808BF00F0E2F845EC104BF0
:1095D000BFE6000000000000422E86400000F07F41
:1095E0000000000000000000EF39FAFE422E864025
:1095F00051302DD5104987C0422ED63F00000000C3
:10960000000000000000F03FB2A2F03FEE6B03004C
:10961000DE6B030000000000FE822B654715F73F5C
:10962000926B0300000000000000E0FE422EE63FC7
:10963000763C7935EF39EA3D0000303E000000000D
:109640009C7500883CE4377E046B0300000000003A
:109650000000000000000040000000000000700159
:1096600070B504462DED028B4D1E00EBC500B0EE2B
:10967000408AF0EE608A90ED000B35F0060017D0BE
:1096800053EC182B51EC100BF6F723FE41EC100BAA
:109690006D1E04EBC50090ED001B51EC100B53EC5C
:1096A000112BF6F7F5FF41EC100B35F00600E7D172
:1096B000022D36D0042D1CD0062D1CBFBDEC028B14
:1096C00070BD53EC182B51EC100BF6F702FE94ED25
:1096D0000A1B53EC112BF6F7DBFF53EC182BF6F7B4
:1096E000F8FD94ED081B53EC112BF6F7D1FF41EC7C
:1096F000100B53EC182B51EC100BF6F7EAFD94ED20
:10970000061B53EC112BF6F7C3FF53EC182BF6F79F
:10971000E0FD94ED040B53EC102BF6F7B9FF41EC90
:10972000100B53EC182B51EC100BF6F7D2FD94ED07
:10973000021B53EC112BF6F7ABFF53EC182BF6F78B
:10974000C8FD94ED001B53EC112BF6F7A1FFBDEC07
:10975000028B41EC100B70BD10B553EC102B51EC8B
:10976000100BF6F795FF41EC100B10BD0000000048
:109770009FED050B10B553EC102B51EC100BF6F7C9
:10978000A8FD41EC100B10BD0000000000000070AF
:109790009FED050B10B553EC102B51EC100BF6F7A9
:1097A00098FD41EC100B10BD0000000000000010FF
:1097B00001480068704700002403002002E008C848
:1097C000121F08C1002AFAD170477047002001E03B
:1097D00001C1121F002AFBD1704700000149086037
:1097E00070470000240300202DE9FF5F82B00021B4
:1097F000DDE90430020DDDF840B0034318D044F633
:109800001050A2F2FF3242431514119801281FD0C4
:10981000A5EB0B00401C5FEA000A4FF000064E4F1C
:10982000DFF83891B046504615D5CAF1000413E070
:10983000119801244AA3012801D16FEA0B01029873
:10984000119AC0E90031C0E9024206B0BDE8F09FBC
:10985000CBF10000DFE704460021404A491842EB03
:109860000450CDE9001012E0E00707D032463B4635
:1098700040464946F6F72DFD8046894632463B462E
:1098800010461946F6F725FD06460F466410002CD3
:10989000EAD1DDE90401DDE90023BAF1000F06DABF
:1098A000F6F717FD42464B46F6F713FD05E0F6F7CF
:1098B00096FF42464B46F6F792FF04460E460022BC
:1098C000284BF7F75BF803D84FF0FF30014607E06D
:1098D0000022254B20463146F6F7DAFEF7F71EF850
:1098E000102409E0002C0ADB0A220023F6F782FC90
:1098F000039B30321A55641E50EA0102F2D1641CF7
:10990000039AC4F111031444119A012A03D00122CD
:1099100008430DD10AE0084304D000204FF0110B9A
:10992000119072E7A3EB0B056D1E0DE05B4504DDA6
:109930004FF0000205F1010504E003DA4FF00002E8
:10994000A5F10105002AECD002981199C0E9023175
:10995000C0E9004579E70000000014400000F03F36
:10996000300000000000F0430000E03F30380A28DB
:1099700001D2012070470020704700002DE9FF4F01
:1099800095B09B468946064600250FE2252877D1EB
:1099900000242746F84A0121059400E0044316F804
:1099A000013F203B01FA03F01042F7D130782A281A
:1099B00011D06FF02F033078A0F13002092A16D8A9
:1099C000059A44F0020402EB820203EB42021044C7
:1099D000761C0590EFE759F8042B0592002A03DA6C
:1099E000504244F40054059044F00204761C307850
:1099F0002E2816D116F8010F44F004042A280DD0A1
:109A00006FF02F023078A0F13003092B09D807EB53
:109A1000870302EB4303C718761CF3E759F8047B6E
:109A2000761C30786C280FD006DC4C2817D06828BC
:109A30000DD06A2814D104E0742810D07A280FD1F0
:109A40000DE044F400140AE044F4801401E044F40E
:109A500040147278824202D104F58014761C761C80
:109A6000307866280BD013DC582877D009DC002822
:109A700075D04528F6D04628F4D047281AD19DE164
:109A800018E0632835D0642879D0652812D195E193
:109A9000702873D008DC6728F1D069286FD06E2851
:109AA0000DD06F2806D1B5E073282CD0752875D05D
:109AB000782874D05A46179990476D1C75E1C4F305
:109AC0000250022809D003280DD0D9F8001004282C
:109AD0000DD00D6009F1040967E1D9F80010EA170B
:109AE000C1E90052F6E7D9F800100D80F2E70D70D9
:109AF000F0E719F8041B8DF8001000208DF8010024
:109B0000EA46012003E059F804AB4FF0FF3061074B
:109B10004FF0000102D40DE008F101018846B9427E
:109B20000FDA8045F8DB1AF808100029F4D108E0B4
:109B300008F1010188468142FADB1AF80810002971
:109B4000F6D105985B46A0EB080721463846179AE0
:109B500000F094FA284400EB080507E04DE029E105
:109B60000DE01AF8010B5A4617999047B8F1010811
:109B7000F7D25B4621463846179A13E142E00A22A3
:109B80000092C4F302524FF0000A022A08D059F89A
:109B900004CB032A4FEAEC710AD00DE029E02AE059
:109BA00009F1070121F00702F2E802C1914609E03C
:109BB0000FFA8CFC4FEAEC71042A03D14FFA8CFCAB
:109BC0004FEAEC71002907DA0A460021DCF1000CAB
:109BD00061EB02012D2202E0220504D52B228DF833
:109BE0000420012203E0E20701D02022F7E790469B
:109BF00059E00A2102E010220DE010214FF0000A86
:109C000000910BE010224FF0000A44F004040827F2
:109C1000009203E008224FF0000A0092C4F30252BF
:109C2000022A05D059F804CB0021032A08D009E004
:109C300009F1070121F00702F2E802C1914605E0AF
:109C40001FFA8CFC042A01D10CF0FF0C4FF0000825
:109C5000220728D5702806D0009B83F0100353EA12
:109C60000A0305D00EE040228DF80420012208E00E
:109C70005CEA010206D030228DF804208DF8050040
:109C800002229046009B83F0080353EA0A030AD19C
:109C90005CEA010201D1620705D530228DF804206B
:109CA0004FF001087F1E582804D034A003900EA85E
:109CB00002900DE036A0F9E753466046009AF6F7A9
:109CC00099FA84460398825C0298401E02900270C2
:109CD0005CEA0100F0D1029806A9081A00F1200AF6
:109CE000600702D524F4803400E00127574502DDE7
:109CF000A7EB0A0000E0002000EB0A0100900598A5
:109D00004144401A0590E00306D45B462146179A69
:109D1000059800F0B3F90544002706E001A85A466B
:109D2000C05D179990476D1C7F1C4745F6DBE0032B
:109D30000CD55B462146179A059800F09FF905441B
:109D400004E030205A46179990476D1C0099481E30
:109D500000900029F5DC08E0029802995A46007844
:109D6000491C0291179990476D1CBAF10001AAF1A4
:109D7000010AF1DC65E100000928010030313233CD
:109D80003435363738396162636465660000000037
:109D90003031323334353637383941424344454621
:109DA0000000000000F058F90544761C30780028C7
:109DB0007FF4ECAD19B02846BDE8F08F620700D4FF
:109DC000062709F1070222F0070CFCE80223E1460E
:109DD00003F000485FEA080C02D00FF2702C0DE08F
:109DE0005FEA045C02D50FF2682C07E05FEAC47CEE
:109DF00002D00FF2602C01E0AFF2700C4FF0FF3890
:109E000023F00043CDF850C065280CD006DC45286F
:109E100009D046281DD047283DD13DE0662818D0FE
:109E200067287ED138E00021112F01DB112000E0EE
:109E3000781CCDE9000106A90EA8FFF7D5FCDDE9E5
:109E40000F010E9A03910021009207F1010A04917B
:109E50004DE04FF000400097CDE9011006A90EA893
:109E6000FFF7C2FCDDE90F0203920E9B119900225D
:109E7000DDF80CA00093049211B9791C00EB010AE3
:109E8000B7EB0A0004D4C0F1FF3007F1010A0490D7
:109E9000AAEB0700019044E0012F00DA012700211E
:109EA000112F01DD112000E03846CDE9000106A99F
:109EB0000EA8FFF799FCDDE90F010E9A039100212E
:109EC00004910092BA4621070CD40399514500DA57
:109ED0008A46BAF1010F05DD009AAAF10101515C31
:109EE000302908D0B84202DA10F1040F06DA012155
:109EF000CDE9011015E0AAF10101E9E7002805DC30
:109F0000049901440491AAEB000102E0411C51456F
:109F100000DD8A460499401A401C01904FF0004031
:109F20000290200704D40198504501DBCDF804804D
:109F300000208DF84F0002980DF14F07B0F1004F4F
:109F400025D02B200E9002984FF0020800280CDA42
:109F5000404202902D200E9007E00A210298F6F769
:109F60007FFA3031029007F8011DB8F10001A8F125
:109F70000108F2DC02980028EFD1791E0E980870D3
:109F8000307800F0200040F0450007F8020D12A8DC
:109F9000C01B00F107081498007800B1012000EB05
:109FA0000A01019801EBE07105984144401A401EF6
:109FB0000590E00306D45B462146179A059800F009
:109FC0005DF805441498007818B15A4617999047DF
:109FD0006D1CE00324D55B462146179A059800F0D6
:109FE0004DF805441CE00498002807DBDDE9030177
:109FF000884203DD0098405C179901E017993020F2
:10A000005A469047049805F10105401C04900198B8
:10A01000401E019004D12E205A46179990476D1C7E
:10A02000BAF10001AAF1010ADDDC05E017F8010B25
:10A030005A46179990476D1CB8F10001A8F1010824
:10A04000F4DC5B462146179A0598ABE62D0000002C
:10A050002B000000200000002DE9F04104460025FF
:10A060001E461746880404D405E039462020B04730
:10A070006D1C641EF9D52846BDE8F0812DE9F0413C
:10A08000044600251E469046C80301D5302700E04F
:10A090002027880404D505E041463846B0476D1CAA
:10A0A000641EF9D52846BDE8F0810A68531C0B6090
:10A0B000107070472DE9F0410D460746810090462B
:10A0C000012005F04BFA0646002405FB08F506E0E2
:10A0D0002946012005F042FA46F82400641CBC42DF
:10A0E000F6DB3046BDE8F0812DE9F04180462DEDEC
:10A0F000028B14460E469FED258A900003F0BEFEAB
:10A100000546002714E058F82700F6F77AF941ECE5
:10A11000100BFFF7F9F851EC100BF6F785F900EE8C
:10A12000100A05EB87007F1C30EE088A80ED000ADC
:10A13000A742E8DB00200AE005EB800191ED000A70
:10A1400006EB8001401CC0EE080AC1ED000AA042E7
:10A15000F2DB0027D6ED000A01200CE006EB8001BF
:10A1600091ED000AB4EEE00AF1EE10FA02DDF0EE35
:10A17000400A0746401CA042F0DB28467F1C03F043
:10A1800099FABDEC028B3846BDE8F0810000000072
:10A190002DE9F0470746C06A891E00EB1136C1F36E
:10A1A000C80501F007014FF0010A0AFA01F09846CC
:10A1B0009146C4B23146761C384605F0D9F810B144
:10A1C0000120BDE8F08752464FF40073791991F8E9
:10A1D000340010EA040C01D04FF0010CC44501D149
:10A1E0000220EEE7604081F83400B9F10100FA7016
:10A1F0008146E6D0600010F0FF04E7D101246D1C19
:10A200009D42E3D3D6E7000070B504460020E0701D
:10A21000401E2063204605F0ABF808B1042070BD55
:10A2200004F2322003F08CFCA0F52A41553901D00C
:10A23000032070BD04F16A0003F04CFC0B4DB5EB3C
:10A24000002F06D004F1860003F044FCB5EB002F8C
:10A2500001D1002070BD082205A104F1370003F0F0
:10A2600043FE08B1022070BD012070BD004641547C
:10A2700045584641542020200000000000E0401CCA
:10A2800002780AB18A42FAD1D0B2704770B5154649
:10A290000168846C680A4A8940EAC350590A00235D
:10A2A000241DF5F7A7FF02CC21B1884204D3401A40
:10A2B000241DF8E7002070BD2168084470BD826944
:10A2C000891E921E8A4201D800207047C26A4089C6
:10A2D00001FB0020704700002DE9F05F81468846B1
:10A2E00001F11A0003F02CFC88BB98F8000001274C
:10A2F00000F03F00401E00EB8001DFF85CA001EBA6
:10A30000C00400254FF6FF7B1AF8051001EB08008A
:10A3100003F016FC06466FB1FF2C18D202F01EFFA8
:10A32000074639F81400641C02F018FF87420ED16A
:10A33000374601E05E450AD16D1C0D2DE4D398F837
:10A340000000400606D52FB139F8140010B10020E6
:10A35000BDE8F09F0120FBE7A45301082DE9F04F71
:10A36000ADF23C4DFAA0FEF76FFFFF4D0024686888
:10A3700050F82400F6F745F841EC100B214653EC59
:10A38000102BFAA0FEF760FF641C0A2CEFDBFBA089
:10A39000FEF75AFF4AF29021012005F0DFF88A907B
:10A3A000686864218A9AF7F73DFB42F2107804222C
:10A3B000444641462020FFF77DFE06460422214602
:10A3C0002020FFF777FE0546042221462020FFF7D4
:10A3D00071FE044600274FF0200A4FF0180B4FF093
:10A3E0001C09EA480323416807EBC70001EB800220
:10A3F00092ED000A042202EB80020A448DED810AEC
:10A4000092ED000A082202EB80020A448DED820AD6
:10A4100092ED000A0C2202EB80020A448DED830AC1
:10A4200092ED000A102202EB80020A448DED840AAC
:10A4300092ED000A142202EB80020A448DED850A97
:10A4400092ED000A0BEB80020A448DED860A92ED34
:10A45000000A09EB80020A448DED870A92ED000A9A
:10A460000AEB800008448DED880A90ED000A81AA6D
:10A470008DED890A56F82700009066218A98F6F734
:10A4800017FD7F1C202FACDB0027C14855F8272083
:10A490004146406800EB870090ED000A56F827001F
:10A4A000F6F7B5FC7F1C202FEFDB0027414654F860
:10A4B000272055F82700FDF7FBFB7F1C202FF5DB3D
:10A4C000042240F6C4112020FFF7F4FD8046002747
:10A4D000022358F82700009054F827001A466421F8
:10A4E000FDF77AFB7F1C202FF2DBAAA0FEF7ACFE63
:10A4F00001208A9905F026F82021284603F002F968
:10A500002021304603F0FEF82021204603F0FAF81F
:10A5100004224FF429612020FFF7CCFD05460024DA
:10A52000322155F8242058F82400F7F77BFA641CF0
:10A53000202CF5DB40F6C414042221462020FFF72E
:10A54000B9FD8C90042221464020FFF7B3FD8B908B
:10A55000042221464020FFF7ADFD8A9004222146C7
:10A560004020FFF7A7FD06460027CB46002407EB57
:10A57000C7098C4804EBC40101EB4911406803236F
:10A5800000EB810292ED000A042202EB81020244F8
:10A590008DED810A92ED000A082202EB810202444D
:10A5A0008DED820A92ED000A0C2202EB8102024438
:10A5B0008DED830A92ED000A102202EB8102024423
:10A5C0008DED840A92ED000A142202EB810202440E
:10A5D0008DED850A92ED000A182202EB81020244F9
:10A5E0008DED860A92ED000A0BEB810202448DED9F
:10A5F000870A92ED000A0AEB810108448DED880A72
:10A6000090ED000A81AA8DED890A8C98342150F8CA
:10A610002400009055F82400F6F74AFC641C202C16
:10A62000A7DB8B983222202150F827308C98F6F740
:10A6300001FC7F1C402F99DBDFF86C91002440F671
:10A64000C417D9F80400394600EB840090ED000AE5
:10A650008A9850F824208B9850F82400F6F7D7FBFE
:10A66000641C402CEDDB00248A9856F824203946DF
:10A6700050F82400FDF71CFB641C402CF4DB042282
:10A6800040F271214020FFF715FD8146002402238E
:10A6900059F82400009056F824001A463221FDF79C
:10A6A0009BFA641C402CF2DB40A0FEF7CDFD29464E
:10A6B000012004F047FF2021404603F023F8202129
:10A6C0008C9803F01FF840218A9803F01BF8402172
:10A6D0008B9803F017F84021304603F013F804225A
:10A6E00040F2D9214020FFF7E5FC0646002419215D
:10A6F00056F8242059F82400F7F794F9641C402CEC
:10A70000F5DB40F27125042229464020FFF7D2FCF8
:10A710008B90042229468020FFF7CCFC04460422BB
:10A7200029468020FFF7C6FC8A9004222946802013
:10A73000FFF7C0FC00278C9000254FF0040A4FF073
:10A74000200B07EBC70805EBC50101EB881135E0CD
:10A75000434E4EC4A3D0CDD5FDD4DAD4CBD0D0A3B4
:10A76000A1A3A1A3A10D0A00A0C30220646174618A
:10A770005B25645D3A2025660D0A0000BFAACABCAD
:10A78000B5DAD2BBB2E3A3A10D0A000010C30220C8
:10A7900000C30220B5DAD2BBB2E3CDEAB1CFA3A1A8
:10A7A0000D0A000030C3022020C30220B5DAB6FE35
:10A7B000B2E3CDEAB1CFA3A10D0A0000A74803235D
:10A7C000406800EB810292ED000A0AEB810202442C
:10A7D0008DED810A92ED000A082202EB810202440B
:10A7E0008DED820A92ED000A0C2202EB81020244F6
:10A7F0008DED830A92ED000A102202EB81020244E1
:10A800008DED840A92ED000A142202EB81020244CB
:10A810008DED850A92ED000A182202EB81020244B6
:10A820008DED860A92ED000A1C2202EB81020244A1
:10A830008DED870A92ED000A0BEB810108448DED46
:10A84000880A90ED000A81AA8DED890A8B981B2158
:10A8500050F82500009056F82500F6F729FB6D1CEE
:10A86000402DFFF670AF54F82730192240218B9805
:10A87000F6F7E0FA7F1C802FFFF65EAFDFF8E0818D
:10A88000002540F27127D8F80400394600EB850016
:10A8900090ED000A8A9850F8252054F82500F6F724
:10A8A000B6FA6D1C802DEEDB00258C98394650F8E9
:10A8B00025208A9850F82500FDF7FAF96D1C802DA7
:10A8C000F3DB042290218020FFF7F4FB05460027EC
:10A8D000022355F82700009054F827001A46192142
:10A8E000FDF77AF97F1C802FF2DB4FF49037394661
:10A8F000012004F033FE034600900C2280212846FC
:10A90000F7F76EF857A0FEF79FFC3146012004F0E0
:10A9100019FE4021484602F0F5FE40218B9802F0D6
:10A92000F1FE80218A9802F0EDFE8021204602F09F
:10A93000E9FE80218C9802F0E5FE4FF4007B594639
:10A9400001A8F5F7A1FCDFF82C81DFF82C91002499
:10A950000DF1040A3E463146012004F0FFFD074692
:10A96000D8F8040004EBC40100EB4131324638460C
:10A97000F5F771FCD9F804003A4600EB84004FF477
:10A98000904190ED000A0098F6F77AFAFDF7AAF9DF
:10A990000AEB8400641C80ED000A802CDBDB802243
:10A9A000114601A8FDF754F934A0FEF74DFC8021B3
:10A9B000284602F0A7FE1C210DF20440F5F764FCC6
:10A9C000324E334F00240DF2044570685A4600EBB6
:10A9D000442181A8F5F73FFC786881AA00EB840048
:10A9E000802190ED000A01A8F6F74AFA05EB8400F1
:10A9F000641C80ED000A072CE7DB072211460DF2EC
:10AA00000440FDF725F923A0FEF71EFC07220DF5F3
:10AA100084610DF20440FFF767FB044607221146EC
:10AA20000DF58460FDF714F90DF5846000EB8400EA
:10AA3000DFED1C0A10ED010A20EE200A10EE100ACC
:10AA4000F5F7DFFC41EC100B17A053EC102B009432
:10AA5000FEF7FAFB0DF23C4DBDE8F08F50C302202B
:10AA600040C30220B5DAC8FDB2E3CDEAB1CFA3A15D
:10AA70000D0A000070C3022060C30220B5DACBC407
:10AA8000B2E3CDEAB1CFA3A10D0A000090C302202A
:10AA900080C30220B5DACEE5B2E3CDEAB1CFA3A1FF
:10AAA0000D0A00000000C84225662C204C6162653A
:10AAB0006C202564000000002DE9F04705685FEA7E
:10AAC0000108074626D04146384602F075FE0228A6
:10AAD00041D3411C1CD0A969814219D84646287827
:10AAE0004FF0FF3904281CD03446A869641CA042EA
:10AAF00002D80224022E0AD32146384602F05CFE18
:10AB000040B3012804D0411C02D0B442EDD1002052
:10AB1000BDE8F0872E6916B1A869B042DFD80126DA
:10AB2000DDE701223146284602F06FFB040039D0F0
:10AB3000601C37D001231A4621462846FFF728FB20
:10AB4000022808D0012808D0B8F1000F07D0F87902
:10AB5000022806D00DE00120DAE74846D8E70220B7
:10AB600006E0701C844204D0B868301AB861032033
:10AB7000F8712878042802D1F879022814D04E46BA
:10AB80004A462146284604F037FD40B9B8F1000096
:10AB90000AD001462246284604F02EFD20B10128A5
:10ABA0000FD001242046B3E72C61D5E90501891EA9
:10ABB000884201D2401E6861287940F00100287166
:10ABC000F0E73446EEE700002DE9F35F0E680098E9
:10ABD00000248846D0F840B02546705D6D1C2028C2
:10ABE00023D32F2821D05C281FD0FF2C46D2A0F1E0
:10ABF00081017D290BD8715D6D1C01EB0020A1F155
:10AC0000400280B23F2A02D380397F2936D2012107
:10AC100002F076FA070031D0802F12D201466BA0E5
:10AC2000FFF72CFB50BB0CE06D1C715D2F29FBD096
:10AC30005C29F9D07219C8F80020202805D2042513
:10AC40000EE02BF81470641CC7E7002508E00BEB3E
:10AC5000440030F8020C202801D02E2802D1641EB6
:10AC6000002CF4D100212BF814103CB100980B22D9
:10AC70002021806B03F04DF9002703E00620BDE89A
:10AC8000FC9F7F1C3BF817002028FAD02E28F8D014
:10AC90001FB145F0030500E0641E2CB10BEB44002E
:10ACA00030F8020C2E28F7D14FF00008C1464FF0C3
:10ACB000080A3BF817607F1C06B3202E03D02E2E07
:10ACC00004D1A74202D045F00305F2E7D04501D2F6
:10ACD000A74219D1BAF10B0F0ED0A74201D045F00F
:10ACE00003050BD84FEA896027464FF008084FF05C
:10ACF0000B0A4FEA1069DCE745F003050098806B0A
:10AD00000178E5293DD03EE0802E08D3304602F0A0
:10AD100025FA002102F0F4F9064645F00205FF2E5F
:10AD20000FD9AAF10100804503D345F00305D046B1
:10AD3000BFE70098310A826B02F8081008F1010899
:10AD400018E026B1314624A0FFF798FA18B15F2623
:10AD500045F003050EE0A6F14100192802D849F09C
:10AD6000020907E0A6F16100192803D8203E49F046
:10AD70000109B6B20098816B01F8086008F101087A
:10AD800097E705210170BAF1080F03D14FEA8960F6
:10AD90004FEA1069C9F38100032803D06FEA090163
:10ADA000890701D145F00205A90709D409F003017B
:10ADB000012901D145F01005012801D145F0080510
:10ADC0000098806BC572002059E70000222A3A3CA7
:10ADD0003E3F7C7F000000002B2C3B3D5B5D000074
:10ADE0002DE9F05F894606464022002103F091F8E4
:10ADF00085203070C02086F82000484605F0F9FE16
:10AE0000014606F1240004F04AFE402400254FF0DC
:10AE100001084746AA464FF0C10B06F804B0641C6F
:10AE200006F804A0641C27B139F815700FB16D1C29
:10AE3000EDB23019394604F032FEA41CE006F2D11E
:10AE400008F1010000F0FF0839F815000028E4D1EE
:10AE500086F8235086F80180BDE8F09F10B50446BF
:10AE60000420F8F7EBFC0148046010BD1800002036
:10AE700070B5054600244FF47A7603E0304600F0C2
:10AE800005F8641CAC42F9D370BD000070B54FF0FA
:10AE9000E02500216C69094AAB6912685043AA6930
:10AEA0009A42FCD002D2A3EB020302E0A4EB02061A
:10AEB0003344194413468142F1D370BD1800002079
:10AEC0002DE9F0410F4604460021066800F005FB1D
:10AED000E8B900253046216B04F04AFAB8B9317858
:10AEE0000429616B097803D0E52905D021B107E079
:10AEF00041F3C011491C03D06D1CBD420AD000E0D3
:10AF000000250121204600F0A5F80028E2D0042801
:10AF100000D10720BDE8F0812DE9F05F0446002153
:10AF2000D0F8009000F0D9FA00284BD199F8000031
:10AF300004280CD0FF254FF0FF382F46C4F83C8082
:10AF40004846216B04F014FA06004CD13CE0206C1A
:10AF500005F04FFE82462DE0D9F80C00243002F0B7
:10AF6000EFFD504526D1D9F80C0040254FF00008E0
:10AF700090F8236016E0E80600D1AD1CD9F80C006B
:10AF8000284402F0DDFD02F0E9F8216C074631F8B3
:10AF9000180002F0E3F8874207D1761EF6B208F1F6
:10AFA0000108AD1C002EE6D100E01EB9216C31F87D
:10AFB000180030B10021204600F0CEF85FEA000B07
:10AFC000CAD05846BDE8F09F616B087850B1CA7A84
:10AFD000E52802F03F02A27130D0130704D50F2AF2
:10AFE0002CD105E0042633E00F2A01D0C5B11CE0C6
:10AFF000226C32B3430605D54F7B20F04000A36A94
:10B000000546E363A84208D1487BB84205D1104603
:10B01000FFF762F908B16D1E00E0FF25EDB210E008
:10B02000084604F076FDB84212D0A16BC87AC0077A
:10B0300004D10B22606B02F057FF48B1FF25C4F822
:10B040003C800021204600F005F806003FF478AF70
:10B050003046B7E72DE9F04705460468806A89461F
:10B0600000F12008286B30B12178042906D04FF474
:10B070000011414505D80420BDE8F0874FF080510C
:10B08000F7E75FEAC8515ED1401C2863E96A0027F0
:10B0900029B16089401E10EA582F05D053E021895C
:10B0A000B1EB581F21D94EE0284602F085FB064639
:10B0B00001281ED9701C34D0A069B0423DD8B9F126
:10B0C000000F12D02846E96AFFF7F6FC06000ED002
:10B0D000012E0ED0701C24D0E87940F00400E871F5
:10B0E000204604F0B7FDE0B905E02F63C3E7072071
:10B0F000C2E70220C0E74FF40072002104F13400DF
:10B1000002F007FF002731462046FFF7D8F84FF03E
:10B11000010920630BE084F80390204604F09AFDB7
:10B1200008B10120A8E7206B401C7F1C20636089C8
:10B13000B842F0D8206BC01B206331462046EE6237
:10B14000FFF7BDF82863C8F3080020443430C5F881
:10B150002880686300208FE72DE9F0470426FF254B
:10B16000894604462F46D0F800805FE0404604F050
:10B17000FFF806005ED1616B0878A0B198F8002056
:10B18000042A12D0CA7AE52802F03F02A27108D040
:10B190002E2806D022F02003082B1CD000234B457C
:10B1A0001BD0FF2532E0042644E0B9F1000F02D0A5
:10B1B000832841D02AE0852828D1A06AE063204670
:10B1C00002F0DFFC060035D1D8F80C00007900F061
:10B1D0003F00A07130E00123E1E70F2A01D00DBB51
:10B1E0001BE0420605D54F7B20F04000A26A0546D1
:10B1F000E263A84208D1487BB84205D1206C04F034
:10B20000C3F908B16D1E00E0FF25EDB20021204614
:10B21000FFF720FF060009D00CE0084604F079FC97
:10B22000B84209D04FF0FF30E06305E0216B002900
:10B230009CD10EB1002020633046BDE8F0870000AD
:10B240002DE9F04F876B0446D0F80090D0F840808D
:10B25000F87A95B010F0A00F03D0062015B0BDE825
:10B26000F08F002500E06D1C38F815000028FAD199
:10B2700099F80000042817D00C22394612A802F0D1
:10B280003FFE9DF85300C0076AD00020F8720126E7
:10B2900020643346424612A9384602F047FA204657
:10B2A000FFF73AFEE8BB4FE00F200E35B5FBF0F597
:10B2B000AD1C29462046FFF703FE0028CED1694287
:10B2C0002022A06A02EB41110844E063E0794107C3
:10B2D00033D500F00300E071B9F80A00D4E9043175
:10B2E00042029A1841F10001C4E90421204601F00C
:10B2F00075FF0028B2D12146684602F026FC0028DE
:10B30000ACD1D4E90423D9F80C00383004F0A2FB06
:10B31000D4E90423D9F80C00283004F09BFBE07931
:10B3200000E014E040F00101D9F80C0080F8211091
:10B33000684604F0B8FB002890D14146D9F80C00CB
:10B34000FFF74EFD002089E7761C642EA1D3642E02
:10B3500010D0042882D19DF85300F872C4F84080C0
:10B360009DF85300800707D50D200C35B5FBF0F68E
:10B37000761C02E0072071E7012631462046FFF7E0
:10B380009FFD050075D1761E5FEA060B58D0A16AB5
:10B39000CBF1000001EB4011204600F09EF80500C3
:10B3A00067D1A06B04F0B5FB01904846216B03F018
:10B3B000DFFF05005DD1206C0090666B01980BF0FB
:10B3C000FF0A70730F20F07200203073014606F1FF
:10B3D0001A0004F064FBAAF1010000EB800101EB0C
:10B3E000C008002701E0854204D0009830F81850CA
:10B3F00008F1010820482946C05D304404F04FFBA5
:10B400000DB94FF6FF757F1C0D2F4FF6FF70EAD375
:10B41000854203D0009830F8180008B94AF0400A75
:10B4200086F800A0012089F8030000212046FFF7DC
:10B4300011FE05001DD1ABF101005FEA000BB4D194
:10B440004846216B03F094FF050012D12022002111
:10B45000606B02F05EFDD4E90D010B2202F050FD9D
:10B46000A06B616BC07A00F018000873012089F8A6
:10B4700003002846F2E60000A45301082DE9F0413C
:10B48000C16B0446866A0568481C02D0204600F05D
:10B4900024F800281AD1E5274FF001082846216B2F
:10B4A00003F066FF78B929780429616B10D00F701A
:10B4B00085F80380A16AB14208D200212046FFF737
:10B4C000C9FD0028EAD0042800D10220BDE8F0819F
:10B4D0000A7802F07F020A70EAE72DE9F041076876
:10B4E00006460D463878042806D04FF40010A842CE
:10B4F0003CD9E8063AD102E04FF08050F7E7B56258
:10B50000B46834B93878032807D30020BC6AF071D6
:10B510001CB178894FEA402812E03889B0EB551FFA
:10B5200024D9B86A12E0304602F046F90446401CBD
:10B530001AD0022C1AD3B869A04217D9A5EB080576
:10B5400045452146EFD23846FEF7B9FEC6E90B4025
:10B5500060B100EB55203063C5F308003844343047
:10B5600070630020BDE8F0810120FBE70220F9E7CD
:10B5700010B520B1012805D0022809D105E0FCF75B
:10B5800043FE04E0FDF7F4FC04E0F6F787F808B1A9
:10B59000012010BD002010BD30B54FF4007428B15B
:10B5A00001281CD0022827D0012030BD39B11F4806
:10B5B00001290BD0022904D003290ED103E0002079
:10B5C00030BD1460FBE7B0F8500020E0816CB0F8AB
:10B5D0004C00C30543EA512025E0042030BD00297A
:10B5E000EDD0012905D0022913D00329F5D1082077
:10B5F0000DE04FF4484016E00029E0D00C4D012941
:10B600006B8808D0022904D00329E6D1580A10809B
:10B61000D5E71480D3E7E889A97948435843C1178F
:10B6200000EBD15040121060C9E70000F005002087
:10B63000D81800202DE9F0411C0015460E4607D011
:10B6400048B14FF40072012811D0022821D11BE02B
:10B650000420BDE8F0811A4602E0FCF7D5FD224641
:10B6600029463046FCF7C2FF0028F6D113E0174602
:10B6700069023A463046FDF7B9FC641E05F1010542
:10B6800006F50076F4D106E029463046F6F784F850
:10B6900008B10120DDE70020DBE7002070472DE93D
:10B6A000F0411C0015460E4607D048B14FF4007219
:10B6B00001280ED002281ED118E00420BDE8F08138
:10B6C000E2B229463046FDF741F8B0B1FCF79CFDE7
:10B6D000F6E7174669023A463046FDF701FD641E5B
:10B6E00005F1010506F50076F4D106E0294630465D
:10B6F000F6F7EAF808B10120E0E70020DEE77CB5C4
:10B700000D4600211446009101AA694600F059F83F
:10B7100000280AD101998A694B89921E00995A43DF
:10B720004B4351082960590821607CBD70B5164D06
:10B7300000244FF40D763146002003F00FFF45F84A
:10B74000240018B1641CE4B2032CF4D34FF4147633
:10B750003146002003F002FF0C4D314628600020E6
:10B7600003F0FCFE68604FF40071002003F0F6FE69
:10B77000A860032C06D1296821B1696811B108B10C
:10B78000002070BD012070BD88C10220040300208C
:10B7900038B5044601F09CFA002807D169462046D6
:10B7A00005F0F2F9002801D10021216038BD38B53B
:10B7B0000446694605F0E8F9002801D1002121601E
:10B7C00038BD2DE9F7478DB014468A4600226946F8
:10B7D0000DA801F063FD5FEA00097AD100982060AE
:10B7E0000098D0E90516B21E914202D8CAF800109E
:10B7F0006FE001780024012904D004291AD0D0F880
:10B8000024803BE002250290294602A801F0D4FFE3
:10B81000411C03D0012803D028B105E0012000E03D
:10B82000022081464DE0641C00986D1C80698542B1
:10B83000EAD346E00025B61EC76A00E045B939469E
:10B840007F1C009803F094FD5FEA000939D1009A4B
:10B850000820511991F8341007E0CB0700D1641C7F
:10B860004908401EA6F1010601D0002EF5D16D1C3D
:10B87000C5F30805002EE1D123E065B9414608F182
:10B880000108009803F074FD5FEA000919D1009FD8
:10B890004FF400753437009800780228384604D0F9
:10B8A00002F018F9000107D007E002F049F900B9E9
:10B8B000641CAD1EBF1C02E0641C2D1F3F1D761EC4
:10B8C000DBD1CAF8004000984461017941F00101E0
:10B8D000017110B04846BDE8F0872DE9F74793B0F5
:10B8E00091460D46002212A913A801F0D7FC0600CC
:10B8F00064D1F5B31298B04600904146CDF8088067
:10B900006846FFF7EAFD060019D101216846FFF7F6
:10B9100023FC060013D112980078042813D00020CD
:10B9200002460D99095CA954401C521C0B2AF8D3FD
:10B930004046A8541AB1521EA95C2029F9D0042E01
:10B9400023D0B6B13AE0002427464FF0020A13E0B4
:10B950000D990AEB4700084402F0F2F8002101F0CB
:10B96000CFFB80B1FF2802D9010A2955641C285554
:10B9700000E00DE0641C7F1C0D984078B842E7D8C9
:10B9800005F80480DBE73F20F1E785F8008000261A
:10B99000B9F1000F12D01298016A03F0E9FC060019
:10B9A0000CD11299087803280ED004280AD0272039
:10B9B0000844343002F08EF8C9F8000016B0304662
:10B9C000BDE8F0876420F3E74320F1E72DE9FC416F
:10B9D00000259046074604464E1E0FE001AB0122AB
:10B9E0006946404600F0CEFE0198012808D19DF836
:10B9F00000006D1C04F8010B0A2801D0B542EDDBF4
:10BA00000020207015B13846BDE8FC810020FBE71E
:10BA10002DE9F04F87B017469946044602A905F074
:10BA2000B3F85FEA000A6FD194F82900B0F1000A78
:10BA3000F9D1D4F8488004F14C004FF0010B01908B
:10BA4000B8F1000F76D0F94371EA090135D0D4E995
:10BA50000410CB1B70EB090201D20F468146C4E9EA
:10BA60000C7957EA09004FD07F1E49F1FF331D467C
:10BA70003A462046FEF70AFC0146A0630298FEF70C
:10BA80001EFC00287ED002997A0A42EAC5524B89F0
:10BA90005B1E1A401518208EC005E4D0E26BAA4246
:10BAA000E1D094F82800400638D548780123019960
:10BAB000FFF7F5FD002866D12AE058F8049BA1683D
:10BAC0000226D1B10025B61C00910F4620466D1C00
:10BAD00001F072FE0146012854D9481C53D0781C4D
:10BAE0008142F2D04E4504D848F8045B009848F8EB
:10BAF000040B029880698842E4D8A06C4E45066029
:10BB000003D80020C8F80000DEE04FF0110ADBE0A7
:10BB100094F8280020F0400084F8280002980123BF
:10BB20002A4640780199FFF785FD00282BD1E5636F
:10BB3000CAE0FFE7D4E90410CB1B70EB090205D281
:10BB400094F82820920701D40F468146D4E90C01CD
:10BB5000CDE9040100200090C4E90C0057EA090077
:10BB60005FD0029840894FEA4028DDE9040108438C
:10BB700025D0781E49F1FF3142460023F4F73AFB05
:10BB8000054601E078E08CE00E46DDE90401401E48
:10BB900041F1FF31424600230490F4F72BFB281AB1
:10BBA0008E410CD3A8F10101CA4304980021104032
:10BBB0003F1AC4E90C0169EB0109A16B0CE0A16813
:10BBC00049B900212046FEF777FF0146012854D0ED
:10BBD000481C66D0A160A16319B30026B8EB07002A
:10BBE000354676EB09000AD294F8280080072046F3
:10BBF0002AD5FEF761FF010029D14746B146D4E9B5
:10BC00000C32DB1942EB0902C4E90C32F80508D00A
:10BC10000298FEF754FB78B3790A41EAC951084407
:10BC20000090208EC00542D0E26B009882423ED048
:10BC300094F8280040062CD50298012301994078F9
:10BC4000FFF72DFD68BB1EE001F0B6FD0146481C64
:10BC500027D0012911D90298806988420DD9A163A2
:10BC6000D4E90C3013EB08026841C4E90C20B7EBAF
:10BC7000080769EB0509B1E7FFE7022084F829000E
:10BC800007B0BDE8F08F94F8280020F0400084F859
:10BC900028000298DDE9002140780123FFF7CAFC63
:10BCA00018B184F829B00120EAE70098E063D4E9EC
:10BCB0000C01D4E90423121A8B4105D2E4E90401F2
:10BCC000207E40F0200020765046D9E72DE9F14F44
:10BCD0009AB0022201A91AA801F0E0FA0400019822
:10BCE00004907CD14FF48C6001F030FA5FEA0009D7
:10BCF00010D016A804991290CDF8509009F5007054
:10BD0000C86004A81A9901F071FC040006D0042C44
:10BD100006D088E011201BB0BDE8F08F082482E037
:10BD2000002104A8FEF7C8FE5FEA000801984FF062
:10BD30000002144641894FEA4121CDE9081203D09F
:10BD4000B8F1010F02D002E0072400E00224B8F1AC
:10BD5000FF3F01D014B104E0012402E003F07AFFB8
:10BD6000044601F0BCFD0090D4BB41460198FEF7AB
:10BD7000A6FA019E074634364FF400720021304681
:10BD800002F0C7F801984FF0100A007804282AD072
:10BD90000B222021304602F0BCF82E25357086F8A3
:10BDA0000BA006F11600009903F04CFE4246314606
:10BDB000019803F033FE06F12000202231460446AC
:10BDC00002F09EF886F821500198069A017803291E
:10BDD00003D1816A914200D10022214601E025E091
:10BDE0001CE003F01BFE01984FF0010B458985B163
:10BDF0000198076380F803B07F1C03F02BFF040059
:10BE00000CD14FF400720021304602F082F86D1E12
:10BE1000EED104A8FFF714FA040009D0002241462D
:10BE200004A803F083FC484601F094F9204672E729
:10BE300001980178042914D0119C009904F116008E
:10BE400003F000FE42462146019803F0E7FD84F826
:10BE50000BA0019981F803B0019803F0B7FE0446E6
:10BE6000E1E7C06800990C3003F0ECFD0198414611
:10BE7000C068343003F0E6FD01980899C068383096
:10BE800003F0E0FD01980899C068283003F0DAFD5E
:10BE900001980321C26882F82110C06880F804A0CC
:10BEA00004A803F000FED7E72DE9F74F88B0174646
:10BEB0000998012803D913200BB0BDE8F08F08A81A
:10BEC00001F092FD002801DA0B20F5E7FD4951F859
:10BED00020504DB100212970C0B20190FFF748FBFE
:10BEE000C10703D00320E7E70C20E5E7400701D5B1
:10BEF0000A20E1E703AA01210198FFF74DFB002882
:10BF00007DD1039880287AD3099909B1002100E0F6
:10BF10003F218946A0EB0901781E0742039100D119
:10BF20007FB94FF4FA60B1FBF0F20020E64B00E07D
:10BF3000401C33F810409442FAD8E34A163232F8E3
:10BF40001070B7F5007F00D37F0A87B1802F00D92A
:10BF50008027B1FBF7F0012640F6F672904200D33D
:10BF600002264FF6F672904203D3032621E0012702
:10BF7000EFE7032E1DD0012E25D04000001D00F25A
:10BF8000FF104FEA50284FF0010A2020834609EBAA
:10BF90000A000490404400EB0B04E219A2EB0900F4
:10BFA000884247D802AA03210198FFF7F5FAA8B9F9
:10BFB0000FE040F2072202EB80004FEA50284FF0DA
:10BFC000200A0020E2E700EB4000401C4008C01CB3
:10BFD000D5E7029810B1B0F5004F01D901200290C9
:10BFE0002118401E491E8143081B0290032E13D0C6
:10BFF00080440398A0EB0A02A2EB080200E0D8E01C
:10C00000A2EB0B01B1FBF7F10591022E09D0032E33
:10C010000CD0012E12D016E00499824408440490FA
:10C02000E7E740F6F672914204D30CE04FF6F67063
:10C03000814201D20E203FE70C200AE0B0F5803F9C
:10C0400006D2012005E0B0F5803F01D2042000E0D7
:10C0500006200690099808B1F02038E005F1340078
:10C060004FF400720021009001F053FF05F5F974C0
:10C0700001206070A0700020E07006982071FE2002
:10C080006071039909EB010043F6C161B0FBF1F067
:10C090003F2141EA90010290A171E0713F2104F13A
:10C0A000080003F0CFFC04F10C00039903F0CAFC74
:10C0B0004AF6552105F2322003F0F1FCDDE90010CB
:10C0C00001230022FFF7EBFA002872D1F82005F1D6
:10C0D00034044FF4007500902A460021204601F0F8
:10C0E00018FF0B2279A1204601F00AFF294604F12E
:10C0F0000B0003F0D4FC67731FFA8AF104F10E0001
:10C1000003F0CDFC01202074032E0ED0410204F177
:10C11000110003F0C4FC0399B1F5803F07D289B246
:10C1200004F1130003F0BBFC05E00021EFE704F18C
:10C13000200003F087FC009860753F2104F118008F
:10C1400003F0ADFCFF2104F11A0003F0A8FC4946FE
:10C1500004F11C0003F076FC01F0C1FB80250146D0
:10C160004FF0290A0290032E24D004F1270003F097
:10C1700069FC1FFA88F104F1160003F090FC84F8C2
:10C18000245084F826A0132253A104F12B0001F0BF
:10C19000B7FE04F5FF704AF65521069003F07FFCC8
:10C1A00001234A4621460198FFF779FA002800D179
:10C1B00021E085E004F1430003F044FC414604F132
:10C1C000240003F03FFC022104F12C0003F03AFCB0
:10C1D000012104F1300003F062FC062104F1320079
:10C1E00003F05DFC84F8405084F842A013223FA184
:10C1F00004F14700CBE7032E06D1012309F1060223
:10C2000021460198FFF74BFA049D4FF0000A4FF4C6
:10C2100000720021204601F07CFE00980290032E5F
:10C2200013D0012E0FD06FF0FF0101432046029181
:10C2300003F008FC2A466D1C012321460198FFF7F4
:10C240002EFAE8BB11E02E49EFE760F0FF0120462F
:10C25000029103F0F7FB4FF0FF31201D03F0F2FBDA
:10C260006FF0704104F10800E2E74FF40072002122
:10C27000204601F04EFE012009E02A466D1C0123F4
:10C2800021460198FFF70BFAD0B90298401C0290A2
:10C290004045F2D30AF101005FEA000AB7D0032E4D
:10C2A00000D05F462A466D1C012321460198FFF706
:10C2B000F6F928B97F1EF5D1032E4BD1114923E0A1
:10C2C00050E000007CC10220C2530108EBFE904DFB
:10C2D00053444F53352E30004E4F204E414D452094
:10C2E0002020204641542020202020004E4F204E68
:10C2F000414D45202020204641543332202020004B
:10C3000000FFFF0052526141204603F09BFB16499B
:10C3100004F5F27003F096FB059904F5F470491EDC
:10C3200003F090FB022104F5F67003F08BFB4AF654
:10C330005521069803F0B3FB012309F101022146C0
:10C340000198FFF7ACF9012309F107022146019892
:10C35000FFF7A5F9002211460198FFF71DF9002803
:10C360003FF4B3AD0120A7E57272416117B581B00A
:10C37000144602980090684601F036FB002802DA65
:10C380000B2004B010BD0B4B002253F8201001B15C
:10C390000A700199002900D00A7043F8201001D0DA
:10C3A000012C01D00020ECE7002201A902A800F036
:10C3B00075FFE6E77CC102202DE9F74F98B0040035
:10C3C0000DD04FF0000802F01F06324601A919A84F
:10C3D000C4F8008000F062FF050004D006E10920E7
:10C3E0001BB0BDE8F08F019802904FF48C6000F014
:10C3F000ADFE07000DD014A802991090129707F512
:10C400000070C86002A8199901F0F0F8050002D088
:10C4100006E01120E4E71098C07A000600D5062552
:10C4200016F01C0F7ED04DB1042D03D102A8FEF7EB
:10C4300007FF054646F008064DB1D4E09DF80E0012
:10C4400010F0110F6FD1700701D50825CBE0300730
:10C450006AD501F044FA814601984FF0200A4FF066
:10C46000010B017804292AD00F9849460E3003F0B9
:10C47000E9FA0F984946163003F0E4FA0F9981F86B
:10C480000BA00F99019801F012FB814600220F9931
:10C49000019803F0C3FA0F9800211C3003F0D2FA80
:10C4A0000198B9F1000180F803B078D0D0F830A03D
:10C4B000002202A803F03AF9050055D093E020606D
:10C4C0000198C068343001F005FBA0600198C06895
:10C4D000383001F00AFBC4E904010198C16891F801
:10C4E000211001F00201E171C0684946083003F0F3
:10C4F000A9FA01984546C16881F81480C068494688
:10C500000C3003F09FFA0198C1684D75C268002194
:10C5100082F804A0C068343003F094FA0198002235
:10C52000C06802E02BE036E03BE01346383003F011
:10C5300091FA019800221346C068283003F08AFA65
:10C54000019902A8C96881F821B003F0ACFA05008E
:10C5500049D1A168D1B10022204603F0E7F8054691
:10C56000A0680199401E07E05146019802F000FFC3
:10C5700005460199A9F10100086175B133E095BB49
:10C580009DF80E00C10602D504252CE007E0B10796
:10C5900003D5C00701D0072525E0300701D546F0B7
:10C5A00020060198016B21640F99616401780429C8
:10C5B0001ED00F9901F07BFAA0600F981C3001F09B
:10C5C00089FAC4E90408C4F8488084F82980002165
:10C5D000C4F83C80C4E90C1184F8286001982060FC
:10C5E0000198C088A080384600F0B4FD2846F7E6E0
:10C5F000C068343001F06EFAA0600198C06838302D
:10C6000001F073FAC4E904010198C06890F82100B0
:10C6100000F00200E0710498E06106989DF80F10A8
:10C6200020F0FF000843206211986062CBE773B5E9
:10C6300084B0040007D00022694605A800F02EFE51
:10C64000050003D055E0092006B070BD00994FF4F5
:10C650008C60216000F07AFD06000DD001A92664EF
:10C66000A163216806F50070C8602046059900F0B6
:10C67000BDFF050002D036E01120E5E7A06BC07ACF
:10C68000000628D4A079C00637D50098017804297F
:10C6900004D0616B01F00BFAA0601CE0A268E261BB
:10C6A0002169E27921F0FF0111432162E26B6262AC
:10C6B000C068343001F00EFAA0600098C0683830CD
:10C6C00001F013FAC4E904010098C06890F8210051
:10C6D00000F00201E1710098C188A180204600218C
:10C6E000FEF7FBFE0546304600F034FD042D06D073
:10C6F0000DB1002020602846A6E70525F3E70525B3
:10C70000F7E700B595B0029100210391049101462D
:10C7100002A802F0ECFF039800280DDB024601ABF3
:10C7200005A9029800F002FC30B9019903988842EB
:10C7300002D1049815B000BD4FF0FF30FAE710B5F4
:10C7400096B004460020CDE90210049003E002A850
:10C75000641C02F0CCFF21780029F8D1039800284E
:10C760000DDB024601AB05A9029800F0DFFB30B9F2
:10C7700001990398884202D1049816B010BD4FF079
:10C78000FF30FAE72DE9FC5F894600259A461646F8
:10C79000044669461D6004F0F7F900281AD194F8A0
:10C7A0002900002816D194F82800C00711D0D4E938
:10C7B0000C02D4E90431181A04F14C0361EB0201B4
:10C7C0000193831B4FF0010B71F1000100D206466B
:10C7D0008EE00720BDE8FC9F208EC0056CD1D4E917
:10C7E0000C230098550A45EAC3554089401E054070
:10C7F00013D152EA030005D0A06C28B12046FDF702
:10C8000045FD05E0A06803E02046A16B00F0D4FFE1
:10C81000022819D3411C49D0A063A16B0098FDF7F1
:10C820004EFD88B100EB0508770A23D00098EA197D
:10C8300041898A4200D94F1B40783B4642464946CF
:10C84000FEF7F8FE90BB03E0022084F82900C1E760
:10C8500094F8280040060BD5E16BA1EB0800B84224
:10C8600006D209EB40204FF40072019901F048FB19
:10C870007D022FE0E26B42451CD094F82800400670
:10C880000CD50098012301994078FEF708FF68B99C
:10C8900094F8280020F0400084F828000098012334
:10C8A000424640780199FEF7C5FE18B184F829B0D8
:10C8B00001208FE7C4F83C80208EC0F30800C0F54B
:10C8C0000075B54200D9354601192A4648464C3113
:10C8D00001F016FBD4E90C20521940F10000C4E924
:10C8E0000C20DAF80000A9444119761BCAF80010A0
:10C8F000002E7FF471AF00206CE72DE9FF410F4659
:10C90000064603A904F040F904002FD1AFB14FF45B
:10C910008C6000F01BFC050015D0C6F838D03564DB
:10C92000316805F50070C86000213046FEF714FC40
:10C93000044604280BD054B115E000213046FEF720
:10C94000CCFD044612E0112004B0BDE8F081394668
:10C95000304600F0C6FF00213046FEF77BFB044660
:10C96000042800D10024284600F0F4FB2046EBE721
:10C97000F3B5B9B03AA801F037F80222694639A8F0
:10C9800000F08CFC040072D1009814904FF48C607D
:10C9900000F0DCFB05000DD036A8149922902495F8
:10C9A00005F50070C86014A8399900F01FFE040056
:10C9B00003D09FE011203BB0F0BD2298C07A10F068
:10C9C000A00F01D0062495E000980178042913D027
:10C9D0002199152226A80B3101F092FA482214A9B8
:10C9E00002A801F08DFA02A83A9900F0FFFD0400B8
:10C9F00015D0042C3CD038E0C168402226A801F0B4
:10CA00007FFA482214A902A801F07AFA02A83A99FA
:10CA100000F0ECFD040002D0042C02D025E0082434
:10CA200068E002A8FEF70CFC040063D10098C0681F
:10CA3000467890F82340243001F082F807460098A9
:10CA4000402226A9C06801F05BFA0098C0684670D1
:10CA50000098C16881F82340C0683946243003F04B
:10CA60001EF802A803F01FF804467CB342E044E03D
:10CA700002A8FEF7E5FB04003CD10F9C13220DF148
:10CA80009A0104F10D0001F03BFA9DF8980001268F
:10CA900040F02000E0720098C670E17AC90620D507
:10CAA000049A169991421CD0214601F000F80146E3
:10CAB0000098FDF704FC010009D0009802F058FC32
:10CAC0000400009800F1540103D013E009E00224AF
:10CAD00010E04A782E2A04D1049A02F09FFF0098B1
:10CAE000C67014A8FEF7CAFC040003D1009803F036
:10CAF0006DF80446284600F02DFB20465BE7000059
:10CB00002DE9F1439AB0022218A91AA800F0C6FB39
:10CB1000002875D1189A002400921A9800E0641C2D
:10CB2000015D2029FBD211784FF000090DF1480872
:10CB3000042930D100252E4628E01A99485D6D1C45
:10CB4000A0F181027D2A0ED8A5420BD2495DA1F148
:10CB500040023E2A02D9403A7E2A03D841EA002008
:10CB60006D1C00E00020012100F0CAFA07007DD012
:10CB700001465648FDF782FB002877D1162E75D066
:10CB800008EB0600394602F08AFFB61CA542D4D352
:10CB9000344650E0641EA4B3011911F8011C202989
:10CBA000F8D000258DF848902E461A99885D761C9D
:10CBB000A0F181027D2A10D80A2D0DD2A6420BD2F7
:10CBC000895DA1F140023E2A02D9403A7E2A03D86B
:10CBD00041EA0020761C00E00020012100F090FADC
:10CBE00000F0BCFA002100F08BFA07004BD00146A0
:10CBF0003648FDF743FBC8BBFF2F03D90A2002E0EC
:10CC000042E018E00B20A8423DD9FF2F03D9390A92
:10CC100008F805106D1C404608F805706D1CA6420A
:10CC2000C3D320210B2D02D241556D1CFAE79DF88C
:10CC30004800E52827D000216846CDF80890FEF787
:10CC40004CFC002820D101216846FEF785FA012519
:10CC5000E8B1042818D10020002C15D00121684625
:10CC6000FEF72EF900280FD1202200E00BE0002172
:10CC70000D9801F04EF918980078042822D00D99EB
:10CC80000820C87208E006201BB0BDE8F0831898A1
:10CC90000078042804D06CB10B2212A90D9806E08C
:10CCA0000D996008224648700D9812A9801C01F069
:10CCB00027F902E00D99E52008701898C57002F078
:10CCC00085FFE1E70D9983200870E9E7B15301087A
:10CCD000F0B593B0044612A903F056FF050023D126
:10CCE00094F8280081061FD5400611D51298E26BF2
:10CCF0000123407804F14C01FEF7D1FC10B1012072
:10CD000013B0F0BD94F8280020F0400084F828000B
:10CD100000F0E5FD064612980178042905D0216C43
:10CD200002F026FB050055D079E0204600F056FAC7
:10CD3000050074D14FF4187000F008FA070008D00D
:10CD400012982146C760684600F0FFFE050002D039
:10CD50003CE01120D4E71298C1680A7942F0200221
:10CD60000A71E179C26841F0010182F82110C068BE
:10CD7000A168343002F066FED4E904231298C0683A
:10CD8000383002F067FED4E904231298C0682830D6
:10CD900002F060FE12983146C0680C3002F052FE7C
:10CDA00012980021C2685175C068103002F04AFE26
:10CDB000684602F078FE050008D1129802F006FFDE
:10CDC000054614F8280F20F020002070384600F0A7
:10CDD000C1F924E0656C2946E87A40F02000E87249
:10CDE000A268206802F01AFE05F11C00216902F019
:10CDF00029FE314605F1160002F024FE002105F15E
:10CE0000120002F04CFE12980121C17002F0DEFE09
:10CE1000054694F8280020F0200084F828002846D1
:10CE20006EE771B5B3B002222EA933A800F036FA2E
:10CE300004002E98009077D14FF48C6000F086F9B2
:10CE400005000DD02FA800990E90109505F50070E3
:10CE5000C8606846339900F0C9FB040003D060E065
:10CE6000112034B070BD0E98C07A000601D506249A
:10CE700057E09DF80600C00701D0072451E02E9826
:10CE80002490017804290ED00D9900F010FE06467A
:10CE90009DF80600C00633D52E981496129000789F
:10CEA000042816D01DE0C068343000F013FE06469A
:10CEB00026902E98C068383000F017FECDE9280182
:10CEC0002E98C06890F8210000F002008DF89700BD
:10CED000DEE7DDE92801CDE916019DF897008DF820
:10CEE0004F00002112A8FEF7F8FA040019D1002122
:10CEF00012A8FEF731F90400BFD0042C00D084B989
:10CF00006846FEF7BBFA04000BD136B10022314669
:10CF100024A802F00BFC040003D12E9802F056FE68
:10CF20000446284600F016F920469AE72DE9FC5FF2
:10CF300089464FF0000B9A46164604466946C3F8E8
:10CF400000B003F021FE002808D194F82900002841
:10CF500004D194F82800800702D40720BDE8FC9F84
:10CF60000098017804F14C000190042907D1D4E91C
:10CF70000C108A1940EB0B03511A834102D3206B2A
:10CF8000811901D3206BC643B0E0208EC0057FD14C
:10CF9000D4E90C230098550A45EAC3554089401E40
:10CFA00005401AD152EA030005D0A06C38B12046E2
:10CFB000FDF76CF907E0A06838B9002100E0A16B2B
:10CFC0002046FDF779FD00287DD001282ED0411C98
:10CFD00057D0A063A16801B9A06094F8280040066A
:10CFE0000DD50098E26B012340780199FEF757FBBD
:10CFF000A0BB94F8280020F0400084F82800A16B22
:10D000000098FDF75CF988B100EB0508770A26D097
:10D010000099EA194889824200D9471B48783B4663
:10D0200042464946FEF73BFBC0B903E0022084F8C4
:10D03000290093E7E16BA1EB0800B8420CD209EBA1
:10D0400040214FF40072019800F05AFF94F8280034
:10D0500020F0400084F828007D022DE011E0E16B13
:10D06000414513D0D4E90413D4E90C20511A984156
:10D070000CD200980123424640780199FEF7DAFA73
:10D0800020B1012084F8290068E701E0C4F83C8061
:10D09000208EC0F30800C0F50075B54200D93546B2
:10D0A00020442A4649464C3000F02AFF94F82800D4
:10D0B00040F0400084F82800D4E90C134A19A94430
:10D0C00043EB0B0300E014E0C4E90C23D4E90410A3
:10D0D0008F1A70EB030701D211461846C4E90410F9
:10D0E000DAF800004119761BCAF80010002E7FF410
:10D0F0004CAF14F8280F40F02000207000202DE7DE
:10D1000070B580281BD345F2205409B10D4D00E0C5
:10D110000D4D00231022E11A01EBD17103EB6101E7
:10D1200035F82160864206D001D20B4600E00C465D
:10D13000521EF0D104E01AB105EB8100408870BDA9
:10D14000002070BD72A80208EE53010801460020BD
:10D1500002F004BA0146002002F0F4B930B5B0F58F
:10D16000805F01D21B4900E01B4931F8022B002AE5
:10D1700015D0904213D331F8023B1C0ADDB252FAAB
:10D1800083F3834221D9092C09D2DFE804F0050991
:10D190000E11131517191B00801A31F8100030BD3D
:10D1A000811A01F00101401A00E0103880B230BD50
:10D1B0002038FBE73038F9E71A38F7E70830F5E7A9
:10D1C0005038F3E7A0F5E350F0E7002CCDD101EBA8
:10D1D0004501CAE7F6FC0308E8FE030870B50646F9
:10D1E000C07903280FD1B569B46808E0621C2146F4
:10D1F000306802F001FA002806D1641C6D1E002D73
:10D20000F4D10020F071002070BD2DE9F0470646F2
:10D2100080698F1E801E9246B84200D800273C4687
:10D22000B8460025F06A00EB1431304602F0A0F851
:10D2300018B14FF0FF30BDE8F08704F0070201207D
:10D240009040B269C4F3C801C0B24FF480534FF4A8
:10D250000079921E06EB010C641C9CF834C00CEAA9
:10D26000000C4006000E944202D3002420461946CA
:10D27000BCF1000F05D0A0460025BC4207D100201C
:10D28000D9E76D1C5545F8D108F10200D3E7002815
:10D29000E0D10120491C4945DCD3C3E72DE9FF5FFC
:10D2A000002790460E460F6000F09EFB050003D558
:10D2B0000B2004B0BDE8F09FC84850F825409CB151
:10D2C0003460207828F0010620B16078FEF7E5F997
:10D2D000C1070BD02770E8B2B8466070FEF748F976
:10D2E000C10708D00320E4E70C20E2E70EB14007B5
:10D2F00004D40020DDE71EB1400701D50A20D8E79D
:10D30000002529462046FCF77FFF022820D16E46E3
:10D3100004EB051090F8F61100F5F97019B108301A
:10D3200000F0D8FB00E0002046F825006D1C042D1D
:10D33000EED3002756F8275025B129462046FCF7A2
:10D3400063FF00E00320022802D37F1C042FF1D3E7
:10D35000042879D0022879D24FF0FF3A4FF40076B2
:10D3600001280CD004F13F0000F0EAFBB0426DD17F
:10D3700004F14A0000F0E4FB002868D083E00B20B1
:10D3800002E0401C402806D2211891F834100029F0
:10D39000F7D040285AD304F19C0000F0D1FBB0F53F
:10D3A000807F53D194F8A000012707FA00F0B3461C
:10D3B00058454BD104F17C0000F097FBC14610EBBF
:10D3C000050841EB0906012E40D204F1880000F067
:10D3D00081FBE06194F8A200A070012836D194F896
:10D3E000A10087403804000C60812FD004F1900028
:10D3F00000F070FB0746801CA061B0F1004F25D201
:10D4000004F18C00256200F065FB2844E06204F121
:10D41000840000F05FFB284460626189E06A07FBDA
:10D420000101B8EB010176EB09060FD304F194007A
:10D4300000F050FB0146A0622046FCF740FF014689
:10D44000204601F095FF18B1012032E766E016E0B2
:10D4500000255E46601990F83410812904D14830C7
:10D4600000F038FB022802D02035B542F2D3B54295
:10D4700063D0C4F814A00426C4F810A0A7E004F1F7
:10D48000580000F027FBE06194F84470A770012F6A
:10D4900001D0022F51D1474394F841006081E8B395
:10D4A000411E084249D104F1450000F049FB2081AA
:10D4B000000742D104F1470000F042FB060004D10E
:10D4C00004F1540000F006FB064604F1420000F0AF
:10D4D00037FB010031D02389C81900EB13129642A3
:10D4E0002BD3B01A6689B0FBF6F0B8B1012640F62E
:10D4F000F67C604500D302264FF6F67C604500D3EB
:10D500000326801C2A44E2622944A061C4E9085130
:10D51000032E14D013B13944A16200E00DE0022EB5
:10D520001ED000F0010100EB400001EB5000E1696A
:10D5300000F2FF10B1EB502F14D20D20B9E604F128
:10D540005E0000F0FDFA0028F7D120890028F4D110
:10D5500004F1600000F0BEFAA062A0698000E6E776
:10D560004000E4E7C4F814A08020C4F810A02071A3
:10D57000032E2CD104F1640000F0E2FA012826D138
:10D58000691C204601F0F4FE08BB84F8048004F214
:10D59000322000F0D5FAA0F52A41553917D104F10F
:10D5A000340000F097FA0E49884210D104F5067055
:10D5B00000F090FA0B49884209D104F5077000F099
:10D5C00089FA606104F5087000F084FA2061064968
:10D5D00026700888401C0880E0808AE67CC1022012
:10D5E00052526141727241610003002073B50446DA
:10D5F0000568019801E0401C019001782F29FAD0BC
:10D600005C29F8D00021A16001980078202807D279
:10D61000A16B8020C87200212046FDF75EFF7CBD13
:10D6200001A92046FDF7D0FA0028F8D12046FDF7E1
:10D6300073FCA16BC97A28B10428F0D14907EED454
:10D6400005207CBD4907FCD4A079C006F8D5287810
:10D65000042809D0208DC0F3080041192846343130
:10D6600000F025FAA060DBE7A168E1612069E179BB
:10D6700020F0FF0008432062E16B6162E86834300B
:10D6800000F028FAA060E86890F8210000F002019C
:10D69000E171E868383000F028FAC4E90401BFE716
:10D6A00003490A685206FCD5C2B24A6070470000BE
:10D6B0000010014010B5002821D0114B0022001F9E
:10D6C000196803E0814203D80A4649680029F9D164
:10D6D00052B11368841A9C4204D100681844106047
:10D6E000104602E0506000E0186039B102680B1A81
:10D6F000934203D10B681A4402604968416010BD2F
:10D700001C03002070B50E460546002405E055F8C0
:10D710002410012001F016FF641CB442F7DB2946F7
:10D72000BDE87040012001F00DBF00007CB5164639
:10D730001C4605460B2200F0E3FB052C11D91D4ABF
:10D740000CE00021B61C2346044663F35F04400846
:10D75000E30300D55440491C1029F4D33088002835
:10D76000EFD107226B4604F00F003030392800D982
:10D77000C01D9854521E2409F5D17E2000219854D2
:10D78000541E06E081387D2802D8A14206D0491CEB
:10D79000491C914202D2685C2028F3D1082A02D2A7
:10D7A000985C521C00E020206854491C0829F5D3DD
:10D7B0007CBD0000211001002DE9F04104680D46F8
:10D7C000022972D3A169A9426FD921784FF0FF369F
:10D7D000012909D002292CD0F20D02EA850703297C
:10D7E00036D0042977D141E0606A05EB550700EB9C
:10D7F0005721204601F0BCFD00286DD1C7F3080079
:10D8000020447F1C90F83480606A00EB572120464A
:10D8100001F0AEFD48BBC7F30800204490F8341077
:10D8200048EA0120E90701D0060955E0C0F30B06DC
:10D8300052E0606A00EB1521204601F099FDA0B985
:10D84000E8B204EB4000343000F07AF9064643E0D9
:10D85000606A00EBD511204601F08AFD28B938191D
:10D86000343000F037F920F0704635E0D0E9041389
:10D8700051EA03022FD08268AA1A491E43F1FF33EE
:10D88000490A41EAC3516389B1FBF3F3C179022923
:10D890000CD0032913D002291DD0606A00EBD511EA
:10D8A000204601F065FDB8B90EE014E09A4212D8A6
:10D8B00002D16FF000460FE005F101060CE080692F
:10D8C0009042EAD96E1C07E03819343000F002F9B2
:10D8D00020F0004600E001263046BDE8F08100203F
:10D8E00070472DE9F0474FF00009064681F81A907D
:10D8F000006B0C46002875D030680178042905D0EB
:10D90000F06B401C20D00025376C16E0C068214623
:10D91000BDE8F04700F086B80021FFF7F1FB38B111
:10D92000FF2803D9010A62196D1C9176FF2D01D3DE
:10D93000002506E061196D1C887637F8020B002877
:10D94000EAD1611981F81A900021A37E0A464FF0AE
:10D950002E0C706B805C521C202822D0052800D130
:10D96000E520092A07D113B9651885F81AC065188A
:10D97000491C85F80DC0651868738BB9A0F1410783
:10D98000192F0CD8776B092A97F80C8001D3102730
:10D9900000E0082718EA070F01D02030C0B2A876AF
:10D9A000491C0B2AD5D333B9621882F81A90706BD0
:10D9B000007B00B9002160184D4680F80D90706B17
:10D9C000C07A2073706B1C3000F084F8C4E9000545
:10D9D000706B183000F0B4F82081706B163000F0D6
:10D9E000AFF86081BDE8F08710B503464FF0FF3017
:10D9F0001C68002C13D0214600E0491C0A78202A1C
:10DA00000ED33A2AF9D114F8012B303A0A2A06D259
:10DA10008C4204D1032A02D2491C1046196010BD61
:10DA2000002010BD2DE9F041402700260C46054698
:10DA3000B04617E0F80600D1BF1CE81900F080F8E6
:10DA40000021FFF75DFB90B1FF2803D9010AA2195D
:10DA5000761C9176FF2E0AD2A119761C887608F1E1
:10DA60000108BF1C95F823104145E3D816B93F20A3
:10DA7000A0760126A119002088766073287920738A
:10DA8000C00602D50020014603E005F1380000F091
:10DA90002CF8C4E9000105F10C0000F051F8608198
:10DAA00005F10E0000F04CF82081BDE8F08170B562
:10DAB00006460D4601F11A0000F042F8044630789F
:10DAC000032805D105F1140000F03AF844EA0044B7
:10DAD000204670BDC178827842EA01214278007800
:10DAE00042EA012140EA0120704710B5C1798279EC
:10DAF0000B0E42EA01211A02437942EA116243EA1B
:10DB000001211302027943EA116342EA01211A0258
:10DB1000C37842EA116243EA0121130243EA116326
:10DB200082781B0242EA012143EA11630A0241782A
:10DB300000780A43190241EA126140EA022010BD4E
:10DB40004178007840EA0120704710B50446086823
:10DB50002060C869A06091F82000E071086A002286
:10DB600020F0FF00C4E90402496A2046E163FDF7A2
:10DB7000B4FC002804D12046BDE8104000F001B8F4
:10DB800010BD2DE9F04104460068216BC66801F024
:10DB9000EFFB002822D1616B0878852842D1202232
:10DBA000304600F0ADF97778002120467F1CFDF764
:10DBB00051FA002812D1216B206801F0D9FB00280E
:10DBC0000CD1616B0878C0282CD1202206F12000EE
:10DBD00000F096F9F81E112802D30420BDE8F08168
:10DBE00040257F0100212046FDF734FA0028F5D1B9
:10DBF000216B206801F0BCFB0028EFD1616B087835
:10DC0000C1280FD17019202200F07AF92035BD42C9
:10DC1000E8D3304602F0D3FF0446B01CFFF790FF74
:10DC2000844201D00220D9E70020D7E71FB5F4F7DE
:10DC300035F80823022219214FF4B470FAF766FE72
:10DC4000B420FDF70BF94FF4165002F02DF8F8F759
:10DC50008FFFF6F781F8FAF79FF8F6F713FA01202D
:10DC600001F0CCFB00F0F2FD42F2273141F28730A7
:10DC7000FAF7C0FE584841685A208847574F4FF47A
:10DC800078401024386056A0CDE900402346C822D1
:10DC900032211E20F8F717FF564E4FF4FA751DE09B
:10DCA00055A0CDE900401023C82296211E20F8F788
:10DCB0000AFF2846FDF7DCF853A0CDE90040102309
:10DCC000C82296211E20F8F7FEFE2846FDF7D0F860
:10DCD000D6F8840208B30020C6F88402FAF794FA52
:10DCE0000028DDD1F3F7DAFCFDF720FD4A480122D8
:10DCF0004AA10068FEF73AFB4FF40071012001F0E1
:10DD00002DFC47494FF6FF75A6230860F0229621A7
:10DD10001E200095F6F786F91EE00120DCE741A001
:10DD2000CDE900401023C82296211E20F8F7CBFE33
:10DD3000C820FDF79DF8A623F02296211E2000950D
:10DD4000F6F770F9C820FDF793F8D6F8840200289A
:10DD500040D00020C6F8840203AA02A92FA0FDF734
:10DD6000CEFC0028DBD11F20386034A0CDE9004074
:10DD70001023C82296211E20F8F7A5FE32A0CDE977
:10DD800000401023C822AA211E20F8F79CFE34A0D0
:10DD9000CDE900401023C822BE211E20F8F793FED3
:10DDA00002980094820A0523AA218E20F8F750FEDB
:10DDB00003980094820A0523BE218E20F8F748FEBE
:10DDC0002DA000F0A9FE42F21070FDF751F8FCF70B
:10DDD000C5FAFEE70120BDE70C0200202400002068
:10DDE00041706F6C6C6F2053544D333246342F4664
:10DDF0003700000000804042534420436172642099
:10DE00004572726F72210000506C6561736520432A
:10DE10006865636B2120000088C10220303A000051
:10DE20000C030020534420436172642046617466F1
:10DE300073204572726F7221000000004641544603
:10DE400053204F4B21000000534420546F74616CE9
:10DE50002053697A653A20202020204D420000009E
:10DE600053442046726565202053697A653A202024
:10DE70002020204D42000000616C6C00F0B50B309A
:10DE8000154D20F007010024144A0FE003688B426F
:10DE90000BD38B4205D95E1A43184768C3E9006764
:10DEA00000E04368136002C004E0021D106800280F
:10DEB000ECD12046002802D1286808B10020F0BD2E
:10DEC000064A07481060074A121A22F00702C0E902
:10DED000002401202860D7E7200300201C03002035
:10DEE000F4C30220F0C5022010B510F8013B11F870
:10DEF000014B1B1B521E01D0002BF6D0184610BD43
:10DF0000002A05D011F8013B00F8013B521EF9D15F
:10DF10007047C9B200F8011B521EFBD170470000C8
:10DF2000034810B50068FDF733FC002010BD000069
:10DF3000040300200148FDF73ABC0000B8C20220EB
:10DF4000FDF7B2BF10B586B004460020059005AAC3
:10DF500069462046FDF7C1FC010004D007A0FBF78D
:10DF600073F906B010BD6A4621460AA0FBF76CF9AA
:10DF700021460EA0059AFBF767F9F2E70D0ABBF1FF
:10DF8000C8A1CAA7B0DCA3ACB4EDCEF3C2EB3A256E
:10DF9000580D0A000D0AB4C5C5CC257320B5C4C5FB
:10DFA000CCB7FBCEAA3A25730D0A0000B4C5C5CC88
:10DFB000257320B5C4D0F2C1D0BAC53A25580D0A90
:10DFC0000D0A000010B50146074A084812680068AB
:10DFD000FDF7FCFC01460078002804D0BDE81040A5
:10DFE00003A0FBF731B910BD040300200C0300208F
:10DFF0000D0A54686520537472696E67205265611A
:10E000006465642049733A25730D0A00024602488C
:10E0100000230068FDF7FCBC04030020FDF756BE9A
:10E02000034603480A4619464068FEF79FB90000B8
:10E0300088C102200A46014601480068FEF7BCB9C3
:10E040000403002001460148FEF7F1BAB8C20220DD
:10E05000034910B50968FEF754FBC0B210BD0000BB
:10E0600004030020034910B50968FEF768FBC0B23D
:10E0700010BD0000040300202DE9F05F804600265B
:10E08000354632A0FBF7E0F80027DFF8D8A0DFF82C
:10E09000D8B026E03548344B4FF40072D146DAF858
:10E0A00000100068FEF76EFB060004D0014630A0A9
:10E0B000FBF7CAF818E0BBF80010CA4629448DB235
:10E0C0000024D94607E0DAF80000015D2CA0FBF738
:10E0D000BBF8641CA4B2D9F800008442F3D37F1CBF
:10E0E000BFB2B7EB582FD5D35FEAC85022D01F4834
:10E0F000C8F308021C4BD046DAF800100068FEF79F
:10E1000041FB060004D001461EA0FBF79DF811E07C
:10E11000BBF800005F46284485B2002407E0D8F829
:10E120000000015D16A0FBF78FF8641CA4B23868EC
:10E130008442F4D31DB1294617A0FBF785F81CA033
:10E14000FBF782F83046BDE8F09F00000D0A5265EB
:10E1500061642066696C6520646174612069733A4A
:10E160000D0A00000C03002010030020040300200F
:10E1700052656164204572726F723A25640D0A001F
:10E18000256300000D0A52656164204572726F724A
:10E190003A25640D0A0000000D0A52656164656449
:10E1A0002064617461206C656E3A25640D0A00007C
:10E1B000526561642064617461206F7665720D0A36
:10E1C0000000000010B525492548FEF796FB002801
:10E1D00042D124A0FBF738F8214C26A0A16AFBF716
:10E1E00033F8A18827A0FBF72FF82AA0A168FBF736
:10E1F0002BF8D4E904232CA0FBF726F830A0616AA1
:10E20000FBF722F833A0E16AFBF71EF835A0216B7B
:10E21000FBF71AF837A0E16BFBF716F814A0FBF731
:10E2200013F80E4938A01A31FBF70EF80B4C3BA03F
:10E23000D4E90023FBF708F821893DA0FBF704F897
:10E24000618940A0FBF700F8217B43A0FAF7FCFFAF
:10E2500007A0FAF7F9FF002010BD000098C10220C6
:10E26000B8C202200D0A2044495220696E666F3AF6
:10E270000D0A00006469722E647074723A25640D90
:10E280000A0000006469722E6F626A2E69643A2582
:10E29000640D0A006469722E6F626A2E73636C7576
:10E2A00073743A25640D0A006469722E6F626A2ED7
:10E2B0006F626A73697A653A256C6C640D0A0000B6
:10E2C0006469722E6F626A2E635F6F66733A2564AB
:10E2D0000D0A00006469722E636C7573743A2564CC
:10E2E0000D0A00006469722E736563743A25640D2B
:10E2F0000A0000006469722E626C6B5F6F66733A8D
:10E3000025640D0A0000000046696C65204E616DB1
:10E31000652069733A25730D0A00000046696C6533
:10E320002053697A652069733A256C6C640D0A0084
:10E3300046696C6520646174612069733A25640DD7
:10E340000A00000046696C652074696D6520697378
:10E350003A25640D0A00000046696C65204174741A
:10E36000722069733A25640D0A000000FEF700BBB5
:10E3700070B5064601460F48FEF759F9002817D137
:10E380000DA0FAF761FF0D4C04F11A050B4909487D
:10E39000FEF7B3FA00280BD1A17E002908D0314640
:10E3A00007A0FAF751FF294606A0FAF74DFFEDE75F
:10E3B00070BD0000B8C202200D0A000098C1022002
:10E3C00025732F0025730D0A0000000010B50446C8
:10E3D000FEF796FB010004D003A0BDE81040FAF759
:10E3E00033BF214608A0F8E70D0AB4C5C5CCC5CC9B
:10E3F000B7FBC9E8D6C3CAA7B0DCA3ACB4EDCEF373
:10E40000C2EB3A25580D0A000D0AB4C5C5CCC5CCDF
:10E41000B7FBC9E8D6C3B3C9B9A63A25730D0A003C
:10E420001CB5034600200446009001AA6946184620
:10E43000FDF7C7F990B9019988694C89801E009948
:10E4400060434C43B0F5A04F03D26208410804A0DA
:10E4500002E0C10AE20A0CA0FAF7F6FE20461CBD53
:10E460000D0AB4C5C5CCD7DCC8DDC1BF3A256420D0
:10E470004B420D0ABFC9D3C3BFD5BCE43A256420C3
:10E480004B420D0A000000000D0AB4C5C5CCD7DC14
:10E49000C8DDC1BF3A2564204D420D0ABFC9D3C3B0
:10E4A000BFD5BCE43A2564204D420D0A00000000AF
:10E4B00001480068006970470403002001480068B3
:10E4C000006B704704030020FEF7ABBC70B5054637
:10E4D0000C460EA0FAF7B8FE214612A0FAF7B4FED9
:10E4E0001648154B224629460068FEF71FFD04001A
:10E4F00002D0014612A002E00F48016815A0FAF709
:10E50000A3FE1AA0FAF7A0FE204670BD0D0A4265D0
:10E5100067696E2057726974652066696C652E2E76
:10E520002E0D0A0057726974652064617461206C55
:10E53000656E3A25640D0A001403002004030020D0
:10E540005772697465204572726F723A25640D0ABC
:10E550000000000057726974656420646174612072
:10E560006C656E3A25640D0A0000000057726974EC
:10E57000652064617461206F7665722E0D0A00005B
:10E5800010B504462EA1F1F796FE002837D02FA132
:10E590002046F1F790FE002833D030A12046F1F755
:10E5A0008AFE002830D030A12046F1F784FE0028F2
:10E5B0002DD031A12046F1F77EFE00282AD031A1CE
:10E5C0002046F1F778FE40B332A12046F1F773FE02
:10E5D00030B333A12046F1F76EFE20B333A12046BD
:10E5E000F1F769FE10B334A12046F1F764FE00B3E1
:10E5F00034A12046F1F75FFEF0B1002010BD334892
:10E6000010BD3248103010BD3048203010BD2F48AA
:10E61000303010BD2D48403010BD2C48503010BD5A
:10E620002A48603010BD2948703010BD274880301E
:10E6300010BD2648903010BD2448A03010BD000009
:10E64000636F6E76315F626961730000636F6E762F
:10E65000315F77656967687400000000636F6E76EC
:10E66000325F626961730000636F6E76325F776557
:10E670006967687400000000636F6E76335F6269DB
:10E6800061730000636F6E76335F776569676874E6
:10E69000000000006663315F626961730000000082
:10E6A0006663315F77656967687400006663325F2F
:10E6B00062696173000000006663325F77656967B5
:10E6C00068740000646174610000000000C30220EF
:10E6D00010B504461DA1F1F7EEFD002815D0204627
:10E6E000FFF74EFF0446016819A0FAF7ADFD1EA022
:10E6F0006168FAF7A9FD24A0A168FAF7A5FDE16811
:10E70000BDE8104027A0FAF79FBD2DA0FFF7E0FF5E
:10E710002EA0FFF7DDFF31A0FFF7DAFF32A0FFF7F1
:10E72000D7FF35A0FFF7D4FF36A0FFF7D1FF39A000
:10E73000FFF7CEFF3AA0FFF7CBFF3CA0FFF7C8FFE3
:10E740003DA0FFF7C5FF3FA0C3E70000616C6C0070
:10E750000D0A6D6F64656C2E6E616D652069733A8C
:10E760002025730D0A0000006D6F64656C2E6172C8
:10E770007261792E616464726573732069733A20E3
:10E78000305825580D0A00006D6F64656C2E6D6160
:10E79000786C656E6774682069733A2025640D0A89
:10E7A000000000006D6F64656C2E7265616C656EB3
:10E7B0006774682069733A2025640D0A0000000020
:10E7C000636F6E76315F626961730000636F6E76AE
:10E7D000315F77656967687400000000636F6E766B
:10E7E000325F626961730000636F6E76325F7765D6
:10E7F0006967687400000000636F6E76335F62695A
:10E8000061730000636F6E76335F77656967687464
:10E81000000000006663315F626961730000000000
:10E820006663315F77656967687400006663325FAD
:10E8300062696173000000006663325F7765696733
:10E8400068740000646174610000000070B5324CAF
:10E850002EA0206000F008FC60602020A060103432
:10E860002EA0206000F000FC60604FF49070A0606B
:10E8700010342EA0206000F0F7FB60604020A06004
:10E8800010342DA0206000F0EFFB60604FF490404A
:10E89000A06010342CA0206000F0E6FB8025C4E9C5
:10E8A000010510342BA0206000F0DEFB60604FF407
:10E8B0009030A06010342BA0206000F0D5FBC4E99C
:10E8C000010510342AA0206000F0CEFB60604FF4F8
:10E8D0001010A060103429A0206000F0C5FB60601B
:10E8E0000720A060103428A0206000F0BDFB60600D
:10E8F0004FF46070A060103426A0206000F0B4FBDC
:10E90000606042F21070A06070BD0000636F6E76B0
:10E91000315F62696173000000C30220636F6E762D
:10E92000315F77656967687400000000636F6E7619
:10E93000325F626961730000636F6E76325F776584
:10E940006967687400000000636F6E76335F626908
:10E9500061730000636F6E76335F77656967687413
:10E96000000000006663315F6269617300000000AF
:10E970006663315F77656967687400006663325F5C
:10E9800062696173000000006663325F77656967E2
:10E990006874000064617461000000002DE9FC41AE
:10E9A0008846044631A1F1F786FC28B12046FFF7DE
:10E9B000E7FD0646002546E041462DA0FFF7EEFFA5
:10E9C00041462EA0FFF7EAFF414630A0FFF7E6FFE1
:10E9D000414631A0FFF7E2FF414633A0FFF7DEFFDB
:10E9E000414634A0FFF7DAFF414636A0FFF7D6FFD5
:10E9F000414637A0FFF7D2FF414638A0FFF7CEFFD0
:10EA0000414639A0FFF7CAFF41463AA0C8E705FBD7
:10EA100008F77068A74202D200EB870004E06FF0AD
:10EA2000030101EB840108440068F1F7EAFCA74206
:10EA3000CDE9000101D23A4600E0621E2FA0316804
:10EA4000FAF702FC6D1CF468B4FBF8F2B4FBF8F1C1
:10EA500008FB124008B1022000E001200844A8424F
:10EA6000D5D8BDE8FC412BA0FAF7EEBB616C6C0079
:10EA7000636F6E76315F626961730000636F6E76FB
:10EA8000315F77656967687400000000636F6E76B8
:10EA9000325F626961730000636F6E76325F776523
:10EAA0006967687400000000636F6E76335F6269A7
:10EAB00061730000636F6E76335F776569676874B2
:10EAC000000000006663315F62696173000000004E
:10EAD0006663315F77656967687400006663325FFB
:10EAE00062696173000000006663325F7765696781
:10EAF0006874000064617461000000000D0A2573F1
:10EB00005F666C6F617441727261795B25645D3A16
:10EB1000202566000D0A00002DE9F04F89B08046DF
:10EB20007BA1F1F7C8FBA0B14FF0000A5446D346D1
:10EB3000CDF814A0CDF818A014216846CDF81CA07B
:10EB4000F1F7A2FB4046FFF71BFD724F05002AD0EC
:10EB50003AE071A0FFF7E0FF72A0FFF7DDFF75A0BC
:10EB6000FFF7DAFF76A0FFF7D7FF79A0FFF7D4FF12
:10EB70007AA0FFF7D1FF7DA0FFF7CEFF7EA0FFF7C1
:10EB8000CBFF80A0FFF7C8FF81A0FFF7C5FF83A0E0
:10EB9000FFF7C2FF5EA0FFF79BFDF9F76FF90020BA
:10EBA00009B0BDE8F08F42467EA16846FAF75CFBEB
:10EBB000014601223868FDF7FFFBB0B977A0FFF7E7
:10EBC000DFFC0546C0F80080686810B9404600F0D8
:10EBD0004BFA74A168462A68FAF746FB4D480122B1
:10EBE00069460068FDF7E8FB28B1694670A0F2F7B6
:10EBF000BDF9C820D4E7694673A0F2F7B7F9D5E9A3
:10EC0000001028B175A0F2F7B1F978A0296871E079
:10EC10007EA0F2F7ABF9C920C2E7DFF814823D48C5
:10EC2000824B0B22D8F800100068FDF7ABFD5FEABD
:10EC3000000A06D0024669467EA0F2F797F9CA207C
:10EC4000AEE70027DFF8E4910DE0D8F80000C25DE0
:10EC50000D2A1DD07EA108A8FAF706FB08A905A871
:10EC6000F1F71DFB7F1CD9F800008742EDD3A8689F
:10EC7000B0F5903F40D30A21B0FBF1F1B4FBF1F2C3
:10EC800001FB1241B9B1A04215D9012C34D112E0D7
:10EC900005A8FAF71DFB51EC100BF1F7C5FB014677
:10ECA000CDF814B0CDF818B0CDF81CB0686840F8B5
:10ECB0002410641CD6E7A04201D8642602E0012C8F
:10ECC0000DD00A3663A0F2F751F9002706EBD6788B
:10ECD000B7EB680F05DA60A0FAF7B6FA04E0002691
:10ECE000F0E75EA0F2F742F97F1CBFB2322FEFD3FC
:10ECF00031465BA0FAF7A8FAA868A0428DD8EC606C
:10ED0000224659A02968F2F731F9504648E7000039
:10ED1000616C6C0004030020636F6E76315F626982
:10ED200061730000636F6E76315F77656967687441
:10ED300000000000636F6E76325F626961730000ED
:10ED4000636F6E76325F77656967687400000000F4
:10ED5000636F6E76335F626961730000636F6E7616
:10ED6000335F776569676874000000006663315F30
:10ED700062696173000000006663315F77656967EF
:10ED8000687400006663325F6269617300000000AE
:10ED90006663325F776569676874000064617461F7
:10EDA00000000000303A2F25732E747874000000A4
:10EDB0000D0ACEC4BCFE5B25735DB4F2BFAACAA720
:10EDC000B0DC0D0A000000000D0ACEC4BCFEC3FB7F
:10EDD000CEAAA3BA25730D0A00000000CAFDD7E928
:10EDE000C3FBCEAAA3BA25730D0A00000D0AD5FDF8
:10EDF000D4DAD0B4C8EB2573A3ACC7EBC9D4BAF34B
:10EE00002E2E2E2E2E2E0D0A000000000D0ACEDE14
:10EE1000B7A8BBF1C8A1C4A3D0CDB2CECAFD5B25B3
:10EE2000735DB5C4CAFDD7E90000000010030020DF
:10EE30000C030020B6C1C8A15B25735DCEC4BCFE27
:10EE4000B5C4CAFDBEDDB3F6B4ED3A25640D0A00C3
:10EE5000256300000D0A5B003D000000200000005B
:10EE60005D202564252500000D0A5B25735DB5C472
:10EE7000C4A3D0CDB2CECAFDD2D1D0B4C8EBB5BDFB
:10EE8000C4DAB4E6D6D02120C4A3D0CDB3A4B6C88A
:10EE9000CEAA2025640D0A0070B54E4D064600240A
:10EEA000686828B14CA13046F1F705FA002865D012
:10EEB000484D1035686828B14AA13046F1F7FBF992
:10EEC00000285BD0434D2035686828B149A1304601
:10EED000F1F7F1F9002851D03E4D3035686828B17E
:10EEE00047A13046F1F7E7F9002847D0394D4035C2
:10EEF000686828B146A13046F1F7DDF900283DD019
:10EF0000344D5035686828B144A13046F1F7D3F943
:10EF1000002833D02F4D6035686820B143A13046BA
:10EF2000F1F7C9F950B32B4D7035686820B142A193
:10EF30003046F1F7C0F908B3264D8035686820B136
:10EF400040A13046F1F7B7F9C0B1224D903568685D
:10EF500020B13FA13046F1F7AEF978B11D4DA03593
:10EF6000686820B13AA13046F1F7A5F930B13BA16C
:10EF70003046F1F7A0F948B1002070BD0120696862
:10EF800000F0E0FA6C600120EC6070BD12A0FFF7A9
:10EF900083FF14A0FFF780FF16A0FFF77DFF18A0E6
:10EFA000FFF77AFF1AA0FFF777FF1CA0FFF774FFA7
:10EFB0001EA0FFF771FF20A0FFF76EFF21A0FFF753
:10EFC0006BFF23A0FFF768FF25A0FFF765FF022076
:10EFD00070BD000000C30220636F6E76315F62690E
:10EFE00061730000636F6E76315F7765696768747F
:10EFF00000000000636F6E76325F6269617300002B
:10F00000636F6E76325F7765696768740000000031
:10F01000636F6E76335F626961730000636F6E7653
:10F02000335F776569676874000000006663315F6D
:10F0300062696173000000006663315F776569672C
:10F04000687400006663325F6269617300000000EB
:10F050006663325F7765696768740000616C6C0095
:10F0600064617461000000002DE9F14F9B4C606801
:10F0700020B99BA10098F1F71EF920B1974D1035EA
:10F08000686838B10BE08021012000F067FA606009
:10F09000BDE8F88F95A10098F1F70DF920B18F4EDA
:10F0A0002036706838B10BE04FF49061012000F019
:10F0B00055FA6860ECE791A10098F1F7FCF820B1EF
:10F0C000864F3037786838B10BE04FF480710120FB
:10F0D00000F044FA7060DBE78BA10098F1F7EBF8E1
:10F0E00038B1DFF8F8A10AF1400ADAF8040038B1C3
:10F0F0000BE04FF49031012000F030FA7860C7E760
:10F1000085A10098F1F7D7F820B1744850304068D5
:10F1100040B10CE04FF40071012000F01FFACAF872
:10F120000400B5E77FA10098F1F7C5F820B16B485E
:10F130006030406840B10CE04FF49021012000F0B5
:10F140000DFA664950314EE07AA10098F1F7B3F814
:10F1500038B1DFF8888108F17008D8F8040040B1B0
:10F160000CE04FF40071012000F0F8F95B496031C8
:10F1700039E073A10098F1F79EF838B1DFF85CB17F
:10F180000BF1800BDBF8040040B10CE04FF41001F0
:10F19000012000F0E3F9C8F8040079E76BA10098BA
:10F1A000F1F789F820B14D489030406838B10BE054
:10F1B0001C21012000F0D2F9CBF8040068E766A119
:10F1C0000098F1F778F838B1DFF8109109F1A0094B
:10F1D000D9F8040048B10DE04FF46061012000F05F
:10F1E000BDF93E499031486052E75EA10098F1F7C1
:10F1F00062F828B15DA10098F1F75DF840B16BE0CD
:10F2000049F64041012000F0A9F9C9F804003FE7A0
:10F21000606820B98021012000F0A0F96060686872
:10F2200028B94FF49061012000F098F96860706887
:10F2300028B94FF48071012000F090F9706078686F
:10F2400028B94FF49031012000F088F97860DAF89D
:10F250000400544628B94FF40071012000F07EF9F3
:10F2600060601E4C5034606828B94FF49021012032
:10F2700000F074F96060194C6034606828B94FF48C
:10F280000071012000F06AF96060D8F8040044467B
:10F2900028B94FF41001012000F060F96060DBF83C
:10F2A00004005C4620B91C21012000F057F9606081
:10F2B0000A4C9034606828B94FF46061012000F076
:10F2C0004DF96060D9F804004C4628B949F6404130
:10F2D000012000F043F960600020D9E600C302205D
:10F2E000636F6E76315F626961730000636F6E7683
:10F2F000315F77656967687400000000636F6E7640
:10F30000325F626961730000636F6E76325F7765AA
:10F310006967687400000000636F6E76335F62692E
:10F3200061730000636F6E76335F77656967687439
:10F33000000000006663315F6269617300000000D5
:10F340006663315F77656967687400006663325F82
:10F3500062696173000000006663325F7765696708
:10F36000687400006461746100000000616C6C00EE
:10F3700070B50446006B0E460025B0420FD0204603
:10F3800000F068FC05000AD160780123324604F1E0
:10F390003401FCF74FF908B16E1E0125266328469B
:10F3A00070BD000070B5134A131893F8203093B164
:10F3B000114B53F820308B421AD90F4B02EB8002CD
:10F3C0000C3B53F820305069B1FBF3F150F8214069
:10F3D0000020034608E011688847012070BD556988
:10F3E0000E18401C45F82630A042F8DB002070BD06
:10F3F000022070BD3C0000209853010830B504463F
:10F400000748084D002150F82400820005EB8400D5
:10F41000406900F0B3F80120291981F8200030BDBF
:10F42000805301083C0000202DE9F0411E4E0546A6
:10F43000002470190F4690F8200010B93168284652
:10F4400088474FF0FF326FB3184B53F82510B7FBC6
:10F45000F1F0B7FBF1FC01FB1C7101B1401C134939
:10F460000C3951F82510491E1CD406EB8506776926
:10F4700057F821C0BCF1000F04D0002484420FD102
:10F48000002206E0641CF9E774698F18521C44F8E6
:10F4900027008242F8D353F825004843BDE8F081A5
:10F4A000491EE5D51046F9E73C0000208C530108C1
:10F4B00070B50546114E1248002400EB8502214626
:10F4C00056F8250005E0536953F8213003B1641C58
:10F4D000491C8842F7D821460AA0F9F7B5FE56F82C
:10F4E000252029460EA0F9F7AFFE4FF47A70444369
:10F4F00056F82500B4FBF0F080B270BD80530108CF
:10F500003C0000200D0A6D795F6D656D5F7065725E
:10F510007573656420757365643A256400000000A6
:10F520000D0A6D795F6D656D5F70657275736564E9
:10F53000206D656D74626C73697A655B25645D3AF4
:10F5400025640000002906D0034A02EB800292687D
:10F55000891AFFF727BF70473C00002010B504460A
:10F56000FFF762FF411C05D0034901EB8401896864
:10F57000084410BD002010BD3C00002001E000F850
:10F58000011B521EFBD270472DE9F04780460F4603
:10F5900001F11A00FEF7D4FA20BB3878012600F0FA
:10F5A0003F00401E00EB8001DFF8489001EBC004F3
:10F5B00000254FF6FF7A19F805003844FEF7C0FA27
:10F5C00036B1FF2C0ED228F814000646641C01E068
:10F5D000504507D16D1C0D2DEDD33878400607D569
:10F5E000FF2C02D30020BDE8F087002128F814107A
:10F5F0000120F8E7A45301082DE9F0470226174639
:10F600000D46044602296FD3A069A8426CD9207820
:10F610004FF00109012806D0022838D0032846D02F
:10F62000042861D143E0616A05EB550801EB5821DC
:10F630002046FFF79DFE060056D1C8F3080020447F
:10F64000343008F10108E90704D00178FAB262F316
:10F650001F1100E03946017084F80390616A20466A
:10F6600001EB5821FFF784FE06003DD1C8F30800E6
:10F6700020443430E90702D0C7F3071105E00178D0
:10F68000C7F3032201F0F001114301702AE0606A20
:10F6900000EB15212046FFF76BFE060024D1E8B2EF
:10F6A00004EB4000B9B2343000F0F9F91AE0606AB6
:10F6B00000EBD5112046FFF75BFE060014D140F2A7
:10F6C000FF1000EA8500217805193435042905D09A
:10F6D0002846FEF7FFF967F31B0007462846394620
:10F6E00000F0B0F984F803903046BDE8F08738B5F3
:10F6F00045680446002D16DB60196D1C01733D2D15
:10F700000DDB6B462A4604F10C012068FDF70EFC68
:10F710000098A84201D1002501E04FF0FF35656057
:10F72000A068401CA06038BD006870472DE9F04714
:10F7300089460468924680460F464E46022936D3D3
:10F74000A069B84233D9BAF1000F0ED0207804284E
:10F7500003D198F80700022807D04FF0FF32514636
:10F760002046FFF749FF002822D139464046FEF7E0
:10F7700023F8050033D0012D19D0681C1AD0207849
:10F78000042806D0002239462046FFF735FF00281E
:10F790000ED16069411C05D0401C6061207940F0A9
:10F7A00001002071701CA84206D12E4613E00220F1
:10F7B000BDE8F0870120FBE72078042809D1A6EBFB
:10F7C0000902002349462046521CFAF7E1FC0028B2
:10F7D000EED12E46B146A0692F46B842C5D8207852
:10F7E000042815D1BAF1000F04D098F807000328B7
:10F7F00002D00DE0002109E0D8F80800504507D8F4
:10F80000D8F818100144514502D3022188F8071096
:10F810000020CDE72DE9F04F05468BB000200C46C7
:10F82000064608900090019002909146142103A88A
:10F83000F0F72AFD2046FEF7A3FE8068A84200D814
:10F84000451E2046FFF710FC5FEA00080DD0224657
:10F8500047A103A8F9F708FD4848012203A9006859
:10F86000FCF7AAFDDFF818A132E046A0F1F77EFB15
:10F8700007200BB0BDE8F08F4048464B0B22DAF86A
:10F8800000100068FCF77EFF089020B1014642A0FE
:10F89000F1F76CFB1CE00024DFF8F8B014E0DAF8B4
:10F8A00000005746025D0D2A16D040A109A8F9F7BD
:10F8B000DBFC09A96846F0F7F2FC38682146025DD6
:10F8C0003BA0F1F753FB641CDBF800008442E6D355
:10F8D000AE42D1D9002438E06846F9F7F9FC51EC82
:10F8E000100BF0F7A1FD0746002000900190029058
:10F8F00048F826706A46214630A0761CF1F736FBA0
:10F900003846F0F77EFD41EC100B611C53EC102BD8
:10F9100033A0F1F72BFBD6E704FB09F6AE4202D881
:10F9200008EB860001E008EB85000068F0F769FD50
:10F9300041EC100BAE4201D8314600E0294653ECB1
:10F94000102B30A0F9F780FC641CB5FBF9F2B5FB75
:10F95000F9F109FB125008B1022000E0012008442F
:10F96000A042D9D814A0F9F76FFC089881E70000ED
:10F97000303A2F25732E74787400000004030020A1
:10F980000C030020B3F5CABCBBAFB3F6B4EDA3A122
:10F99000A3A10000100300200D0AB6C1CAFDBEDD00
:10F9A000B3F6B4EDC1CB3A25640D0A00256300001F
:10F9B0005B25645D3A2025630D0A0000BBD8B3B512
:10F9C0005B25645D20B5A5D0D0CAFDBEDDCAC75B8E
:10F9D000737472696E675D3A2025730D0A0000002A
:10F9E000BBD8B3B55B25645D20B5A5D0D0CAFDBE3C
:10F9F000DDCAC75B666C6F61745D3A2025660D0ACF
:10FA0000000000000D0A666C6F61744172726179CA
:10FA10005B25645D3A2025660000000070B50C4649
:10FA20000646154691B204F11A0000F038F8307815
:10FA3000032806D1290C04F11400BDE8704000F041
:10FA40002EB870BD0170090A4170090A8170090A57
:10FA5000C170704710B5110A027041EA036141702C
:10FA60001A0A090A41EA02618170120A090A41EA86
:10FA70000261C170120A090A41EA02610171120AA7
:10FA8000090A41EA02614171120A090A41EA026166
:10FA9000120A8171090A41EA0261C17110BD017047
:10FAA000090A417070472DE9F04104460068C568B5
:10FAB000284601F084F80146A81CFFF7F0FF6F7894
:10FAC00020467F1CE16BFBF708FD06464FF001085E
:10FAD0000FE020222946606BFEF712FA21687F1E94
:10FAE00081F803800DD0002120462035FBF7B2FAC3
:10FAF00006463EB9216B2068FFF73AFC0600E8D0C5
:10FB000000E026B1012E02D00220BDE8F08130468F
:10FB1000FBE7014600200B22430803EBC01011F85D
:10FB2000013B521E1844C0B2F6D1704710B586B0E2
:10FB3000044614216846F0F7A7FB22460EA168464A
:10FB4000F9F792FB01460F4801220068FCF734FCEC
:10FB5000694628B10CA0F1F709FAC82006B010BD1B
:10FB60000FA0F1F703FA2046FEF7D6FF214613A0B7
:10FB7000F9F76AFB0120F1E7303A2F25732E7478EC
:10FB800074000000040300200D0ACEC4BCFE5B25F7
:10FB9000735DB4F2BFAACAA7B0DC0D0A0000000072
:10FBA0000D0AD0C2B5C464617461CEC4BCFEC3FB8F
:10FBB000CEAAA3BA25730D0A00000000D2D1C7D087
:10FBC000BBBBB5BD2025732E7478740070B5044698
:10FBD00000F040F8050036D1207803282CD1207998
:10FBE000012829D1420204F1340000210646FEF723
:10FBF00090F94AF6552104F23220FFF750FF1349DD
:10FC00003046FFF71FFF124904F50670FFF71AFF91
:10FC100004F507706169FFF715FF04F508702169A5
:10FC2000FFF710FF226A0123521C226360783146DD
:10FC3000FBF735FD00202071002260781146FBF7AC
:10FC4000ABFC00B10125284670BD00005252614155
:10FC5000727241612DE9F0410446C0780027F8B185
:10FC6000266B04F134016078012332468846FBF7A5
:10FC700016FD08B1012713E00020E070606AE16919
:10FC8000301A88420CD2A57808E0E06901230644C6
:10FC9000607832464146FBF702FD6D1E022DF4D21C
:10FCA0003846BDE8F08100000749064AC1E9002056
:10FCB00000208860C860086188610C20486108469F
:10FCC000F3F768BF00100140F003002070B594B056
:10FCD000064613AB11AA694600F0D8F9002824D1D2
:10FCE0008DF840001D4C042514E0206805EBC1018F
:10FCF00013AB405812AA08A900F0C8F9002814D183
:10FD0000694608A800F0E2FB88B19DF84000401C5D
:10FD10008DF84000207D9DF840108842E5D8207D78
:10FD20009DF8401088420ED1042014B070BD9DF89B
:10FD300048009DF84410884201D90220F5E79DF85B
:10FD40004000A075EBE710A9304600F053FA0028F8
:10FD5000EBD19DF8400060750020E6E70C02002022
:10FD60002DE9F0417E4E9AB0B57D307DA8427CD918
:10FD70000421306801EBC50119AB405818AA10A93D
:10FD800000F084F910A977A0F9F75EFA00240DF1CC
:10FD9000180832E0308B0121A140084217D02221FF
:10FDA00072A0F9F751FA204600F08CFA811970A080
:10FDB0002431F9F749FA22216CA0F9F745FA2046D7
:10FDC00000F080FA3044243048F824000BE020464C
:10FDD00000F078FA3044416A48F82410F07D00B30E
:10FDE00064A0F9F731FA9DF86000401E844202D009
:10FDF00062A0F9F729FA641CE4B29DF8600084421D
:10FE0000C8D35FA0F9F720FA00F0A2FA707D0B28A2
:10FE100014D2DFE800F0080D31384048525E6B78AC
:10FE2000890058A0DDE7306850F83500804704E0CD
:10FE3000306850F8351006988847074600F054FAA5
:10FE40009DF8640001286ED04FA0F9F7FDF996F8EF
:10FE5000EC0000280DD0D6F8F0000A21B0FBF1F23A
:10FE600001FB1202B0FBF1F100E002E047A0F9F75C
:10FE7000EBF91AB0BDE8F081306850F83520DDE9C3
:10FE800006019047D9E7306806AC50F8353094E861
:10FE900007009847D1E7306806AF50F8354097E83B
:10FEA0000F00A047C9E70A980090306806AF50F8E5
:10FEB000354097E80F00A047BFE7DDE90A01CDE92B
:10FEC0000001306806AF50F8354097E80F00A047B2
:10FED000B3E70AAB06AF93E807008DE80700306888
:10FEE00050F8354097E80F00A047A6E70AAC06AFE8
:10FEF00094E80F008DE80F00306850F8354097E81F
:10FF00000F00A04799E70BAC06AF94E80F0001ACD7
:10FF100084E80F000A980090306850F8354097E860
:10FF20000F00A04789E711E00CAC06AF94E80F0082
:10FF300002AC84E80F00DDE90A01CDE90001306878
:10FF400050F8354097E80F00A04776E7F07D394636
:10FF500018B116A0F9F778F979E717A0FAE70000C9
:10FF60000C0200200D0A2573280000002563000004
:10FF70002573000030582558000000002C000000B8
:10FF800029000000256C64003B0D0A0046756E6375
:10FF900074696F6E2052756E2054696D653A2564E0
:10FFA0002E2531646D730D0A000000003D30582588
:10FFB000583B0D0A000000003D256C753B0D0A0002
:10FFC000F0B500252E462F462C4603782C2B03D067
:10FFD000292B04D01BB103E014B9012600E05CB367
:10FFE00017B1222B26D026E0A3F1300CBCF1090F6B
:10FFF00015D9A3F1610CBCF1050F10D9A3F1410C87
:020000040801F1
:10000000BCF1050F0BD9582B09D0782B07D0222B28
:100010000CD0202B1ED02C2B1CD0FF270CE05EB95F
:10002000612B00D3203B01F8013B13E026B90127E7
:100030003C460FE0002426B10020087017702846C7
:10004000F0BD3CB15C2B02D16D1CEDB2401C0378BD
:1000500001F8013B6D1CEDB2401CB6E730B5002540
:1000600015700AE001F8014B1478401C641CE4B2DE
:1000700014709C4201D3012030BD0478202C01D0A3
:10008000002CEFD10D70002030BD00002DE9FF4F96
:10009000002482B089469846A24627460125264676
:1000A0002246EB46029915E0202810D002F07F038B
:1000B000052B0CD202B9802202F07F03042B01D160
:1000C0002A280AD1521C0BF80300D2B201E0852A7B
:1000D00004D0491C08780028E6D16AB102F07F02FA
:1000E00000200BF8020041A1584600F0EFF938B1AA
:1000F000012188F8001000224FF00008029B15E053
:10010000002088F80000F6E708F1010000F0FF0881
:1001100013F8010F202801D02A2807D1184600F033
:100120007DF9282802D02A2800D0C246187828282D
:1001300001D00028E8D10299BAF1000F01D0514452
:10014000491C4FF000084346087888B1282804D09D
:10015000292806D0222810D011E083B9641CE4B20B
:100160000DE063B924B1641E14F0FF0402D00DE069
:100170004FF00108012F27D02FE04BB100234CB1E5
:100180002C280CD0202816D0282814D05AB110E0E2
:100190000123F4E7202815D009F8010B12E001250E
:1001A000521CD2B207E0052E03D20BF80600761CD3
:1001B000F6B26D1CEDB2012C04D1022D02D1032543
:1001C0007F1CFFB2491CBFE700200BF8060007A107
:1001D000684600F07BF900B90027049807700020FA
:1001E00089F8000006B04046BDE8F08F766F69647C
:1001F000000000002DE9F04300248946304DB5B0E1
:10020000214622466B18491CC9B29A760A29F9D3AD
:1002100002E010F8011F99B101782829F9D1461C94
:100220004FF0010833AA69463046FFF7C9FE06447D
:100230009DF8CC0040B1012824D0FF2836D10BE036
:10024000012035B0BDE8F0839DF8000070B334A9FB
:10025000684600F0EBF808B10220F2E7204600F013
:1002600031F8284434994162298B08FA04F081431B
:100270002983042029198876641CE4B20A2C15D934
:100280000320DEE7684600F036F9471C204600F000
:1002900019F841196846243100F024F9298B08FA2D
:1002A00004F00143281929838776E5E73078292867
:1002B00001D00028B6D189F800400020C1E7000035
:1002C0000C020020024610B500200146054B05E057
:1002D0005C18491CA47EC9B22044C0B29142F7D335
:1002E00010BD00000C020020094800680169C943E4
:1002F000CA070849D1F8F02004D14FF6FF731A4419
:10030000C1F8F020406A1044C1F8F00070470000C6
:1003100040C102200C02002000EBC00101EB0010E4
:100320004FF0FF3101EB800010B581B24FF47A70CD
:10033000F8F7F0FB01490120C87510BD0C02002040
:100340000346012000E05843491EC9B2FBD2704762
:1003500007486FF00101026811610268090CD1625F
:10036000C1600068002141620248C0F8F010704787
:1003700040C102200C0200202DE9F041164E3088C9
:10038000010426D51549C0B2154F00250D54B96892
:100390001248884704000FD0104800F0B5F8012833
:1003A00001D0040014D0012C09D0022C09D0032C58
:1003B00009D0042C0CD108E0F868804708E009A0B7
:1003C00004E00BA002E00DA000E00FA0F8F73CFF56
:1003D0003580BDE8F08100001C00002028030020CB
:1003E0000C020020BAAFCAFDB4EDCEF3210D0A0015
:1003F000B2CECAFDB4EDCEF3210D0A00B2CECAFDD5
:10040000CCABB6E0210D0A00CEB4D5D2B5BDC6A5A1
:10041000C5E4B5C4BAAFCAFD210D0A0010F8011F2A
:10042000202901D10028F9D1C8B270472DE9F04147
:100430000024884605460A260C600178A1F13002A6
:10044000092A0DD9113A052A0AD9582905D011F0DF
:10045000FF0F0CD00120BDE8F081012C02D0F9E79C
:10046000412900D31026641CE4B2401CE5E7102E9D
:1004700001D084B112E0032C01D20220EBE72878EE
:10048000302802D16878582801D00320E3E7A41E61
:10049000E4B2AD1C01E00420DDE70CB1641EE4B25F
:1004A0002F783846303F092F01D9A0F13707214670
:1004B0003046FFF745FFD8F8001007FB0011C8F8D9
:1004C000001015F8010F0028E7D1C4E702780B7877
:1004D0009A4201D00120704712B1401C491CF5E737
:1004E0000020704702780A700278002A02D0401C6F
:1004F000491CF7E77047002102781AB1491CC9B2BC
:10050000401CF9E708467047F0B58DB004461E233D
:1005100008AA6946FFF7A2FD0990002872D19DF84C
:100520002000271800253E4C8DF820509DF8200013
:1005300054F820106846FFF7C9FF38B19DF8200035
:10054000401CC0B28DF820000728EFD39DF8200092
:100550000426344C072855D2DFE800F00404395A49
:10056000605F5E0030A0F8F76FFE30A0F8F76CFE19
:100570003EA0F8F769FE4DA0F8F766FE5BA0F8F71D
:1005800063FE6AA0F8F760FE78A0F8F75DFE86A02B
:10059000F8F75AFE8BA0F8F757FE93A0F8F754FE31
:1005A00097A0F8F751FE9CA0F8F74EFEA1A0F8F72F
:1005B0004BFEA7A0F8F748FEB3A0F8F745FEC0A091
:1005C000F8F742FECBA0F8F73FFED7A01BE016A03D
:1005D000F8F73AFEE4A0F8F737FE8DF820500BE06C
:1005E000216806EBC0000958EFA0F8F72DFE9DF832
:1005F0002000401C8DF82000217D9DF820008142C4
:10060000EED856E257E2F8F71FFE00200DB0F0BD1D
:1006100005A0F8F719FECBE12CE20CE2EBE10000BB
:10062000600000200C0200200D0A00002D2D2D2D51
:100630002D2D2D2D2D2D2D2D2D2D2D2D2D2D2D2DEA
:100640002D2D2D2D55534D4152542056332E332DE3
:100650002D2D2D2D2D2D2D2D2D2D2D2D2D2D2D2DCA
:100660002D2D2D2D2D2D2D200D0A00002020202098
:1006700055534D415254CAC7D3C9414C49454E54B4
:10068000454BBFAAB7A2B5C4D2BBB8F6C1E9C7C92A
:10069000B5C4B4AEBFDAB5F7CAD4BBA5BDBBD7E904
:1006A000BCFE2CCDA8B9FD200D0A0000CBFC2CC44B
:1006B000E3BFC9D2D4CDA8B9FDB4AEBFDAD6FACA69
:1006C000D6B5F7D3C3B3CCD0F2C0EFC3E6B5C4C838
:1006D000CEBACEBAAFCAFD2CB2A2D6B4D0D02ED2EA
:1006E000F2B4CB2CC4E3BFC90D0A0000D2D4CBE6D0
:1006F000D2E2B8FCB8C4BAAFCAFDB5C4CAE4C8EB0C
:10070000B2CECAFD28D6A7B3D6CAFDD7D628313077
:100710002F3136BDF8D6C62CD6A7B3D6B8BACAFD87
:1007200029A1A2D7D6B7FBB4AE0D0A00A1A2BAAFD9
:10073000CAFDC8EBBFDAB5D8D6B7B5C8D7F7CEAAC9
:10074000B2CECAFD292CB5A5B8F6BAAFCAFDD7EE10
:10075000B6E0D6A7B3D63130B8F6CAE4C8EBB2CE0D
:10076000CAFD2CB2A2D6A7B3D60D0A00BAAFCAFDF5
:10077000B7B5BBD8D6B5CFD4CABE2ED6A7B3D6B2DE
:10078000CECAFDCFD4CABEBDF8D6C6C9E8D6C3B955
:10079000A6C4DC2CD6A7B3D6BDF8D6C6D7AABBBB99
:1007A000B9A6C4DC2E0D0A00BCBCCAF5D6A7B3D6C8
:1007B0003A7777772E6F70656E6564762E636F6D0E
:1007C0000D0A000055534D415254D3D037B8F6CFDF
:1007D000B5CDB3C3FCC1EE28B1D8D0EBD0A1D0B415
:1007E000293A0D0A000000003F3A20202020202056
:1007F000BBF1C8A1B0EFD6FAD0C5CFA20D0A000058
:1008000068656C703A202020BBF1C8A1B0EFD6FA21
:10081000D0C5CFA20D0A00006C6973743A20202065
:10082000BFC9D3C3B5C4BAAFCAFDC1D0B1ED0D0ABB
:100830000A00000069643A2020202020BFC9D3C3E9
:10084000BAAFCAFDB5C44944C1D0B1ED0D0A0A0022
:100850006865783A20202020B2CECAFD3136BDF836
:10086000D6C6CFD4CABE2CBAF3B8FABFD5B8F12BCE
:10087000CAFDD7D6BCB4D6B4D0D0BDF8D6C6D7AA98
:10088000BBBB0D0A0A0000006465633A20202020EB
:10089000B2CECAFD3130BDF8D6C6CFD4CABE2CBA4E
:1008A000F3B8FABFD5B8F12BCAFDD7D6BCB4D6B4CD
:1008B000D0D0BDF8D6C6D7AABBBB0D0A0A0000002F
:1008C00072756E74696D653A312CBFAAC6F4BAAF01
:1008D000CAFDD4CBD0D0BCC6CAB13B302CB9D8B13C
:1008E000D5BAAFCAFDD4CBD0D0BCC6CAB13B0D0A75
:1008F0000A000000C7EBB0B4D5D5B3CCD0F2B1E05C
:10090000D0B4B8F1CABDCAE4C8EBBAAFCAFDC3FBE4
:10091000BCB0B2CECAFDB2A2D2D4BBD8B3B5BCFC77
:10092000BDE1CAF82E0D0A002D2D2D2D2D2D2D2DBA
:100930002D2D2D2D2D2D2D2D2D2D2D2D2D2D2D2DE7
:100940002D2D414C49454E54454B2D2D2D2D2D2DF2
:100950002D2D2D2D2D2D2D2D2D2D2D2D2D2D2D2DC7
:100960002D2D2D200D0A00002D2D2D2D2D2D2D2D61
:100970002D2D2D2D2D2D2D2D2D2D2D2D2D2D2D2DA7
:100980002DBAAFCAFDC7E5B5A52D2D2D2D2D2D2DC9
:100990002D2D2D2D2D2D2D2D2D2D2D2D2D2D2D2D87
:1009A0002D2D2D2D200D0A0025730D0A00000000AD
:1009B00042A0F8F749FC8DF8205016E0216806EBBC
:1009C000C0000BAB08580AAA6946FFF75FFB9DF809
:1009D0002010206850F83120694648A0F8F734FC10
:1009E0009DF82000401C8DF82000217D9DF82000FE
:1009F0008142E3D85DE0AFF2D030F8F725FC08AAD9
:100A000069463846FFF7DCFA9DF82000002843D1FC
:100A100009A96846FFF70AFD8DF8200010B10428E7
:100A20003AD102E03AA009991CE03CA0F8F70CFC8E
:100A30000120E0753DE038A0F8F706FC08AA6946F9
:100A40003846FFF7BDFA9DF8200028BB09A9684683
:100A5000FFF7ECFC8DF8200010B104281CD104E055
:100A600033A00999F8F7F0FB23E034A0F8F7ECFB8A
:100A7000E5751EE028A0F8F7E7FB08AA69463846A6
:100A8000FFF79EFA9DF8200030B909A96846FFF7E4
:100A9000CDFC8DF8200008B10220B7E5099810F0D0
:100AA000FF0084F8EC0001D029A000E02FA0F8F7A7
:100AB000CBFB19A0A7E50120A8E500002D2D2D2DC9
:100AC0002D2D2D2D2D2D2D2D2D2D2D2D2D2D2D2D56
:100AD0002D2D2D2D2DBAAFCAFD204944202D2D2DB1
:100AE0002D2D2D2D2D2D2D2D2D2D2D2D2D2D2D2D36
:100AF0002D2D2D2D2D2D2D2D200D0A002573206936
:100B0000642069733A0D0A3058253038580D0A00B0
:100B10004845583A305825580D0A00003136BDF87E
:100B2000D6C6B2CECAFDCFD4CABE210D0A0000007F
:100B30004445433A256C750D0A0000003130BDF87C
:100B4000D6C6B2CECAFDCFD4CABE210D0A0000005F
:100B500052756E2054696D652043616C63756C61DC
:100B600074696F6E204F4E0D0A00000052756E20A2
:100B700054696D652043616C63756C6174696F6E57
:100B8000204F46460D0A000070B50D4604000CD0FB
:100B9000206850B1017841B1C188A288914204D146
:100BA0004078FAF77AFDC00703D0002028600920BA
:100BB00070BD20682860002070BD0160704730B5AE
:100BC000034640784FF4004544010020014620349C
:100BD0000AE002290BD0C20700D02A4602EB5000DF
:100BE0005A5C104480B2491CA142F2D330BD0321AB
:100BF000F9E770B5054600244FF4004611E0FCF714
:100C0000ADFAE10700D0314601EB5401C2B2114404
:100C100089B2CA0700D0324602EB510101EB102025
:100C200084B235F8020B0028E9D1204670BD0000DF
:100C30000000010203040102030406070809000082
:100C400000000000000000000000000000003F4025
:100C500000000000000000003000400030004000B4
:100C6000000009000BC03D000BC03D00090018C08A
:100C700024407FE0224031800000180024C01B0087
:100C80000D803240018003801C4027401C800740BB
:100C900000401000600000000000000000000000A4
:100CA000000000001F802040402000004020204025
:100CB0001F8000000000090006001F8006000900D8
:100CC0000000040004003F80040004000000001045
:100CD00000600000000000000000040004000400A8
:100CE00004000400000000000040000000000000BC
:100CF0000000002001C006003800400000001F80F6
:100D00002040204020401F800000000010403FC0D5
:100D100000400000000018C021402240244018403C
:100D2000000010802040244024401B80000002006E
:100D30000D0011003FC0014000003C8024402440D1
:100D40002440238000001F8024402440344003803E
:100D500000003000200027C03800200000001B8069
:100D60002440244024401B8000001C0022C022405C
:100D700022401F800000000000000840000000002A
:100D800000000000000004600000000000000000FF
:100D900004000A00110020804040090009000900F9
:100DA00009000900000000004040208011000A00F6
:100DB00004001800200023402400180000001F80B9
:100DC0002040274029401F400000004007C0390054
:100DD0000F0001C0004020403FC0244024401B8041
:100DE00000001F8020402040204030800000204034
:100DF0003FC0204020401F80000020403FC02440D2
:100E00002E4030C0000020403FC024402E00300063
:100E100000000F001080204022403380020020405C
:100E20003FC0040004003FC02040204020403FC09D
:100E30002040204000000060202020203FC02000F3
:100E4000200020403FC024400B0030C02040204004
:100E50003FC020400040004000C03FC03C0003C0F5
:100E60003C003FC0000020403FC00C4023003FC07A
:100E700020001F802040204020401F800000204094
:100E80003FC024402400180000001F802140214062
:100E900020E01FA0000020403FC02440260019C0D1
:100EA000004018C02440244022403180000030001F
:100EB00020403FC020403000000020003F80004024
:100EC00000403F80200020003E0001C007003800A5
:100ED0002000380007C03C0007C038000000204058
:100EE00039C0060039C0204000002000384007C04B
:100EF000384020000000304021C02640384020C04B
:100F00000000000000007FE04020402000000000C2
:100F100070000C00038000400000000040204020D2
:100F20007FE00000000000002000400020000000E2
:100F30000000001000100010001000100010000051
:100F4000000040000000000000000000028005409A
:100F5000054003C0004020003FC00440044003801F
:100F60000000000003800440044006400000000030
:100F70000380044024403FC000400000038005403F
:100F8000054003400000000004401FC024402440EE
:100F90002000000002E005500550065004202040CB
:100FA0003FC00440040003C000400000044027C0CC
:100FB00000400000000000100010041027E00000B6
:100FC000000020403FC00140070004C00440204012
:100FD00020403FC000400040000007C0040007C0A0
:100FE000040003C00000044007C00440040003C024
:100FF000004000000380044004400380000004100F
:1010000007F0045004400380000000000380044007
:10101000045007F00010044007C002400400040020
:101020000000000006400540054004C0000000002C
:1010300004001F80044000400000040007800040BE
:10104000044007C000400400070004C001800600FF
:101050000400060001C0070001C0060000000440B3
:1010600006C0010006C0044000000410071004E0A0
:101070000180060004000000044005C00640044052
:1010800000000000000004007BE0402000000000A1
:1010900000000000FFF000000000000040207BE0A6
:1010A00004000000000040008000400020002000FC
:1010B00040000000000000000000000000000000F0
:1010C00000000000000000001FCC000C0000000029
:1010D00000000000080030006000080030006000E0
:1010E0000000022003FC1E20022003FC1E20022020
:1010F000000000000E1811043FFF10840C7800005F
:1011000000000F0010840F3800C0077818840078A2
:10111000000000780F8410C411240E9800E40084AD
:1011200000080800680070000000000000000000D7
:10113000000000000000000007E018182004400232
:101140000000000040022004181807E00000000022
:1011500000000240024001800FF001800240024086
:1011600000000080008000800FF800800080008078
:1011700000000001000D000E000000000000000053
:10118000000000000080008000800080008000805F
:1011900000800000000C000C0000000000000000B7
:1011A0000000000000060018006001800600180022
:1011B0002000000007F0080810041004080807F0D9
:1011C00000000000080408041FFC000400040000E4
:1011D000000000000E0C10141024104411840E0C9A
:1011E000000000000C1810041104110412880C7087
:1011F0000000000000E00320042408241FFC002459
:10120000000000001F981084110411041088107051
:101210000000000007F0088811041104188800700D
:10122000000000001C00100010FC13001C00100047
:10123000000000000E3811441084108411440E3850
:10124000000000000700088C10441044088807F0D4
:101250000000000000000000030C030C0000000070
:101260000000000000000001010600000000000076
:101270000000000000800140022004100808100453
:101280000000022002200220022002200220022070
:101290000000000010040808041002200140008033
:1012A000000000000E001200100C106C10800F00E7
:1012B000000003E00C1813E4142417C4082807D016
:1012C00000000004003C03C41C40074000E4001C74
:1012D000000410041FFC1104110411040E88007096
:1012E000000003E00C1810041004100410081C1077
:1012F000000010041FFC100410041004080807F07C
:10130000000010041FFC1104110417C41004081875
:10131000000010041FFC1104110017C01000080089
:10132000000003E00C181004100410441C78004066
:10133000000010041FFC10840080008010841FFC3B
:1013400010040000100410041FFC1004100400001E
:10135000000000030001100110011FFE100010002A
:10136000000010041FFC110403801464181C1004F6
:10137000000010041FFC1004000400040004000C12
:10138000000010041FFC1F0000FC1F001FFC1004C5
:10139000000010041FFC0C04030000E010181FFCE8
:1013A000100007F00808100410041004080807F0E3
:1013B000000010041FFC10841080108010800F00AB
:1013C000000007F0081810241024101C080A07F267
:1013D000000010041FFC1104110011C011300E0C8C
:1013E000000400000E1C11041084108410441C38EA
:1013F00000001800100010041FFC1004100018005A
:10140000000010001FF810040004000410041FF86E
:10141000100010001E0011E0001C007013801C0062
:1014200010001FC0103C00E01F0000E0103C1FC077
:1014300000001004180C163401C001C01634180C3A
:10144000100410001C00130400FC13041C00100006
:1014500000000804101C1064108413041C041018ED
:1014600000000000000000007FFE40024002400239
:101470000000000030000C0003800060001C00032E
:10148000000000004002400240027FFE0000000019
:10149000000000000000200040004000400020004C
:1014A0000000000100010001000100010001000135
:1014B000000100004000400020000000000000008B
:1014C000000000000098012401440144014400FC94
:1014D000000410001FFC0088010401040088007053
:1014E000000000000070008801040104010400886D
:1014F00000000000007000880104010411081FFCB6
:101500000004000000F8014401440144014400C803
:1015100000000000010401040FFC1104110411007B
:101520001800000000D601290129012901C901067E
:10153000000010041FFC008401000100010400FCF5
:10154000000400000104190419FC00040004000058
:1015500000000000000300010101190119FE000054
:10156000000010041FFC0024004001B4010C010421
:1015700000000000100410041FFC00040004000020
:101580000000010401FC0104010001FC0104010050
:1015900000FC010401FC008401000100010400FCC6
:1015A0000004000000F8010401040104010400F833
:1015B0000000010101FF00850104010400880070A2
:1015C000000000000070008801040104010501FF13
:1015D00000010104010401FC0084010401000180F8
:1015E0000000000000CC0124012401240124019802
:1015F000000000000100010007F8010401040000E0
:101600000000010001F8000400040004010801FCCE
:101610000004010001800170000C001001600180D5
:10162000010001F0010C003001C00030010C01F09C
:10163000010000000104018C00740170018C0104A0
:101640000000010101810171000E0018016001809C
:10165000010000000184010C013401440184010CEB
:101660000000000000000000000001003EFC4002FD
:1016700040020000000000000000FFFF000000002A
:1016800000000000400240023EFC0100000000009B
:10169000000000006000800080004000400020004A
:1016A000200000000000000000000000000000001A
:1016B000000000000000000000000000000000002A
:1016C000000000000000000000000000000000001A
:1016D00000000000000F80380FFE380F8038000037
:1016E00000000000000000000000000000000000FA
:1016F0000100000600000C00003800003100000668
:1017000000000C0000380000300000000000000065
:10171000000061800067F807F98000618000618047
:101720000061800061800067F807F9800061800037
:10173000000000000000000001C0E003E0F00630FF
:10174000080418081FFFFE040E080787F00381E055
:1017500000000000000001F000060C000404080670
:101760000C7001F9C0000E00003BE000EC18070807
:1017700008040C180003E00000000001E00007F07E
:1017800003F818041C0804170807E1D003C0E000A0
:1017900023B0003C080020080000100000000000FA
:1017A000000100003100003200001C0000000000B9
:1017B0000000000000000000000000000000000029
:1017C0000000000000000000000000000000000019
:1017D00000007F0001FFC00780F00C00181000041B
:1017E0002000020000000000002000021000040C95
:1017F00000180780F001FFC0007F0000000000001B
:101800000000000000000000000000000000420096
:10181000006600006600003C0000180003FFC000E6
:101820001800003C00006600006600004200000056
:101830000000080000080000080000080000080080
:1018400001FFC000080000080000080000080000B8
:10185000080000000000000100003100003200001C
:101860001C0000000000000000000000000000005C
:101870000000000000000000000008000008000058
:101880000800000800000800000800000800000828
:101890000000080000080000000000000000000038
:1018A0000000380000380000380000000000000090
:1018B0000000000000000000000000000000000028
:1018C0000000000600001C000070000180000E00F7
:1018D00000380000C0000700001C000030000000BD
:1018E0000000000000007F8001FFE0038070060020
:1018F0001804000804000806001803807001FFE0C7
:10190000007F8000000000000000000001000801CE
:10191000000801000803FFF807FFF80000080000B6
:101920000800000800000000000000000001C038AE
:1019300002C0580400980401180402180404180690
:101940001C1803F81801E0F8000000000000000077
:101950000001C0E003C0F0040008040808040808FF
:1019600006180803F41801E7F00001E00000000089
:101970000000000000000300000D000011000061E5
:101980000000810803010807FFF80FFFF8000108B5
:101990000001080000000000000000E007FCD00685
:1019A0000808061008061008061008061838060F62
:1019B000F00607C0000000000000000000003F80AB
:1019C00001FFE00384300208180410080410080422
:1019D0001008071810030FF00007C00000000000F7
:1019E0000000000003C0000700000600000600F829
:1019F0000607F806180006E00007000006000000D1
:101A0000000000000001E1E003F7F00634100418C4
:101A100008041808040C08040C0806161803F3F050
:101A200001C1E000000000000000F80003FC3003EA
:101A3000063804020804020804020804041003081B
:101A4000F001FFC0007F0000000000000000000067
:101A50000000000000000000000070380070380036
:101A600070380000000000000000000000000000CE
:101A70000000000000000000000000000000301A1C
:101A800000301C000000000000000000000000000A
:101A90000000000000000000000800001400002208
:101AA000000041000080800100400200200400107E
:101AB00008000800000000000000210000210000D4
:101AC0002100002100002100002100002100002150
:101AD00000002100002100000000000000000000C4
:101AE000080008040010020020010040008080006F
:101AF0004100002200001400000800000000000067
:101B00000003C00004C000040000080038080F38BB
:101B10000808380810000C300007E00003C000007F
:101B20000000000000003F8000FFE0038070020F13
:101B30001006708804C088048308047F8802C0905F
:101B400003012000FE400000080000180001F8001A
:101B50003E0801C20007020007E20000FE00001F6D
:101B6000C80001F800003800000804000807FFF86A
:101B700007FFF80408080408080408080408080611
:101B8000180803F41801E7F00001E000000000006D
:101B900000003F8001FFE00380700200180400088D
:101BA0000400080400080400100600200780C0009C
:101BB000000004000807FFF807FFF804000804000D
:101BC0000804000804001802001003807001FFE000
:101BD000007F8000000004000807FFF807FFF804FA
:101BE0000808040808040808040808043E0804005B
:101BF0000806001801006000000004000807FFF854
